:020000040800F2
:10000000F0FF01204990050875E3000859490408EC
:10001000C1900508C1900508C190050800000000C6
:1000200000000000000000000000000071E3000874
:100030006DE300080000000069E30008690D040892
:10004000C1900508C1900508C1900508C190050838
:10005000C1900508C19005082D840408F5830408A3
:10006000BD830408858304085577040829720508B0
:100070001972050809720508F9710508E571050886
:10008000D1710508BD710508C19005080000000088
:100090000000000000000000000000001D770408C0
:1000A000D1F503081DF60308C1F5030841F603085E
:1000B00011F6030801F60308F1F50308C1900508DD
:1000C000C1900508C1900508C1900508C1900508B8
:1000D000C1900508890E0408CD0D04080000000039
:1000E000E5760408C1900508B51701080000000076
:1000F000000000000000000000000000A9710508D9
:1001000000000000C1900508E1F50308C190050852
:1001100000000000000000000000000000000000DF
:1001200095710508817105086D71050859710508FB
:1001300045710508000000000000000000000000FC
:10014000000000000000000000000000D9F90008D5
:10015000317105081D71050809710508C190050870
:10016000C1900508C19005080000000000000000D3
:10017000000000000000000000000000000000007F
:1001800000000000C1900508000000000000000011
:08019000C1900508C1900508AB
:08019800E88B050001000000E6
:1001A0000B3001001A000000A437002074730020F7
:1001B0000000000040B806081F50010024000000A5
:1001C0006437002090730020000000005CB806082F
:1001D0000502010004000000CC700020B473002070
:1001E0000000000080B80608030101000A000000BA
:1001F000D0360020B873002000000000158E0008E3
:100200001302010004000000342C0020C4730020FD
:100210000000000084B806080D1001003400000042
:1002200014630020C873002000000000FD91030843
:1002300009020100010000002C700020FC73002066
:100240000000000088B80608F90101000400000061
:10025000D4620020007400200000000099E7030829
:10026000FB01010001000000185E00200474002062
:1002700000000000B9040508FC01010009000000AD
:10028000E45C00200874002000000000C904050898
:10029000F701010006000000D85C00201474002063
:1002A000000000008AB80608160215003F00000092
:1002B0009C3400201C740020000000006905050823
:1002C0003400010010000000085C00205C74002075
:1002D0000000000015530208110201000800000090
:1002E000E05B00206C7400200000000090B806085D
:1002F0001212010004000000D85B0020747400207A
:100300000000000098B80608183001003400000012
:10031000A45B00207874002000000000D9050508C7
:10032000FD01010021000000BC540020AC7400203D
:1003300000000000F3E60308000201000B000000CB
:10034000A04F0020D074002000000000ADF704088A
:100350002A02010008000000B0440020DC740020E4
:10036000000000009CB806082052010008000000B0
:1003700058440020E474002000000000813D020881
:1003800006100100240000004C330020EC74002013
:1003900000000000E50405080C0201000400000054
:1003A000183D00201075002000000000DDF7040853
:1003B000FE01010014000000986700201475002061
:1003C00000000000B5F70408010201000B00000066
:1003D000AC940020CCA90020000000009DF7040888
:1003E0000202010003000000A4940020D8A900200C
:1003F00000000000000000001B02010010000000CF
:1004000090940020DCA90020000000005DF80408A2
:100410001B1001000C000000608F0020ECA90020E0
:10042000000000004D53010821020100F00000000F
:10043000948D0020F8A90020000000007139010807
:1004400037100100300000007C990020E8AA00204D
:1004500000000000A4B806080E020100020000001F
:100460005C94002018AB002000000000D4B80608FF
:100470001610010006000000549400201CAB002060
:1004800000000000D6B806082F100100220000006E
:10049000A8A9002024AB002000000000DCB806085A
:1004A0002322010010000000A093002048AB002090
:1004B0000000000000B906081E000100090000004D
:1004C0009493002058AB00200000000010B90608EB
:1004D000052001000C000000B893002064AB002050
:1004E000000000001CB90608FD0701007C000000A8
:1004F0005E8C002070AB002000000000AD1E0108E3
:10050000F59101006C000000208D0020ECAB002074
:1005100000000000513801082320010010000000F5
:10052000DE98002058AC00200000000001C0010847
:1005300012200100110000007C93002068AC002014
:100540000000000028B90608F62101000C00000098
:1005500044BB0020ECBB0020000000003CB90608B2
:100560001C0202001C0000005CBB00203CBC002000
:1005700000000000890105081400010005000000CA
:1005800014BB002058BC00200000000048B9060839
:10059000012001000C000000C4B1002060BC00205C
:1005A000000000004EB906080C400600E400000000
:1005B000E8AF00206CBC00200000000039FF0208FA
:1005C0000A90010024000000A4AF002050BD0020CC
:1005D00000000000B9BF01080E300300BC0100009C
:1005E000E0AD002074BD002000000000415302086F
:1005F0001300010004000000C0B8002030BF00203C
:10060000000000005CB906080101010004000000C0
:1006100024AD002034BF00200000000000000000D6
:1006200000010100040000001CAD002038BF0020C4
:100630000000000060B9060802010100030000008C
:1006400018AD00203CBF00200000000079FF020828
:10065000220201001C010000A8B6002040BF0020BB
:1006600000000000710405081900010005000000E9
:10067000BCCA0020A0CB00200000000064B906081E
:100680001A0001000E00000000CA0020A8CB0020C4
:10069000000000006AB90608150010007000000094
:1006A0001CC80020B8CB00200000000000000000A3
:1006B0002A00080060000000FCCA002028CC0020AE
:1006C00000000000593D02082C000400100000004A
:1006D00098CC002088CC002000000000213B0208BC
:1006E0002B00120024000000CCCC0020A8CC00205D
:1006F00000000000F53A02082920140078000000EC
:100700000CC50020F0CC002000000000000000001C
:10071000190201001000000064C4002068CD002010
:10072000000000007DF704082902010040000000DD
:10073000C8CF002074D600200000000078B9060859
:100740000A0201001400000020D20020D4D60020AC
:100750000000000095090308F831010006000000C0
:1007600000D20020E8D6002000000000B8B906083A
:1007700003000100010000007CD30020F0D600201F
:100780000000000000000000101001000200000046
:100790000CD00020F4D6002000000000BEB90608EE
:1007A000020001000C0000002CD70020E8D8002037
:1007B000000000000000000025201E002C010000A9
:1007C00038D70020F4D8002000000000000000000E
:1007D000280204000400000080E1002058E400200A
:1007E0000000000059F8040827020400040000007B
:1007F0007CE100205CE40020000000004DF80408CB
:100800001F02080010000000B8DE002060E4002095
:10081000000000005DF704081A0201003C0000001F
:1008200060DA002070E400200000000035060508B2
:10083000031201003D00000008E30020ACE40020AA
:1008400000000000C0B906083810010001000000D7
:100850002CDA0020ECE4002000000000FEB90608BD
:1008600004000800800000007CE50020FCE500207A
:100870000000000000000000100201000100000064
:100880008CFF002088FF00200000000000BA06084E
:100890002B0201000B000000F0E6002090FF00207A
:1008A0000000000002BA06081D0202000600000057
:1008B00010FD00209CFF0020000000000000000050
:1008C000081203000F00000018FD0020A40A0120F8
:1008D00000000000F5F704082700010004000000F4
:1008E000CCEB0020B40A0120000000000EBA06087C
:1008F0000403090412010002EF020140830456328E
:100900000002010203010000120100020202004085
:100910008304405700020102030100000902640041
:10092000030100C032090400000103000000092196
:10093000110100012236000705830309000A080B94
:100940000102020201000904010001020201000586
:1009500024001001052401000204240202052406DB
:100960000102070582030800FF09040200020A00D1
:100970000000070501024000000705810240000059
:1009800009024300020100C0320904000001020212
:1009900001000524001001052401000104240202C5
:1009A0000524060001070582030800FF0904010071
:1009B000020A00000007050102400000070581024D
:1009C00040000000FF000000140000FF00000000D5
:1009D00000000000AA550701000001AA550501000A
:1009E000002D202D2D202D2D2D2D202D2D2D2D00B8
:1009F00000000000000000000000000000000000F7
:100A00000800000020B90508FF1FFF1F7D0000003F
:100A1000AD830008A9830008A58300089983000816
:100A200095830008A18300089D83000821840008A5
:100A300015840008ED83000801840008D9830008AC
:100A4000C5830008B1830008010000000000803F5A
:100A500005010905A101A10005010930093109328B
:100A6000093309350934093609371581257F750899
:100A70009508810205091901290815002501950825
:100A800075018102C0C0000009022200010100E0DE
:100A900032090400000103010200092111010001D3
:100AA0002236000705830309000A000000600240A7
:100AB0001060024000000000000000000000000084
:100AC000000B00000000000000000000000000001B
:100AD00000600240286002400100000000000000A9
:100AE00000000000060C00000000000000000000F4
:100AF0000000000000600240406002400200000070
:100B00000000000000000000100D000000000000C8
:100B10000000000000000000006002405860024039
:100B2000030000000000000000000000160E00009E
:100B30000000000000000000000000000060024013
:100B4000706002400400000000000000000000008F
:100B5000200F000000000000000000000000000066
:100B600000600240886002400500000000000000B4
:100B7000000000002610000000000000000000003F
:100B80000000000000600240A0600240060000007B
:100B90000000000000000000301100000000000014
:100BA000000000000000000000600240B860024049
:100BB000070000000000000000000000362F0000C9
:100BC000000000000000000000000000006402407F
:100BD000106402400000000000000000000000005F
:100BE00000380000000000000000000000000000CD
:100BF0000064024028640240010000000000000080
:100C000000000000063900000000000000000000A5
:100C10000000000000640240406402400200000046
:100C20000000000000000000103A0000000000007A
:100C30000000000000000000006402405864024010
:100C4000030000000000000000000000163B000050
:100C500000000000000000000000000000640240EE
:100C6000706402400400000000000000000000006A
:100C7000203C000000000000000000000000000018
:100C8000006402408864024005000000000000008B
:100C900000000000264400000000000000000000EA
:100CA0000000000000640240A06402400600000052
:100CB00000000000000000003045000000000000BF
:100CC000000000000000000000640240B864024020
:100CD0000700000000000000000000003646000091
:100CE0000000000000000000000000000000000004
:100CF00001020304010203040607080921E50008B4
:100D0000D9EB000851E70008C5840008A58A00084F
:100D1000D5840008F18400089D8400088D840008B3
:100D20000000000000000000AA550B010000AA55B9
:100D300005010000AA550902000000AA5503009F02
:100D400001000000C01200006C73002000000000D1
:100D500044730020000000000100000000000100BA
:100D6000E0017EFFFFFFFFFFFF000000FFFFFFFF2E
:100D700008FF000014340608903306080000000045
:100D800001000308A086010004000000000000002C
:100D90000000000000000000000000000000000053
:100DA0000000000000000000000000000000000043
:100DB0000000000000000000143406081C3406087F
:100DC0000000000085E50308E803000004000000BF
:100DD0000000000000000000000000000000000013
:100DE0000000000000000000000000000000000003
:100DF000000000000000000000000000243406088D
:100E000000000000000000002D0703087D00000026
:100E1000FF000000000000000000000000000000D3
:100E200000000000000000000000000000000000C2
:100E300000000000000000000000000000000000B2
:100E4000C4B406080000000000000000F914030804
:100E50007D000000FF000000000000000000000016
:100E60000000000000000000000000000000000082
:100E70000000000000000000000000000000000072
:100E800000000000D8430608000000000000000039
:100E9000655B03087D000000FF000000000000000B
:100EA0000000000000000000000000000000000042
:100EB0000000000000000000000000000000000032
:100EC00000000000000000002C34060800000000B4
:100ED000000000005DEB0308E803000003000000D1
:100EE0000000000000000000000000000000000002
:100EF00000000000000000000000000000000000F2
:100F0000000000000000000000000000303406086F
:100F1000000000000000000071CE02081027000051
:100F200003000000000000000000000000000000BE
:100F300000000000000000000000000000000000B1
:100F400000000000000000000000000000000000A1
:100F50009CB006080000000001370208BD490408E3
:100F60005F760000050000000000000000000000A7
:100F70000000000000000000000000000000000071
:100F80000000000000000000000000000000000061
:100F90000000000068B40608000000000000000027
:100FA0008D770408102700000100000000000000F9
:100FB0000000000000000000000000000000000031
:100FC0000000000000000000000000000000000021
:100FD00000000000000000003C3406080000000093
:100FE0000000000089E50308E80300000500000098
:100FF00000000000000000000000000000000000F1
:1010000000000000000000000000000000000000E0
:101010000000000000000000000000004834060846
:101020000000000000000000E50B0308204E000057
:1010300003000000000000000000000000000000AD
:1010400000000000000000000000000000000000A0
:101050000000000000000000000000000000000090
:10106000583406080000000000000000D109030801
:10107000204E0000030000000000000000000000FF
:101080000000000000000000000000000000000060
:101090000000000000000000000000000000000050
:1010A0000000000068340608000000000000000096
:1010B000A9E70308400D0300030000000000000042
:1010C0000000000000000000000000000000000020
:1010D0000000000000000000000000000000000010
:1010E0000000000000000000783406080000000046
:1010F0000000000011AF03081027000001000000ED
:1011000000000000000000000000000000000000DF
:1011100000000000000000000000000000000000CF
:10112000000000000000000000000000BC330608C2
:101130000000000000000000F995010810270000E1
:10114000030000000000000000000000000000009C
:10115000000000000000000000000000000000008F
:10116000000000000000000000000000000000007F
:1011700080340608000000000000000061E403085D
:10118000A861000001000000000000000000000055
:10119000000000000000000000000000000000004F
:1011A000000000000000000000000000000000003F
:1011B000000000008C340608000000000000000061
:1011C00051130408A00F00000100000000000000FF
:1011D000000000000000000000000000000000000F
:1011E00000000000000000000000000000000000FF
:1011F0000000000000000000983406080000000015
:101200000000000015820108102700000100000006
:1012100000000000000000000000000000000000CE
:1012200000000000000000000000000000000000BE
:10123000000000000000000000000000A4340608C8
:101240000000000000000000D17901081A410000F0
:10125000010000000000000000000000000000008D
:10126000000000000000000000000000000000007E
:10127000000000000000000000000000000000006E
:10128000A83406080000000000000000498E000895
:101290001027000001000000000000000000000016
:1012A000000000000000000000000000000000003E
:1012B000000000000000000000000000000000002E
:1012C00000000000A4330608000000000000000039
:1012D000F504020850C300000100000000000000F7
:1012E00000000000000000000000000000000000FE
:1012F00000000000000000000000000000000000EE
:101300000000000000000000B434060800000000E7
:1013100000000000AD9C0008400D0300000000002C
:1013200000000000000000000000000000000000BD
:1013300000000000000000000000000000000000AD
:10134000000000000000000000000000BC3406089F
:101350000000000000000000B9910308400D0300E8
:10136000000000000000000000000000000000007D
:10137000000000000000000000000000000000006D
:10138000000000000000000000000000000000005D
:10139000C43406080000000000000000E1A50108B8
:1013A00050C3000003000000000000000000000027
:1013B000000000000000000000000000000000002D
:1013C000000000000000000000000000000000001D
:1013D00000000000D03406080000000000000000FB
:1013E0006152030840420F000000000000000000AE
:1013F00000000000000000000000000000000000ED
:1014000000000000000000000000000000000000DC
:101410000000000000000000DC34060800000000AE
:10142000000000005192030850C3000000000000BB
:1014300000000000000000000000000000000000AC
:10144000000000000000000000000000000000009C
:10145000000000000000000000000000E834060862
:101460000000000000000000A96201081027000031
:10147000000000000000000000000000000000006C
:10148000000000000000000000000000000000005C
:10149000000000000000000000000000000000004C
:1014A00001FF01000100000099B5010800000000E3
:1014B0000000000038C205085CB30020B0B3002073
:1014C000000000000000000000000000DCDA050859
:1014D00000000000000000000000000094DB050890
:1014E00000000000000000000000000040DB0508D4
:1014F000000000000000000079D2010802B50020C1
:10150000FF010100DDF00108000000000000000004
:1015100068DC05083DF40108000000000000000040
:1015200020DC05082D202D2D202D2D2D2D202D2DBD
:101530002D0000000000000000000000000000007E
:1015400000000000FFFFFFFF35D801080000000089
:10155000000000006CDA050801000000FA0000003D
:101560000100000001000000010100000001010174
:10157000000000002EB100200000F4010100000076
:101580002CB100200000F401010000002AB100206D
:101590000000F4010100000028B100200000F40167
:1015A0000100000026B100200000F401010000004D
:1015B00024B100200000F4010100000022B100204D
:1015C0000000F4010100000041BE010805BE010851
:1015D000000000007CC4050812B1002005320100A3
:1015E00020B100206400F401010000001EB10020C1
:1015F0006400C4090100000010B10020E803D00716
:10160000010000000EB10020E803D0070100000037
:101610000CB10020E803D007010000000AB100204F
:101620001E00B80B0100000018B1002005000F00DB
:10163000010000001AB1002003000A0001000000B0
:1016400008B100201E00F401010000001CB10020C0
:101650000200000008C5050806B10020140064005F
:101660000100000014B100203200E8030100000076
:1016700004B100200000C80001000000E5AF002018
:1016800000C80100E4AF002000500100E3AF0020DB
:10169000005A0100E1AF00200200000014C5050857
:1016A000803A0608883A060800B500200100C409FF
:1016B00000000000FEB400200100C409000000008A
:1016C000FCB400200100C40900000000FAB40020AE
:1016D0000100C40900000000F6B400200100C409A4
:1016E00000000000F8B400200100C4090000000060
:1016F000F4B400200100C40900000000F2B400208E
:101700000100C4090000000043AD002000C8010032
:1017100042AD002000C8010040AD00200000FFFFE6
:101720000A0000003EAD00200100C80001000000DA
:101730003CAD002032003075320000003AAD002090
:101740007EFF14000500000038AD002005002C01CC
:101750000500000037AD0020055A050034AD00201B
:1017600000FF010036AD002002000000480F0020FD
:1017700032AD00200300000020BB050833AD00207F
:1017800000FF010035AD002002000000480F0020DE
:1017900031AD00200300000020BB050890AC002004
:1017A000FF7F01008CAC002000000000FFFFFFFF66
:1017B0000100000088AC002000000000FFFFFFFFD8
:1017C0000100000084AC002000000000FFFFFFFFCC
:1017D0000100000095BD010825BD010800000000C2
:1017E00020C50508D4B10020EE02CA08010000009F
:1017F000D2B1002000C8010064000000D1B1002077
:1018000000C8010064000000D0B100200200000008
:101810002CC605082AAD00200000803E050000000F
:1018200028AD002080C1803E0500000022AD0020D0
:101830000083007D0500000020AD002080C1803EB7
:10184000050000001BAD002000FF010014AD0020CA
:101850006400F4010100000012AD00206400F401F6
:101860000100000010AD00206400F4010100000040
:101870000EAD00200400000038C605080DAD0020A4
:10188000020000004CC60508CFAD00200D0000008E
:1018900058C60508CCAD002000640100CAAD002088
:1018A000320010270A000000C8AD00200D00000023
:1018B00058C60508C7AD00200D00000058C6050831
:1018C000C6AD00200200000090C60508D9B1002076
:1018D000440000009CC60508D7B1002003000000AA
:1018E000B0C70508D8B1002004000000C0C7050833
:1018F000D1AD002003000000D4C70508D0AD002002
:1019000003000000D4C70508D2AF0020000A010080
:10191000D0AF00200000E80301000000CEAF00209F
:101920000000E80301000000CCAF0020000A010025
:10193000CAAF00200000E80301000000C8AF00208B
:101940000000E803010000009CAF00200000E80355
:1019500001000000A2AF00200000E8030100000029
:10196000A0AF00200100E803010000009EAF0020AE
:1019700001050100E0AF002002000000E4C70508F7
:10198000DEAF00200000F40101000000DCAF002009
:101990000000F40101000000DAAF00200000F401B3
:1019A00001000000D8AF00200000F4010100000099
:1019B000D6AF00200000E80301000000D4AF0020F3
:1019C0000000E80301000000F2B000200064010004
:1019D0000A000000F1B00020006401000A000000CD
:1019E000DFB0002019640100DEB00020020000001A
:1019F000F0C70508DCB00020E803D0070A000000AB
:101A0000DAB00020006401000A000000CFB000201E
:101A100000640100CEB0002000640100D6B00020B8
:101A2000006401000A000000D5B00020006401003D
:101A30000A000000D4B00020006401000A00000089
:101A4000D9B0002000FF01000A000000D8B000203B
:101A500000FF01000A000000D7B0002000FF0100D5
:101A60000A000000D3B0002001FF01000A000000BE
:101A7000D2B0002001FF01000A000000D1B0002018
:101A800001FF01000A000000DAAD00200000F401AF
:101A900001000000D8AD00200000E80301000000B4
:101AA000D6AD00200000E80301000000D4AD002006
:101AB0000000E80301000000D2AD00200000E803B0
:101AC0000100000053B50020009601004AB5002037
:101AD00000C8010049B500200064010048B500209D
:101AE0000064010047B500200064010046B50020F5
:101AF0000064010045B50020FF08010044B5002046
:101B00000164010015BC0108D9BB010800000000F8
:101B1000FCC705084DB50020013201004CB500207E
:101B2000010000006CC805084BB50020040000004F
:101B300074C8050843B500200096010042B5002096
:101B40000064010040B500201400E803010000001B
:101B50003EB50020000030750A0000003CB50020B2
:101B600000C801003BB5002000C801003AB50020C4
:101B700000C8010050B500200032010052B500201D
:101B80000014010051B50020004B01004FB50020AA
:101B90000400000088C805084EB50020006401005C
:101BA0000A000000FEB0002000C805000A00000086
:101BB000FDB000200100000098C8050800B1002019
:101BC00000C805000A000000FFB00020010000006E
:101BD00098C80508FCB0002000C805000A000000F5
:101BE000F6B0002000C805000A000000FAB000208E
:101BF00000C805000A000000F7B0002000C805007A
:101C00000A000000FBB0002000C805000A00000028
:101C1000F8B0002000C805000A000000F9B000205C
:101C200000C805000A000000F5B0002000C805004B
:101C30000A000000F4B0002002000000A0C805085F
:101C400062B500200000D007010000005CB5002054
:101C500000C801005BB5002000C801005AB5002093
:101C600000C8010060B500200000D007010000009E
:101C700059B5002000C8010058B5002000C8010077
:101C800057B5002000C801005EB500200000D00755
:101C90000100000056B5002000C8010055B5002025
:101CA00000C8010054B5002000C80100A9B901080E
:101CB00091B9010811D80108ACC80508C3AD0020CE
:101CC000005A0100C2AD002000C80100C0AD0020D4
:101CD000E803D00701000000000000000000000041
:101CE000B9D2010848C9050830AD00200300000042
:101CF00090C905082FAD0020000301002EAD002083
:101D000000030100CDB8010881B8010800000000FF
:101D1000A0C9050841B80108F9B701080000000092
:101D20003CCA050819B90108F5D7010800000000F0
:101D3000BCCA05082CAD00200103010065B50108EF
:101D400045B501080000000030CE050801BF0108BC
:101D5000D5BE010800000000B0CE050869B7010833
:101D600011B701080000000020CF0508B9B901082B
:101D7000F1FB010800000000D8CF050865D3010879
:101D80002DBF01080000000080D0050809BA010835
:101D900000000000000000000CD10508EDBA0108A9
:101DA0008DBA01080000000070D1050895BB01083C
:101DB00051BB01080000000028D205087930020854
:101DC00051BC010800000000B4D2050802B1002097
:101DD0000106010051BA01081DBA01080000000007
:101DE000CCD30508952F0208B9D9010800000000DE
:101DF0003CD4050881BC0108D9DA010800000000C4
:101E0000B8D50508BD30020899DA010800000000C5
:101E1000C4D6050801B100200103010061B9010821
:101E200031B901080000000098D7050895D70108CE
:101E30000000000000000000FCD70508C1B7010841
:101E4000DDD701080000000098D805080000000058
:101E5000000000000000000034D90508FDBC0108A6
:101E600015DC010800000000B4D9050800000000DE
:101E70000000000000000000DCDB0508283700201F
:101E80009CFF2C010000000058B80020E0150C1742
:101E9000000000005AB800200200000014DC050811
:101EA00008AD002088136F17010000000AAD002064
:101EB00088136F1700000000C236002000000000E9
:101EC00000000000C03600200000000000000000FC
:101ED000BE3600200000000000000000BC360020DC
:101EE0000000000000000000BA36002000000000E2
:101EF00000000000B83600200000000000000000D4
:101F0000EC050020000000000000000091AC002063
:101F10000300000004DD050800AD002088136F17E2
:101F200001000000C270002088136F17000000003D
:101F300051B60108000000000000000014DD050893
:101F4000BDB400200100000068DD0508C470002059
:101F50000100000074DD0508BA70002002000000D6
:101F60007CDD05080000000000000000000000000B
:101F700088DD050839B601080000000000000000F7
:101F800024DE050800000000000000000000000042
:101F900078DE0508000000000000000000000000DE
:101FA000E8DE05080CAD00200200000020DF050877
:101FB000BE700020E0150C170000000001F11F3F6B
:101FC00001D6010128750020FFFFFFFF0000803FC0
:101FD0000000000000000000000000000000000001
:101FE00000000000000000000000000000000000F1
:101FF000000000000000803F000000000000000022
:10200000000000000000803F000000000000000011
:10201000000000000000803F000000000000000001
:1020200000000000010000000000FA430000FA4335
:1020300021B10308000000000000000000000000C3
:1020400060FECD0000000000C4D6002008000000A3
:1020500000000000B4D60020080000000000803F0F
:10206000718A00085189000831E70008000000006B
:1020700089840008EDE40008C988000861E40008CC
:10208000000000000000000049840008E189000809
:102090001189000881E60008000000006184000842
:1020A00065E400089D880008BDE30008000000000A
:1020B0000000000055840008FFFFFFFF0100000042
:1020C000A00F0000B80B00000102FFFF01FF00009D
:1020D000FFFFFF0090B006080000080205030300A0
:1020E0000000000098B00608010008020504030083
:1020F00000000000305C06080200FE010110030031
:1021000000000000E03D0608030014020003000088
:1021100000000000A0B0060804001F020200080032
:1021200000000000A8B0060805001F020201080018
:1021300000000000FFFFFFFF00010000204E000034
:102140000000000000000000000018500600000021
:10215000D007000001040C97A0252600010118609B
:1021600007000000A00F000002040E94C0C62D005E
:1021700002031870070000000A1A000003040C9004
:10218000E06735000305189006000000204E0000AF
:1021900000040C8B00093D00000004010000020057
:1021A0000100000210000000070001FF0100000014
:1021B000F4010000A02E060800000000000000004E
:1021C000000000000100000000000000000000000E
:1021D00000000000000000000100000000000000FE
:1021E00000000000000000000102030406070809C7
:1021F00001FF0000A01A0020000000000000000005
:1022000000000000000000000000000000000000CE
:1022100000000000000000000000000000000000BE
:1022200000000000000000000000000000000000AE
:10223000000000000000000000000000000000009E
:10224000000000000000000000000000000000008E
:08225000000000000000000086
:082800000000000000000000D0
:108000002DE9F04700230F6801264FF0030C02E032
:108010000133102B41D006FA03F232EA0704F7D1FC
:10802000D0F800E05C000CFA04F52EEA050EC0F86A
:1080300000E091F80490D0F800A009FA04FE09F1DC
:10804000FF394EEA0A0EB9F1010FA846C0F800E068
:108050006FEA050515D8D0F808E005EA0E05856039
:108060004D79D0F808E0A54045EA0E0585604568E1
:1080700025EA020242608A7945689A4092B22A4310
:108080004260C26822EA0802C260CA79C568A2409A
:1080900001332A43102BC260BDD1BDE8F08700BF79
:1080A000037830B403B30246C0F10105531912F846
:1080B000014FDBB2002CF9D101335B00DAB20C4C7A
:1080C0000B80032322706370017859B102230025CD
:1080D0005A1CD2B2E154A55410F8011F0233DBB28E
:1080E0000029F5D130BC704702221346E7E700BFF4
:1080F000001B0020084AD2E9403199420AD0D11829
:10810000013391F808110170C3F30A03C2F800317A
:108110000120704700207047001B0020064AD2F85B
:108120000839D2F80C29934294BF4FF40060002024
:10813000013B9B1A18447047001B0020012380F864
:108140005130704707B501A8FFF7D4FF0028FAD0D7
:108150009DF8040003B05DF804FB044BD3E9400331
:10816000984288BF03F50063181A7047001B00206F
:1081700001207047024BC3F81029C3F81419704747
:10818000001B0020024BC3F81829C3F81C197047C4
:10819000001B00207047704730B4134DD5E94023D1
:1081A0009A4286BF03F50064A21A9A1A0A44B2F5ED
:1081B000006F13D8A9B101444A1E013810F8014FCD
:1081C000E918824203F1010381F80841C3F30A036D
:1081D000F4D1C5F80431002030BC7047022030BC17
:1081E00070470846F8E700BF001B0020F8B51A4C9E
:1081F00094F82039002BFBD159B301444E1E451E83
:10820000D4F80C29D4F8081915F8017F531CC3F3CE
:108210000A038B422CBF4FF400600020C91A22448D
:1082200001440129C4F80C3982F824790FD10120C6
:1082300038F0F6FCD4F80839D4F80C198B4294BF06
:108240004FF4006200225B1A1344012BEFD0B542B9
:10825000D6D10020F8BD00BF001B002010B5074C90
:10826000E36A0846114643B1E36A052B05D1002AAB
:10827000236B02DDFFF7BAFF236B10BDF82B002044
:1082800010B590F85010002380F8503061B1094CBF
:10829000E26A5AB1E26A052A0AD13C30236BFFF741
:1082A000A5FF236B012010BD0120FCE71046FAE773
:1082B0001846F8E7F82B0020002280F85120DFE76D
:1082C00090F85020531C0244DBB280F8503082F802
:1082D0003C1090F851200AB1132B00D9D0E7704719
:1082E000212838B50C4605D022282DD0202812D0C0
:1082F000002038BD0029FBD0072AF9D1194B586B53
:1083000093F8381093F8392093F83A3020602171AF
:108310006271A371ECE70029EAD0072AE8D1124A7A
:10832000D2F814391BB1D2F81009096898470D4BDF
:10833000256820796179A2795D6383F8380083F834
:10834000391083F83A20D3E70029D1D0022ACFD1BF
:10835000054AD2F81C39002BCAD00988D2F818096E
:108360009847C5E7F82B0020001B0020014B002098
:10837000D8627047F82B0020044B054A00200521E5
:10838000D162C3F81C09C3F814097047001B002010
:10839000F82B0020704700BF704700BF704700BF38
:1083A000704700BF704700BF704700BF704700BFF5
:1083B00008B50248FFF774FE014808BDD42E060830
:1083C000001B002008B50248FFF76AFE014808BDFF
:1083D000E42E0608001B002008B50248FFF760FEE7
:1083E000014808BDF02E0608001B002008B5024811
:1083F000FFF756FE014808BDFC2E0608001B0020B2
:1084000008B50248FFF74CFE014808BD082F0608D2
:10841000001B0020042301480B80704798010020B6
:1084200010B4074A074B92F83C00122403F11402DF
:108430000C8001280CBF184610465DF8044B7047AD
:10844000F82B00209C010020642301480B8070471A
:10845000C4010020432301480B80704728020020FC
:1084600010B5074CD4F8D400FF2807D005490A6C92
:108470004431FFF735FFFF23C4F8D430002010BD8E
:1084800098010020F82B0020EAE700BF08B5D0F8DB
:10849000E4355B6A9847002008BD00BF08B5D0F8F6
:1084A000E4351B6A9847002008BD00BFD0F8E435CA
:1084B00010B504461B689847D4F8E8359B68984780
:1084C000002010BD08B5D0F8E435DB6903B198474A
:1084D000002008BD08B5042290F81211D0F8E83544
:1084E00080F8131180F81221DB689847002008BD3E
:1084F00010B5D0F8E83504461B699847032384F883
:108500001231002010BD00BF0B0617D401EB810310
:1085100000EBC30310B400EB81000124002283F8B8
:10852000764383F8741383F87523426D5DF8044B2A
:10853000136843F4001300201360704701F07F01BB
:1085400001EB810300EBC303012200EB810083F800
:108550001C1183F81E2183F81D2182691368002BEA
:1085600001DA43F0804343F40013136000207047A6
:1085700082B00023016801930B6901930E4B03E065
:108580000A690192013B13D0019A002AF8DA019A94
:10859000094B42F001020192019A0A610A690192B3
:1085A00003E00A690192013B02D0019AD207F8D494
:1085B000002002B0704700BF400D0300436D064A23
:1085C0001A61C278012A06D100F2CC5058614FF0EE
:1085D000802219681A6070471800086010B5802161
:1085E0000446FFF791FF20460021FFF78DFF20464C
:1085F000BDE81040E2E700BF70B44B78012B26D0F5
:108600000B784A6900EB83035C6D25682369D2B15E
:108610008A684A6102F07F0223F4002323F07F037B
:1086200042F4002213432361C378012B04BF0B697A
:108630006361C5F3076363F07B0363F31F65256024
:10864000002070BC70478A6802F07F02E4E782690C
:108650004C691568136944B38E68B4428CBF06F048
:108660007F0404F07F0423F4002323F07F0344F409
:10867000002443EA040388BF4E611361C378012BD1
:108680001DD0C5F3076464F07B0464F31F651560B7
:10869000002BD5D14B69002BD2D002690878516BE1
:1086A000012383400B435363CAE723F4002323F0E1
:1086B0007F0343F400231361C378012BE1D10B78CE
:1086C0000C6900EB8300C5F30763816963F07B03EA
:1086D00063F31F654C610020156070BC704700BFDC
:1086E0002DE9F0434B78012B30D00B784C6900EB2F
:1086F00083035E6D356837691CB38B681C44013C8D
:10870000B4FBF3F4C4F3090203FB02F3C3F3120353
:108710004B61144643EAC44363F31C073761C378D3
:10872000012B04BF0B697361CB78012B44D0C5F3D7
:10873000076363F07B0363F31F6535600020BDE8CA
:10874000F0838A680124C2F31203E3E791F8008002
:108750004E6900EB880EDEF818C0DCF80050DCF83B
:10876000107076B3D1F80890384A06EB0904013C42
:10877000B4FBF9F402EAC444C6F312022243CC78F3
:1087800007F060473A43012C174649D0CCF8102037
:10879000C278012A55D00269516B03FA08F30B43E2
:1087A0005363C5F3076363F07B0363F31F65CCF882
:1087B00000500020BDE8F0834B7973B345F00055BD
:1087C000B5E707F0604747F40027CC78CCF8107085
:1087D000C378012B2FD0012CE3D102699268D20516
:1087E00054BF45F0005545F08055C5F3076262F06F
:1087F0007B0262F31F65CCF80050002B9ED1B0B213
:1088000003308010DEF8D04098D0CA6852F8041BBC
:10881000216001339842F9D190E745F0805586E711
:1088200064F35E77CCF81070C378012BD5D10A6958
:10883000CCF81420D1E70A69CCF81420012CB0D16F
:10884000CBE70B69CCF81430ABE700BF0000F81F92
:1088500038B501EB810400EBC4040D46002184F817
:108860007453C4F88C1384F87513C4F88833C4F8AF
:108870008023C3782821012B01FB050108BFEDB23D
:1088800001F55D7108BFC4F884231DB9FFF7B4FE7C
:10889000002038BDFFF724FF002038BD10B501EBE4
:1088A0008101084A00EBC1010446B1F88C1310465F
:1088B000FFF772FC034A204640230121FFF7C8FF5F
:1088C000002010BD442C0020E8E700BF30B44C78F5
:1088D0000022012C154612D0097800EB81040123F7
:1088E0008B40646D63F31F4501696FF3CF322260E3
:1088F000CB6923EA0503002030BCCB6170470B78BD
:1089000000EB83019C4064F30F058C69ECE700BF2A
:1089100040F2011310B500F5A2710446A0F84431ED
:10892000FFF7D4FF0123A4F89C3304F567712046B8
:10893000FFF7CCFF4FF48173A4F86C3104F5B671E6
:108940002046FFF7C3FFFFF711FD002010BD00BF59
:1089500038B540F2031304460D46A0F8943100F5F3
:10896000CA71FFF7B3FF29462046FFF7D1FF002069
:1089700038BD00BFF0B44B780A78012B4FF00004EB
:1089800000EB820524D0012393406D6D63F31F44F7
:108990002E68330415D48A6891F803C0CF880F4934
:1089A000C2F30A0242F0805343F400430CF0030286
:1089B00043EA824307F00F0243EA825331400B43FC
:1089C0002B600369DA691443DC610020F0BC704756
:1089D0009340AD6963F30F04DAE700BF007833EC2E
:1089E0002DE9F04140F20113044602254FF0400802
:1089F00001270026A0F84431C0F84C8180F8475187
:108A0000A0F84A7180F8486100F5A271FFF7B2FF43
:108A100004F56771A4F89C73C4F8A48384F89F5389
:108A200084F8A0632046FFF7A5FF082203234FF434
:108A30008171C4F87421A4F86C1184F86F3104F5C5
:108A4000B671A4F872512046FFF794FF064B9D8340
:108A5000FFF792FC054A434620463946FFF7F8FEE9
:108A60003046BDE8F08100BF98010020442C002072
:108A700070B50323092240F2031604460D46C0F8E0
:108A80009C2180F89731A0F89A31A0F8946100F504
:108A9000CA71FFF76FFF29462046FFF7A1FF0020AC
:108AA00070BD00BF70B5002540260446A0F8745381
:108AB00080F87753C0F87C6300F55D71FFF75AFFCB
:108AC0004FF48073A4F81C3104F58E71C4F824614E
:108AD00084F81F51A4F822512046FFF74BFFD4F829
:108AE000E835A078012284F812215B68984728466F
:108AF00070BD00BF82B000230193019A094B42F080
:108B000010020192C168019A0A610A69019203E0A8
:108B10000A690192013B02D0019AD206F8D40020E2
:108B200002B07047400D030082B000230193019A08
:108B30000B4B42F020020192019A61F38A120192DA
:108B4000C168019A0A610A69019203E00A69019207
:108B5000013B02D0019A9206F8D4002002B070477F
:108B6000400D03000E4BDA68D20310D4DA68D10648
:108B70000FD4DA68D20510D4DA6812F0E00F0AD107
:108B8000DB6813F0020F14BF082009207047012092
:108B9000704706207047072070470220704700BFCB
:108BA000003C024000207047134AD2F88C00C8B144
:108BB000D2F89030B3B1884212D88B4234BF002330
:108BC0000123DBB25BB1D2F89830C2F8941099421D
:108BD00005D00A4BC2F89810142083F8D8007047CB
:108BE0000023EEE7A1F59C53083BB3F57A7F2CBF39
:108BF00000230123E6E700BFF82B002098010020A6
:108C0000064B93F89D2083F89C108A4205D0044AB5
:108C100083F89D10142082F8D8007047F82B0020AC
:108C200098010020704730B1034B93F89E00012853
:108C300094BF002001207047F82B002008B5FFF7F3
:108C4000F2FF60B1064A92F89F3092F89C205B00D8
:108C500003F00203002A18BF43F001030B6008BDB4
:108C6000F82B002008B5FFF7DEFF18B1024BD3F850
:108C7000A0300B8008BD00BFF82B002070B5FFF7B7
:108C8000D2FF60B10B4AB2F8A4503DB1D2F8A8604F
:108C90000023B3421C4603DB002000E00D7070BDD2
:108CA00002EB44040133B4F8AC40AC42DBB2F0D187
:108CB0000B70F4E7F82B002008B5FFF7B4FF10B1F4
:108CC00000230B70137008BD0420704728B1034BBC
:108CD00093F9DA00003818BF01207047980100208E
:108CE00008B5FFF7F3FF50B1054B93F9DA20012ADD
:108CF000C3BF93F8DD30C3F340030B60002008BD11
:108D00009801002008B5FFF7E1FF18B1024B93F876
:108D1000DC300B7008BD00BF9801002070B5FFF774
:108D2000D5FF38B10E4C94F8DD30DB0703D50023B6
:108D30000B70137070BD0B4D94F9DB3095F8BC606F
:108D400093FBF6F301330B7094F9DB4095F8BC10FC
:108D500094FBF1F301FB134301331370EAE700BF07
:108D600098010020F82B00200320704770B50A4AB4
:108D700092F8C03006255E1CB6FBF5F405FB1464C2
:108D800092F8C150AC4205D002EBC303C3E93101F4
:108D900082F8C04070BD00BFF82B0020002230B523
:108DA00004461046914200DC30BDA35C08255840C3
:108DB00010F0800F4FEA400318BF83F0D503013D48
:108DC000D8B2F5D10132EDE710B5E9B10F4BD3F8C8
:108DD000F400814218DCBAB1D3F8BC309A4213DCFB
:108DE0000B4C013A013903FB012184F8E81004F12E
:108DF000E4000521FFF7D2FF062184F8E90004F121
:108E0000E400BDE81040B1E710BD00BFF82B002022
:108E1000980100200023038083708380C380037245
:108E2000704700BF074A92F8F83092F8FC100133FF
:108E3000DBB2994282F8F83004BF002382F8F830A0
:108E4000704700BFF82B0020F8B5794CD4F84832B1
:108E500083B1D4F84C3293F82E305BB1754B94F853
:108E60005022A3FB0013012A4FEA931330D0022AA9
:108E700008D002B1F8BD704B9842FBD9012384F8A9
:108E80005032F8BDD4F8542264329A423ED894F855
:108E9000F83004EB031393F8D426FF2A06D0674971
:108EA0000132012083F8D42681F8EA00FFF7BAFFE7
:108EB00094F8C8360122092B84F85022DAD1B4F88C
:108EC0007A3713449BB2A4F87A37A4F8CE36F8BDAB
:108ED00094F8F810C4F854328C2303FB014394F83F
:108EE000C80683F86A22002604F517750A220223B1
:108EF000092884F86662C4F8585284F8672284F816
:108F00005032B7D10131A4F8CC16F8BD94F86622DE
:108F100094F867329A42ADD104F25B2004F51975DA
:108F2000002310F8012F082153405A0013F0800F3E
:108F300008BF5B0082F0070214BFD3B2DBB2013975
:108F4000F3D18542EDD194F865229A4239D194F853
:108F5000F860B4F85F5294F86372B4F8610294F860
:108F6000643294F85DC204EB06126DBA40BA43EA6B
:108F70000723ADB294F85E7282F8D416C2F8D856C0
:108F800081B22E4D94F95C02C2F8DC1647EA0C2738
:108F90001BB20121032EA2F8D676A2F8E03682F8A1
:108FA000D50685F8EA1009D894F8C8260C2A2AD0E4
:108FB0000D2A03D104EB4606A6F8CC06FFF732FFD4
:108FC0005CE794F8F83004EB031393F8D426FF2AF7
:108FD00006D01A490132012083F8D42681F8EA002C
:108FE000FFF720FF94F8C8360122092B84F850229D
:108FF0007FF440AFB4F8783713449BB2A4F87837C5
:10900000A4F8D036F8BD94F876170D4A03EB830325
:1090100003EB830349089B0004EB460693FBF1F343
:1090200082FB0312DB17C3EBA203A6F8CC36C5E71D
:10903000F82B0020D34D62103F4B4C0098010020CC
:10904000676666660B4B93F8661293F86722914247
:109050000ED010B493F86622D3F85842511CD2B205
:10906000C0B2C9B283F86612A0545DF8044B7047D1
:10907000704700BFF82B0020FD2870B522D0F028E3
:1090800004D0EF2822D00224204670BD114D0320C9
:10909000052641282E444FF0000405F1010580F01B
:1090A00080030DD0042B0BD9FFF7E6FF2044B54217
:1090B000C4B2E9D015F8010B412880F08003F1D14A
:1090C0000420F3E7044D0B200426E2E7034D0C20B7
:1090D0000626DEE774B7050870B705087CB70508F3
:1090E0000C4AD2F8903730B41C68D2F888575D60CB
:1090F00019810025611C19609D812070D2F890377C
:10910000D2F888171A685A604FF6F67230BC1960A8
:109110009A817047F82B0020144B30B4D3F8944751
:1091200014B300220F2583F89A17090A83F89907C8
:1091300083F89B17C3F89C27C3F8A027C3F8A4277C
:1091400083F8985703F5F360012110F8015F0131AE
:109150002A440E29D2B2F8D183F8A6272046044922
:1091600030BC102238F0BCB830BC7047F82B00205F
:1091700090330020034B002183F8A817C3F8AC17E5
:10918000CAE700BFF82B00202DE9F04FCF4ED04D9D
:1091900086468C4617460FCE05F5F6642DED068BF8
:1091A0000FC40FCE0FC496E8070089B095F8563764
:1091B000039784E80700CDE904EC042B00F2488112
:1091C000DFE813F0B401460141010500C4019FED41
:1091D000C18ADFEDC18AC149C5F8CC17C049C14B6E
:1091E000C14AC5F8C8170399002918BF134638EEBD
:1091F000887AF5EE006AC6EE879ABC4EC5F8D43779
:10920000A6F17E0B06F1C0080027DFEDB97A9FEDCD
:10921000B99A28EE278AB0EE67AA059BBB4200F0F8
:109220000C811BF8013BEA1892F85B47002C00F018
:109230001481002202E0152A00F00F8102EB4201A6
:109240004FEA420918F80100A04202F10102F2D1EE
:10925000294491F8A518002900F066812046029360
:1092600036F018FD029B82465046029336F058FDB8
:109270000178002940F0F180029BA9440133DBB260
:10928000032289F8E53889F8E428BAF1000F00F0E4
:10929000E4804FEA141909F1FF39B9F1030F04F022
:1092A0000F0000F20881944C04EB4901B1F840C072
:1092B0004CFA00F111F0010100F0FD80012101FAEA
:1092C00000F0013800EA0C00A14402934FF00EFDBB
:1092D00099F848C0DFF838E2029B60440EEBC00CFE
:1092E00003228CF807308CF806205EF83000C6F8B0
:1092F00014C000F13F4303F57E0304EB93240121E6
:1093000094F84C309AF8082003F01F045B09032BF3
:1093100001FA04F100F00381042B00F0FB80022B22
:1093200000F0CF80BCF804300693B3FA83F3C3F1A6
:109330001F03C3F3CC0100EB810103F007030C6AA8
:109340009B004FF00F0C0CFA03FC24EA0C040C6297
:109350000C6A02FA03F323430B62022306A9079364
:10936000FEF74EFE039B002B00F08380B5F85437C8
:10937000D5F8981A07EE903AF8EEE77AFCEEE77A1D
:1093800017EE900AB1FBF0F202F57F42FF32120CA9
:10939000B1FBF2F295F85617B2FBF0F0042983B254
:1093A0007ED007EE902AF8EE676A66EE887A29EE9C
:1093B000677A95F8570704990091A6EEA87A01906C
:1093C00051463046C6ED027A86ED037A2BF0FEFA5E
:1093D000002F72DD7368D5F8E82793426FD0012F14
:1093E0006BD0D5F80028934269D0022F65D0D5F80C
:1093F0001828934263D0032F5FD0D5F830289342CA
:109400005DD0042F59D0D5F84828934257D0052F66
:1094100053D0D5F86028934251D0062F4DD0D5F8BF
:109420007828D31A18BF012301370122082F33747B
:10943000727406F118067FF4F0AE304809B0BDEC46
:10944000068BBDE8F08F9FED2E8AF0EE488AC2E6CB
:109450009FED2C8AF0EE488ABDE62B4A224BC5F8D8
:10946000CC270020C5F8D43709B0BDEC068BBDE889
:10947000F08FB0EE690A50F0DDFBFCEEC07A4FF6DB
:10948000FF7317EE902AD5F8981AB1FBF2F21A443E
:10949000120CB1FBF2F295F856170429184680D148
:1094A00007EE900A07EE102AF8EE677AF8EE476AA0
:1094B00067EE8A7A7BE7716154E70123B4E7002302
:1094C000B2E7124B5C6C214359642BE784B7050863
:1094D000F82B0020ACC5A737ACC5A7366100030840
:1094E00089E70308BDFC02087DE70308DC330020A0
:1094F0006F12833A00007A4470B70508A833002041
:10950000282930386F1203390DFE02080038024056
:10951000083500200F4B1C6B2143196302E70D4BEC
:109520001C6C21431964FDE68A469DE69FED0A8A7C
:109530000A4A0B4BC5F8CC27C5F8C83700220123CF
:10954000CDE90332F0EE488A064B50E69FED068ADD
:10955000EEE700BF003802406F12833A6100030853
:1095600089E703087DE7030800000000F8B5054619
:10957000262025F085FA124C0146E8B9D4F89C0A59
:1095800090F838301E3B012B01D937F0DDFE0D4F2E
:109590000026AE4208DBB4F8C03A0133A4F8C03A62
:1095A000236BC4F8D03AF8BD17F8011BD4F89C0A15
:1095B00037F0CAFE0136ECE7002384F8CE3AEFE735
:1095C000F82B00209836002038B5144C94F8C130A0
:1095D00094F8C0209A421AD004EBC303D3E9312097
:1095E00004F52A610023984212DC9378C4F8D40A67
:1095F0005B0884F8CE3AFFF7B9FF94F8C130062132
:109600000133B3FBF1F201FB123384F8C13038BDF2
:10961000D55C01F8015B0133E5E700BFF82B0020C2
:1096200013B504462620019125F02AFA019920B9A4
:10963000204602B0BDE810406EE502B010BD2DE935
:10964000F84F1B4C05461E2094F8D8AA94F8D9BAB6
:1096500094F8DA6AB4F8DC9AB4F8DE8A94F8E07A1E
:1096600025F00EFA30B1B8F1000F03D0C146012643
:109670004FF0000A94F8E23ADA070AD494F8E72A9D
:109680003AB9012F12D0022F03D113F0020F08BFF5
:10969000012685F800A085F801B0AE70A5F8049009
:1096A000A5F806802F722846BDE8F88F3E46F0E701
:1096B000F82B002007B50DF1060215F02BFC70B158
:1096C000084BBDF80620B3F80C1BA3F8A420914268
:1096D00005D00549A3F80C2B142081F8D80003B05D
:1096E0005DF804FBF82B00209801002013B5044618
:1096F000FFF7ECFA08B300230DF106022046ADF89F
:10970000063015F007FCC0B10D4C9DF8062094F909
:10971000DA1084F8EF20032908BF62F07F024FF0CF
:109720000501084808BF84F8EF20FFF737FB062142
:1097300084F8F0000348FFF719FB02B010BD00BF2A
:1097400098010020830200202DE9F743C54CD4F88E
:1097500094370D464BB14FF0020800274FF0010936
:10976000D4F8940737F0ECFD60B9002694F89E30E9
:10977000042B00F27281DFE813F09700F6000A0173
:1097800057016001D4F8940737F0D2FDD4F8AC3714
:109790005A1C2344C4F8AC2783F80E0B94F8A8375E
:1097A000012B0AD0022B11D0002B78D10F280CBF2F
:1097B00084F8A897C4F8AC37D2E7A0F17203012B64
:1097C00001D976286BD184F8A887C9E7102AC7D1B8
:1097D000A5490023012211F8010F013203440E2A8A
:1097E000DBB2F8D194F81C2B84F8A8779A42C4F81D
:1097F000AC77B5D194F81D3B002BB1D194F80F6B29
:10980000732E3FD0762E0FD0722EA9D194F8112B43
:1098100094F8103B53EA0223A2D0C4F88C30B4F879
:10982000123BC4F89030A1E794F8112B94F8103B48
:1098300053EA022394D094F8131B94F8122B94F853
:10984000170BC4F8A03042EA012294F8141B84F8E4
:109850009F1094F8151B84F8201B94F8161BA4F88D
:109860001E2B41EA0021A4F8221BD4F8941009B958
:10987000C4F89430B4F8A430002B7FF477AFA4F888
:10988000A42073E794F8152B94F8143B43EA0223C1
:109890001AB2002B3FF464AFA4F8242B66E784F8D7
:1098A000A877C4F8AC775BE7722E4ED1012384F819
:1098B0009E30002294F8C836402B36D1B4F8A4006C
:1098C000A4F8CE6694F8206B94F89E30B4F81ECBC2
:1098D000A4F8CC360502330394F89C10D4F8A07099
:1098E00005F4706503F440532B434FEA0C1543EA2B
:1098F0008133EDB22B43D4F894501BB2BD4214BF58
:10990000082500251343604514BF042000202B4385
:109910000343B14214BF022100211943534BA4F861
:10992000D01693F8D830A4F8D236D4F8F43023B156
:10993000D4F8A830002B40F0A3804D494D481F2299
:1099400003B0BDE8F04351F000BFD4F8283B4A4AC9
:10995000EB1A934201DC0022ACE77220FFF70AFC0D
:10996000C4F8285BF7E7762E04D1022384F89E30F2
:1099700000229FE7D4F8283B3F4AEB1A9342EADDE6
:109980007620FFF7F7FBC4F8285B002292E7374FF9
:10999000D4F8283B97F8D820EB1AB2B3364A934252
:1099A00036DD94F89F20D2071FD4D4F89410D4F851
:1099B000A02091420FD089B24620FFF731FE97F8E0
:1099C000D830C4F8285B013B87F8D830042384F8EA
:1099D0009E3001226EE7B4F8A410B4F81E2B8A4220
:1099E00003D05020FFF71CFEE9E794F89C1094F890
:1099F000202B8A4206D0B1FA81F149094920FFF7AC
:109A00000FFEDCE7142287F8D8201C4A9342B7DC0B
:109A1000762EA0D17320FFF7ADFB032384F89E3090
:109A2000C4F8285B002245E7732E94D0D4F8281B95
:109A3000114B691A994298DC8DE7D4F8283B0E4AFD
:109A4000EB1A934287DD7620FFF794FB022384F81C
:109A50009E30C4F8285B00222CE7002384F89E3057
:109A60001A4627E7F82B002006370020980100202F
:109A70004F2F0608890200203F0D03003F420F00D0
:109A8000334DD4F82C6B2A2385F8F1300DF1020206
:109A900020230DF10101304685F8F23015F0D1FA9E
:109AA00030B19DF801109DF8027051EA070339D1D9
:109AB000552385F8F330462385F8F430202301A997
:109AC000304685F8F53015F0B6FA0346214813B153
:109AD000BDF804209ABB20494BF0C6FAB4F8227BAB
:109AE0001E4D87B30DF10301304615F0A7FA50B3B0
:109AF0009DF803100DF10602304615F00BFA10B375
:109B0000BDF8062016493B46BA420CBF20222A2245
:109B100028464BF0A9FAB4F8243BA4F8303B03B034
:109B2000BDE8F083304615F071FA394685F8F30048
:109B3000304615F057FA037885F8F430BEE7094946
:109B40004BF092FACAE7084928464BF08DFAE2E753
:109B5000980100208E020020712F0608920200203A
:109B6000692F0608CF680608702F060838B50B68FD
:109B70000E4D5A1C0A6005221A700B6895F8DA20FF
:109B80000C46591C21601A70236895F8DD20591C79
:109B900021601A70B5F8E010204649F023FE2368D2
:109BA00095F8E220591C21601A7038BD98010020F8
:109BB0002DE9F84F2DED028BFFF788F8002844D0EF
:109BC000254B93F9DA0001283FDD93F81041DFF8C7
:109BD00090809FED228A0FF2780BDBE900AB1546EF
:109BE0008E1E02EB44094D4504D1BDEC028B20468C
:109BF000BDE8F88F38F8027B26F8027F07EE907AEE
:109C0000F8EEE77A67EE887A17EE900A4EF094FC49
:109C100052465B464EF0E8FC41EC100B51F0B8FAAE
:109C200051EC100B4EF0A2FF0E2F80B20AD9193062
:109C30003223B0FBF3F080B200EB800000EB800039
:109C4000400080B225F8020BCDE70024CDE700BF2D
:109C50001655B5BBB16B024098010020CDCCCC3D70
:109C60002A37002038B50D46FFF730F8044638B1E2
:109C70000C4890F8DD30DB0704D5B0F8DE00288012
:109C8000204638BD084A90F9DB3092F8BC2093FB9F
:109C9000F2F102FB11320132013100F58A7015F048
:109CA0004DF9ECE798010020F82B00202DE9F04F4A
:109CB000A94D95F8423B8BB08146002B40F0B58012
:109CC000D5F82C6B002E00F0B080A44AD2F81841D1
:109CD00004F0F021B1F1E02F6ED1C2F81831D5F8BF
:109CE000442B944268D004930593ADF81830B5F82E
:109CF000DC3A95F8D8EAADF8143095F8D9CA95F859
:109D0000E03A95F8DAAA8DF818300DF110088DF8C0
:109D100010E08DF811C08DF812A098E8070007AB8D
:109D200003C38F4F1A80C4F342533B44C4F303422E
:109D300093F85210C5F8444B8E4502F1010201D14F
:109D4000944508D030468DF81C108DF81D2015F074
:109D5000F5F8ADF82000304615F041FB032804F07B
:109D6000070B34D0042836D000239A4501A9304689
:109D700018BF8DF81E3015F05BF948B1019BC4F394
:109D8000001103F001038B4202D0304615F0FEF9BA
:109D90000A2207A9404651F072FC68B19DF81E30B6
:109DA000BDF81C2085F8DA3ABDF82030A5F8D82A8D
:109DB000A5F8DC3A4AF028FB95F848AB04AF95F8D3
:109DC000483B032B7BD8DFE803F00A3376A35F44DC
:109DD00097F85730C9E75F4497F85F30C5E73946D1
:109DE000304615F02BF9044658B107A8FFF727FCB9
:109DF0009DF81E109DF810308B4260D0304615F053
:109E000051FA95F8483B013303F0030385F8483BCA
:109E10000CB99A45D3D195F8E23ADB0700D524B1C5
:109E2000336849461B68304698470BB0BDE8F08F51
:109E300001A8FFF704FC95F8E28A9DF8044008F0B9
:109E40000108ECB1B8F1000F39D13A460DF1030128
:109E5000304615F0F6F8044688B307A8FFF7EFFB85
:109E60009DF81C109DF803309DF81D208B4203D1F6
:109E70009DF81030934222D0304615F01DFAC0E70D
:109E8000B8F1000FBDD13946304615F0D4F804467C
:109E9000A8B107A8FFF7D3FBBDF82010BDF810301C
:109EA0008B420CD085F8498B85F84A8B3368304655
:109EB0009B699847A5E795F8E23AD80701D50024B1
:109EC0009FE707A9304615F0B3F804460028F6D0FE
:109ED0001E2024F0D5FD95F84B3B83428046EED002
:109EE00085F84B0B60B1B5F8DE3A002BE7D1079B44
:109EF000D907E4D40121304615F048F9444680E7FB
:109F0000079BDA07DBD50146304615F03FF978E7C5
:109F10003846FFF794FB97E8070007AB03C31A80A6
:109F20009DF810309BB10DF11D0207A9304615F0C8
:109F300088F80DF11E01304615F080F80A2207A9B5
:109F4000384651F09CFB041E18BF012459E708A9AC
:109F5000304615F070F8ECE7F82B0020980100204F
:109F600070B705082DE9F041FD2984B0044669D099
:109F7000F02949D0EF2900F0BF804AB10346861886
:109F800003AD002003F8010B9E4205F8010BF9D147
:109F9000BA4B0B2003F1090501E013F8010F8142D0
:109FA00055D0AB42F9D14B1E152B21D8DFE813F069
:109FB000C500D000DA00E700EE00F400160004014E
:109FC00000012000200023012301230110011001C2
:109FD00010010001200020001B01AD00A84D95F8E4
:109FE000E23ADE0700F16D81B5F8B83BADF80C3010
:109FF0003AB1224403AB13F8011B04F8011BA2423F
:10A00000F9D104B0BDE8F0819E4F03214FF005085F
:10A01000B844002501370CE0FFF72EF8064660191A
:10A020003246FFF79FFF70194745C5B2E9D017F8D0
:10A03000011B412981F08003084601D0042BEBD895
:10A040000426ECE7904F0B214FF00408E0E78C4B1F
:10A05000D3F83C0C80060CD4002AD2D0224403ABA7
:10A0600013F8011B04F8011B9442F9D104B0BDE8B8
:10A07000F08193F84C0B10F0020F93F8640B40D072
:10A08000052834BF02250325142917D97C39C8B205
:10A090000628E1D80629DFD801A050F821F000BF3A
:10A0A00071A2000871A2000859A2000859A0000876
:10A0B00051A2000849A2000841A200080929CBD9F1
:10A0C0000A390A29C8D801A656F821F02DA200089D
:10A0D000A5A2000859A0000859A0000859A000082E
:10A0E00059A0000859A0000859A0000859A000086C
:10A0F00023A2000871A20008644F0C214FF006084B
:10A1000086E70B29A8D10125CDE05D4BB3F8D81B1C
:10A11000CD055ABFCB4303F00103032311F0440FD5
:10A1200018BF042311F0020F18BF072311F4806F2A
:10A1300018BF0923ADF80C305AE7514BB3F8983BE0
:10A1400003EB83035B0003F5C873ADF80C304FE7F6
:10A150004F4BD3ED037AFDEEE77A17EE903AADF868
:10A160000C3045E7464B93F8771B002900F0A080A0
:10A1700001922AF08DFE019AADF80C0038E70192A9
:10A180002AF086FE019AADF80C0031E73C4BD3F87B
:10A19000C83BADF80C302BE7394BB3F8B81B00299E
:10A1A00000F0898001922AF081FE019A80B2E3E7F3
:10A1B000334BB3F83A3C19E7314B3649B3F9383CE5
:10A1C00081FB0301DB17C3EBA103ADF80C300FE7F4
:10A1D0002B4B03EB4101B1F8163C03EB83035B000F
:10A1E000ADF80C3004E7264B93F8E23A03F0010394
:10A1F000ADF80C30FCE6284BDFED286AD3ED007A91
:10A200000C39C9B203EB810393ED127A67EEA67A9B
:10A2100067EE877AFDEEE77A17EE903AADF80C30EC
:10A22000E6E6B3F85E3BADF80C3015E7B3F8603BFB
:10A2300003EB830303EB83039B00ADF80C300BE7C8
:10A24000D3F8583B039307E7D3F8543B039303E752
:10A25000D3F8503B0393FFE6B3F85E3B104903EBA2
:10A26000C3039B00A1FB03135B09ADF80C30F3E6BD
:10A27000B3F8683BADF80C30EEE600BFD8B7050880
:10A28000F82B002074B7050870B705087CB70508DF
:10A290009437002067666666D437002000007A4451
:10A2A0001F85EB51EDB28DF80C508DF80D00D3E603
:10A2B000B3F8900B60E7D3F8D00B80F3100080B2B6
:10A2C0005AE7019224F036FE05F69C33D3ED037A6B
:10A2D000019AFCEEE77A17EE903A9BB200287FF4E1
:10A2E00085AED5F8D41B11F0100F18BF00237DE602
:10A2F00000F01F0240090123032803FA02F304D0EF
:10A3000004280CD0022805D07047074A116C0B4373
:10A3100013647047044A516C0B4353647047024AFC
:10A32000116B0B43136370470038024000487047BD
:10A33000683500200E4B30B4DB68427801780D4C54
:10A34000DB43C3F30223C3F10403DBB202FA03F3DA
:10A3500060181B0101F01F050122490903F0F003F9
:10A36000AA4080F8003344F8212030BC704700BF79
:10A3700000ED00E000E100E0002800F087802DE91A
:10A38000F0411C468388B3FA83F3202B8C4682B0BD
:10A3900011468046C3F11F026ED03D4E3D4DB318AD
:10A3A00005EB820293F87470C2F840CC35F0EAFEF7
:10A3B000B8F804E0D8F80000374ABEFA8EFECEF1B5
:10A3C0001F0101F0FC0303F1804303F59C3301F00E
:10A3D00003014FEA810C4FF00F0800F13F419868EC
:10A3E00008FA0CF820EA080001F57E019860C1F334
:10A3F000872101FA0CF1D3F808C04FF0004020FA91
:10A400000EF041EA0C0199605061136823EA0003E1
:10A410001360536823EA0003536013680343136017
:10A42000936806EB840423EA00039360D36894F8EE
:10A43000841023EA00031029D36020D001F1804169
:10A4400001F59E310B68184308603D4495F8803C47
:10A45000F02B11D93E44F02196F890308DF804305D
:10A4600003224FF4807301A885F8801C8DF8052025
:10A47000ADF80630FFF75EFF02B0BDE8F0819368EB
:10A4800003439360D3681843D060DEE7704700BF92
:10A4900070B70508F82B0020003C0140464B5B6874
:10A4A000C3F308032DE9F041002B62D1EFF31183D0
:10A4B000002B5ED1414A424C116BA068136B99424C
:10A4C000FAD1D2F8903C9842F6D8D2F88C5C4FF48E
:10A4D0007A7404FB05F3181AB0FBF5F004FB0101D4
:10A4E000354D374810264FF47A7401276B68C3F353
:10A4F0000803EBB9EFF31183D3B9136BD0F808E07D
:10A50000D2F830C06345F8D1D2F890CCE645F4D803
:10A51000D2F88C8C04FB08FCACEB0E0CBCFBF8FCFA
:10A5200004FB03C35B1AB3F57A7FDFD3BDE8F08188
:10A53000EFF3118E86F31288D0F808800368DB03EE
:10A5400044BFC2F8887CD0F80880D2F830C0D2F876
:10A55000883C5FFA8EFE8EF31188D2F88CEC63444F
:10A5600004FB0EFCACEB080CBCFBFEFC04FB03C3C1
:10A57000D8E7EFF31180102383F3128810490F4AB4
:10A580008D680B68DC0342BF0123C2F8883C8D68EC
:10A59000136BD2F8881CC0B280F31188D2F88C4CAF
:10A5A0004FF47A70194400FB04F35B1BB3FBF4F324
:10A5B00000FB013194E700BF00ED00E0F82B002024
:10A5C00010E000E02DE9F84FB34C94F8941C0546D8
:10A5D000C1F34001D4F89C0C3AF09CF994F8941C17
:10A5E000D4F8980CC94301F001013AF093F9002D19
:10A5F00000F0C3806E1EA94FA94D5FFA86FB4FF095
:10A600001008D4F89C0C3AF069F9D4F8980C3AF098
:10A6100065F9B4F8A43C002B40F0358194F8A61CF1
:10A62000D4F8A80C3AF076F94FF0FA094FF47A70A2
:10A630004FF0010C7B68C3F30803002B40F0FB8054
:10A64000EFF31183002B40F0F680226BA968236B97
:10A650009A42FAD1D4F8903C9942F6D8D4F88C6C4E
:10A6600000FB06F35B1AB3FBF6F300FB02327B68D8
:10A67000C3F30803002B40F09F80EFF31183002BFE
:10A6800040F09A80236BD5F808A0216B8B42F9D15A
:10A69000D4F8901C8A45F5D8D4F88C6C00FB06F1F0
:10A6A000A1EB0A01B1FBF6F100FB03139B1AB3F512
:10A6B0007A7FDCD3B9F10109BCD1D4F89C0C3AF013
:10A6C0000DF9D4F8980C3AF009F9B4F8A43C002B31
:10A6D00040F0CD8094F8A61CD4F8A80C81F00101BC
:10A6E0003AF018F94FF0FA0C4FF47A704FF0010E6F
:10A6F0007B68C3F30803002B7ED1EFF31183002B9B
:10A700007AD1226BA968236B9A42FAD1D4F8903C93
:10A710009942F6D8D4F88C9C00FB09F35B1AB3FB82
:10A72000F9F300FB02327B68C3F308033BBBEFF392
:10A73000118323BB236BD5F808A0216B8B42F9D181
:10A74000D4F8901C8A45F5D8D4F88C9C00FB09F10C
:10A75000A1EB0A01B1FBF9F100FB03139B1AB3F55E
:10A760007A7FE0D3BCF1010CC2D10BF1FF365FFA66
:10A7700086FBBBF1FF0F7FF444AFBDE8F88FEFF32A
:10A78000118988F31288AE682B68DB0344BFC4F8D4
:10A7900088ECAE68236BD4F8881C5FFA89F989F3DA
:10A7A0001188D4F88C9C0B4400FB09F1891BB1FB88
:10A7B000F9F100FB0313D1E7EFF3118E88F3128850
:10A7C000D5F808A02B68D90344BFC4F888CCD5F8C5
:10A7D00008A0236BD4F8881C5FFA8EFE8EF31188D4
:10A7E000D4F88C6C0B4400FB06F1A1EB0A01B1FB21
:10A7F000F6F100FB031359E7EFF3118188F3128898
:10A80000D5F808902B68DA0344BFC4F888ECD5F873
:10A810000890236BD4F8882CC9B281F31188D4F83E
:10A820008C1C1A4400FB01F3A3EB0903B3FBF1F307
:10A8300000FB023277E7EFF3118188F31288AE68EC
:10A840002B68DB0344BFC4F888CCAE68236BD4F814
:10A85000882CC9B281F31188D4F88C1C1A4400FBEF
:10A8600001F39B1BB3FBF1F300FB0232FFE6D4F8CC
:10A87000C03C002B3FF436AFD4F8AC3CC3F800909A
:10A8800084F8BD9C2EE7D4F8C03C002B3FF4CCAE3E
:10A8900036F08AFAC8E600BFF82B002000ED00E091
:10A8A00010E000E02DE9F84FB04CB14F94F8941C43
:10A8B000D4F89C0CAF4DC1F340013AF02BF894F85A
:10A8C000941CD4F8980CC94301F001013AF022F825
:10A8D0004FF0050B4FF01008D4F89C0C39F0FEFF38
:10A8E000D4F8980C39F0FAFFB4F8A43C002B40F0EF
:10A8F000358194F8A61CD4F8A80C3AF00BF832264F
:10A900004FF47A704FF0010C7B68C3F30803002BFF
:10A9100040F0FA80EFF31183002B40F0F580226BBA
:10A92000A968236B9A42FAD1D4F8903C9942F6D8A0
:10A93000D4F88CEC00FB0EF35B1AB3FBFEF300FBC8
:10A9400002327B68C3F30803002B40F09E80EFF3D4
:10A950001183002B40F09980236BD5F808A0216B60
:10A960008B42F9D1D4F8901C8A45F5D8D4F88CECF8
:10A9700000FB0EF1A1EB0A01B1FBFEF100FB03139A
:10A980009B1AB3F57A7FDCD3013EBDD1D4F89C0C81
:10A9900039F0A4FFD4F8980C39F0A0FFB4F8A43C27
:10A9A000002B40F0D08094F8A61CD4F8A80C81F0BD
:10A9B000010139F0AFFF4FF0320C4FF47A700126ED
:10A9C0007B68C3F30803002B7FD1EFF31183002BC7
:10A9D0007BD1226BA968236B9A42FAD1D4F8903CC0
:10A9E0009942F6D8D4F88C9C00FB09F35B1AB3FBB0
:10A9F000F9F300FB02327B68C3F308032BBBEFF3D0
:10AA0000118313BB236BD5F808A0216B8B42F9D1BE
:10AA1000D4F8901C8A45F5D8D4F88C9C00FB09F139
:10AA2000A1EB0A01B1FBF9F100FB03139B1AB3F58B
:10AA30007A7FE0D3BCF1010CC2D10BF1FF3616F0E6
:10AA4000FF0B7FF449AFBDE8F88FEFF3118988F36E
:10AA50001288D5F808A02B68DB0344BFC4F8886CC3
:10AA6000D5F808A0236BD4F8881C5FFA89F989F31C
:10AA70001188D4F88C9C0B4400FB09F1A1EB0A016E
:10AA8000B1FBF9F100FB0313D0E7EFF3118E88F36C
:10AA90001288D5F808A02B68D90344BFC4F888CC25
:10AAA000D5F808A0236BD4F8881C5FFA8EFE8EF3CD
:10AAB0001188D4F88CEC0B4400FB0EF1A1EB0A01D9
:10AAC000B1FBFEF100FB03135AE7EFF3118188F3AA
:10AAD0001288D5F808902B68DA0344BFC4F8886C54
:10AAE000D5F80890236BD4F8882CC9B281F311886B
:10AAF000D4F88C1C1A4400FB01F3A3EB0903B3FB4D
:10AB0000F1F300FB023276E7EFF3118188F312884C
:10AB1000D5F808E02B68DB0344BFC4F888CCD5F82F
:10AB200008E0236BD4F8882CC9B281F31188D4F8DB
:10AB30008C1C1A4400FB01F3A3EB0E03B3FBF1F3EF
:10AB400000FB0232FDE6D4F8C03C002B3FF433AFEB
:10AB5000D4F8AC3C1E6084F8BD6C2CE7D4F8C03C43
:10AB6000002B3FF4CCAE36F01FF9C8E6F82B0020DE
:10AB700000ED00E010E000E010B4B8B10D4CD4F8E6
:10AB8000C43C102B05D15DF8044B0521002035F0A5
:10AB9000E1BD03EB4302224482F8C91C01210B44AE
:10ABA00082F8C80C82F8CA1CC4F8C43C5DF8044B97
:10ABB000704700BFF82B002000285FD00368374A99
:10ABC0002DE9F04103F13F4404F57E0402EB9422A9
:10ABD000012492F84C2002F01F055209032A04FABE
:10ABE00005F456D0042A4FD0022A48D08588B5FAF9
:10ABF00085F0C0F11F00C0F3CC0603EB860600F021
:10AC0000070082000F24306A944020EA040030627A
:10AC1000306A01FA02F20243002132624FF0010E63
:10AC20000A464FF0030C02270EFA02F838EA050034
:10AC300002F101021CD118680CFA01F420EA0400A8
:10AC40001860186807FA01F606431E609E6826EA37
:10AC500004069E6098689860586820EA080058606A
:10AC600058685860D86820EA0400D860D868D8606E
:10AC7000102A01F10201D7D1BDE8F0817047084ADE
:10AC8000556C2C435464B1E7054A156B2C4314638F
:10AC9000ACE7034A156C2C431464A7E770B70508AA
:10ACA0000038024070B5464E96F8F84C04EB440369
:10ACB00006EBC303650093F8FC3C032B6ED8DFE87A
:10ACC00003F059291E02254406EBC505D5F8000DF1
:10ACD000002870D196F85C3D9C425FD0013404F0AE
:10ACE0000302934286F8F82C58D002EB420406EB9C
:10ACF000C4040223C4F8000D84F8FC3C70BD2B1979
:10AD000006EBC303D3F8002D72B1013AC3F8002D4E
:10AD1000002070BD2B1906EBC303D3F8002D002AC9
:10AD2000F3D1022283F8FC2C254406EBC50595F8E7
:10AD3000083D013BDBB285F8083D8BBB214B96F803
:10AD40005C6DD3F81C11D5F8040D621C02F00302EF
:10AD50004B1E0324B242034485F8FC4CB3FBF1F0D4
:10AD6000C5F8000D1AD0994218D80138C5F8000D61
:10AD7000012070BD3EF0ECF880B1124B2C44D3F8AA
:10AD80001C2106EBC404012102F51C5384F8FC1CB1
:10AD90000F33B3FBF2F3C4F8003D70BD012070BD6A
:10ADA000084BD3F81C21012002F2E733B3FBF2F386
:10ADB000C5F8003D70BD0138C5F8000D002070BD1C
:10ADC000F82B00209801002070B503688CB0FF229A
:10ADD0000446587B8DF80720012100220DF107055C
:10ADE000CDE90252CDE90622CDE908220B92049169
:10ADF0008DF814108DF8281050B310250426EFF3A9
:10AE0000118385F312882268116AD8B2002931D0E3
:10AE100080F3118823681A6A042AF0D1EFF31181B4
:10AE2000102282F312881A6A042A04D02268126A55
:10AE30000AB11B6AA3B9C9B281F3118802A92046DD
:10AE40004CF080FA2268136A002BFCD10CB070BD64
:10AE50001A6A002AE2D01A6A002AF9D1DEE714330E
:10AE60009A68002AFBD102AA1C60C9B25A6081F319
:10AE70001188E7E7166280F3118823681A6A042AAA
:10AE8000BDD1CBE72DE9F04F854C95B000230E46A0
:10AE90004FF4F0722021054604F55660019684F8BF
:10AEA0005D3D84F85E3D50F012FC202104F5746095
:10AEB0004FF4F07250F00BFCDFF8F0C17949322703
:10AEC0004FF0100E4FF47A700126DCF80430C3F313
:10AED0000803002B40F0C380EFF31183002B40F0F8
:10AEE000BE80226BD1F80890236B9A42F9D1D4F836
:10AEF000903C9945F5D8D4F88CAC00FB0AF3A3EB51
:10AF00000903B3FBFAF300FB0232DCF80430C3F3AD
:10AF10000803002B40F08380EFF31183002B7ED1D8
:10AF2000236BD1F808B0D4F830904B45F8D1D4F861
:10AF3000909CCB45F4D8D4F88CAC00FB0AF9A9EB73
:10AF40000B09B9FBFAF900FB03939B1AB3F57A7F5F
:10AF5000DBD3013FB9D1DFF8588198F82920002AC6
:10AF600058D098F82A30032B54D8013B03EB830CBC
:10AF700008EBCC0108F1C40091F8C4E000EBCC0070
:10AF8000BEF1020F4FF0010CC8F82C0088F8B4C0D5
:10AF900000F0F3815BB2581C00F0FD8108EB031355
:10AFA000D3F83C31C1F8C830A3B308F13C0008F134
:10AFB0007803C1E937034FF0020EA1F8D07081F891
:10AFC000D2C081F8C4E01709013F032F02F00F023D
:10AFD00000F27181DFF8DC9009EB4703B3F8400021
:10AFE00040FA02F3DB0740F16681012303FA02F223
:10AFF000013A10404F444DF079FE97F848202A4B13
:10B00000104403EBC000C8F834008379002B53D000
:10B01000412B51D06FF0010015B0BDE8F08FEFF378
:10B02000118A8EF31288D1F808B00B68DB0344BF95
:10B03000C4F8886CD1F808B0236BD4F8889C5FFA08
:10B040008AFA8AF31188D4F88CAC4B4400FB0AF9D5
:10B05000A9EB0B09B9FBFAF900FB039375E7EFF3D2
:10B0600011898EF31288D1F808A00B68DA0344BF67
:10B07000C4F8886CD1F808A0236BD4F8882C5FFA48
:10B0800089F989F31188D4F88C9C1A4400FB09F3E0
:10B09000A3EB0A03B3FBF9F300FB023235E700BF71
:10B0A000F82B002010E000E00835002000ED00E063
:10B0B000F03C002070B705082323C380092135F038
:10B0C00061F8D8F8343013B11A689B881383D4F828
:10B0D000982AC14BB3EB920F80F05581B3EBD20F9E
:10B0E00080F06081B3EB121F80F05E81B3EB521FE2
:10B0F00080F05C81B3EB921F80F05A81B3EBD21FDA
:10B1000080F05881B3EB122F80F056814FF480739A
:10B11000B248A8F83030FFF757FEB0488C213DF018
:10B12000E7FC1B2840F05081D8F83430012284F825
:10B130005D2D0BB12322DA804022A8480A213DF080
:10B14000A7FDA6488A213DF0D3FC98F82830C0F32B
:10B150008012012B88F86C2100F0400000F0AF80D5
:10B16000022B00F0EC80002B00F0CB80B8F86E31A1
:10B1700094F8C816182906D10199A4F8CC16A4F899
:10B18000CE26A4F8D0369548A8F830300222002107
:10B190003DF07EFD642035F025FCDFF840B2D8F8A4
:10B1A0002C300DF10E090DF10F04002600274FF091
:10B1B000100A587BCDF81090002201214FF0800C2E
:10B1C000CDE90E67CDE908220A948DF80EC00592EC
:10B1D0008DF81C200D921092129206910B918DF811
:10B1E00030108DF84410002847D00421EFF311836C
:10B1F0008AF31288D8F82C20D2F820C0D8B2BCF13B
:10B20000000F41D080F31188D8F82C301A6A042A34
:10B21000ECD1EFF311818AF312881A6A042A42D022
:10B22000D8F82C20126A002A3DD01A6A0AB93AE0EE
:10B2300014329368002BFBD104AB5360C2F800B00A
:10B24000CBB283F31188D8F82C301A6A002AFCD1CB
:10B250009DF80F0010F00200ABD16A78AB78297826
:10B2600088F87011C2F12002C3F1100388F871212F
:10B2700088F8723115B0BDE8F08F1A6A002AC8D07C
:10B280001A6A002AF9D1C4E7116280F31188D8F84C
:10B290002C301A6A042AA9D1EFF311818AF312889B
:10B2A0001A6A042ABCD1CBB283F3118804A9584688
:10B2B0004CF048F8C7E70020C8F83400FEE6019BD0
:10B2C000D4F8981A0BB100285FD0454BB3EB910F1F
:10B2D0005FD2B3EBD10F71D2B3EB111F5ED2B3EBE0
:10B2E000511F6DD2B3EB911F6CD2B3EBD11F57D26C
:10B2F000B3EB112F34BF4FF480738023A8F86E3165
:10B3000036E7D4F8981A344BB3EB910F41D2B3EB34
:10B31000D10F53D2B3EB111F40D2B3EB511F4FD219
:10B32000B3EB911F4ED2B3EBD11F39D2B3EB112F38
:10B3300034BF4FF480738023A8F86E3118E7D4F837
:10B34000980A2749B1EB900FD8D2B1EBD00F35D284
:10B35000B1EB101F22D2B1EB501F31D2B1EB901FD5
:10B3600030D2B1EBD01F1BD2B1EB102F34BF4FF452
:10B3700080738023A8F86E31FAE691F8D2306344E6
:10B3800081F8D2301FE60223C2E6134BB3EB910FD4
:10B39000BDD30223B2E7C1F8C8703BE60823ADE78E
:10B3A0004023ABE70423B3E60823B1E61023AFE65E
:10B3B0002023ADE64023ABE68023A9E604239DE7E6
:10B3C00010239BE7202399E7D8F83400202134F09C
:10B3D000D9FE4FF0FF301FE6404B4C001C3D0020D3
:10B3E0008096980010B582B00A88ADF80620002338
:10B3F0000C468DF805308DF8040049F0B7FF0421A4
:10B400000DEB010029F0C6FABDF80630238002B02A
:10B4100010BD00BF10B582B00A788DF80720182340
:10B42000040A8DF804308DF806008DF8054049F0C7
:10B430009DFF04210DEB010029F0ACFA02B010BD14
:10B4400010B582B019220023040A8DF803308DF85C
:10B4500001408DF800200C468DF8020049F086FF6F
:10B460000521684629F096FA9DF80430237002B051
:10B4700010BD00BF38B50C4C0546A11CD52248F0C4
:10B4800047FE2B68A342C5E90043A3EB04000AD0A2
:10B4900004F14002611C2960237802F8013BD5E9E0
:10B4A0000041A142F6D138BD643E0020F0B40D68E1
:10B4B00000240CE0BCF1050F18D8A0F137030A2BCB
:10B4C00014D104EB840415F8010B03EB4404A0F140
:10B4D0003003DEB2092EA0F16107A0F1410CF0D9D2
:10B4E000052FE7D8A0F157030A2BEAD00D601460AE
:10B4F000F0BC7047094B93F85637042B08D9053B2D
:10B50000032B08D801231A4600B103701046704778
:10B5100000230122F8E700231A46F5E7F82B002064
:10B520009FED727A07EE901A20EE070AF8EE677A1E
:10B5300027EE800AFDEEC07A17EE903A2033402BBA
:10B5400000F2C480DFED6A7AB4EEE70AF1EE10FA99
:10B55000F0EE407A0CDD9FED676ADFED676AB0EED2
:10B56000677AB4EEE67AF1EE10FA77EEC67AF6DC98
:10B570009FED627AF4EEC77AF1EE10FA0CD59FEDEA
:10B580005D6ADFED5F6AB0EE677AB4EEE67AF1EEFF
:10B5900010FA77EE867AF6D49FED5A7AF4EEC77AEF
:10B5A000F1EE10FA00F38A809FED577AF4EEC77A35
:10B5B000F1EE10FA44BF9FED517A77EE677A27EEED
:10B5C000A76ADFED525A9FED527ADFED526AA6EE7E
:10B5D000257A67EE865AE6EE076AB6EE007AE5EE61
:10B5E000A67A27EE877ADFED476A70EE267ABDEEFF
:10B5F000E76A16EE103A2033402B64D8B4EEE60A20
:10B60000F1EE10FA0CDDDFED3B5A9FED3B6AF0EEF8
:10B61000676AF4EEC66AF1EE10FA77EEE57AF6DCC8
:10B62000DFED366AF4EEE67AF1EE10FA0CD5DFEDD6
:10B63000315A9FED336AF0EE676AF4EEC66AF1EEB6
:10B6400010FA77EEA57AF6D4DFED2E6AF4EEE67AFC
:10B65000F1EE10FA3DDDDFED266A76EEE77A67EE71
:10B66000A75A9FED2A5A9FED2A6ADFED2A6AA5EEB6
:10B67000856A27EEA55AE5EE866AB8EE006AE5EE21
:10B68000267A67EE867AC7EE206AB7EE006A76EE13
:10B69000865A76EE666A86EE257A80ED091A67EE9E
:10B6A000277A66EE876AC0ED017AC0ED037A80EDF5
:10B6B000007A80ED027AC0ED046A70479FED0C7A43
:10B6C00077EE677A7BE7DFED147ADCE79FED127A9D
:10B6D00089E7DFED0D6AF4EEE67AF1EE10FA44BF89
:10B6E000DFED066A76EEE77AB9E700BF27D4D236F7
:10B6F000DB0F4940DB0FC940E4CB1641DB0F49C0EB
:10B70000E4CB16C1DB0FC93FDB0FC9BF92E741B9DC
:10B710009730083C15A82ABE000000002DE9F84328
:10B72000E14FD7ED7E7A97F86847F8EE670A07F29F
:10B7300064732DED028BC3ED000A002C70D1DFF88D
:10B74000C4E3DFF8C4C39EF8FC60C7F874479CF8F4
:10B750000040002E39D0B7F86E379FEDD46A9FEDC8
:10B76000D47A07EE903AF8EE677A20EE877AC6EE42
:10B77000276AD04B0022012E1A6076EE876AC7EE48
:10B78000267AC3ED017A20D0022E9A60C3ED037AA7
:10B790001BD0032E1A61C3ED057A16D0042E9A61D0
:10B7A000C3ED077A11D0052E1A62C3ED097A0CD0C9
:10B7B000062E9A62C3ED0B7A07D0072E1A63C3EDEB
:10B7C0000D7A02D09A63C3ED0F7A9EF876379FED1B
:10B7D000BA6A9FEDBA7A9FEDBA0ABA4A07EE903A72
:10B7E000F8EEE77A9CF8583BC6EE276A1C4414FB37
:10B7F00006F6F6B207EE906A60EE870AF8EEE77A90
:10B80000C2ED006AA7EEA00A4EF0D8FABDEC028B9A
:10B81000FCEEC07A17EE903A87F87C37BDE8F883E3
:10B8200097F86937DFEDA84A9FEDA82ADFEDA86AEF
:10B83000DFF8D0E2DFF8D0C29EF8FC60C7F874C72A
:10B8400007EE903AB7F86C378CF8004007EE103AE4
:10B85000FCEEE05AB7F86A3706EE103A15EE903A69
:10B86000F8EE655AF8EE677A84EEA55ACCF81430F3
:10B87000012387F87037B8EEC77A27EE822AB8EE30
:10B88000466A67EE266A22EE252A8CED025ACCED36
:10B89000017A8CED036ACCED046A002E95D0DFEDC1
:10B8A0008D7A9FED8D4ADFED8D5AC7EE871AC6EB74
:10B8B0000615A6EB06190CEBC5054FEAC9094FF0B2
:10B8C0000008B1EE611A9FED866A09EB05009FED55
:10B8D000853ADFED853ADFED856A0346002207EE03
:10B8E000902AB8EEE77A27EE027AFDEEC77A17EED5
:10B8F000901A2031402900F2D080B4EEC47AF1EEE3
:10B9000010FAF0EE477A0CDDDFED794A9FED795AB7
:10B91000F0EE672AF4EEC52AF1EE10FA77EEE47A3B
:10B92000F6DCF4EEE57AF1EE10FA0CD5DFED704AB4
:10B930009FED715AF0EE672AF4EEC52AF1EE10FA87
:10B9400077EEA47AF6D4F4EEC67AF1EE10FA40F36C
:10B950009A8074EE677A27EEA75AB0EE630AA5EED6
:10B96000030ADFED664AE5EE004A65EE272AB7EEE8
:10B97000005AE2EEA47AB0EE458AF0EE454AA1EE16
:10B98000A78AE1EE274AC5EE088A84EE880A77EE98
:10B99000067ABDEEE75A15EE101A203140296FD80D
:10B9A000B4EEC67AF1EE10FA0CDD9FED515A9FED20
:10B9B000517AF0EE674AF4EEC74AF1EE10FA77EEEC
:10B9C000C57AF6DCF4EEE57AF1EE10FA0CD59FEDCF
:10B9D000485A9FED497AF0EE674AF4EEC74AF1EE15
:10B9E00010FA77EE857AF6D4F4EEC67AF1EE10FA14
:10B9F0003CDD74EE677A27EEA75AF0EE632AE5EE97
:10BA0000032A9FED3E7AA5EE227A65EE274AB8EE2C
:10BA1000005AE4EE877A67EE857A87EE887A0132FB
:10BA2000A24203F1280343ED048A03ED037A03EDF8
:10BA3000017A43ED028A83ED000AC3ED056AC3ED86
:10BA4000026AC3ED016AC3ED046AC3ED036AFFF63F
:10BA500046AF783085427FF43AAF08F57078B8F594
:10BA6000346F05F570757FF42EAF74E69FED247A80
:10BA7000F4EEC77AF1EE10FA48BF75EEE77ABAE74E
:10BA8000F0EE667AC9E79FED1E5AF4EEC57AF1EE44
:10BA900010FA48BF75EEE77A5DE7B7EE000AF0EE00
:10BAA000408AB0EE408A72E7F03C002083F9223EE3
:10BAB000BD37863570440020555555406E12833A87
:10BAC00048E1FA3E684400200060EA4827D4D236B4
:10BAD0000AD7233C00004842DB0F4940DB0F49C036
:10BAE000DB0FC93F92E741B99730083C00000000E6
:10BAF000DB0FC940E4CB1641E4CB16C115A82ABE22
:10BB0000DB0FC9BFF82B0020287500202DE9F04F6E
:10BB100007EE900A2DED068BDFEDEC6AEC4D9FED04
:10BB2000ED7AB5F8C0379FEDEC3A9FEDEC4ADFEDCA
:10BB3000EC5ADFF8E4B3C5F81808B8EE679A09EED6
:10BB4000903AC6EE893AB5F8C2379BF8942095F83A
:10BB5000C687C5F8D48783B0002005F5F96105F6DE
:10BB6000782405F67C2CA5F8D80705F68820F8EE91
:10BB7000699A08EE103A39EEA96AB8EEC88AB6EEAC
:10BB8000005AB4EEC68A63EE856AF1EE10FAB8BFC9
:10BB9000B0EE468A86EE886AB5F8C437F7EE004AFA
:10BBA000B4EEE46AF1EE10FAB8BFB0EE646AFDEEEE
:10BBB000C66A29EE077AB8EEE66ACDED016AC3EEF1
:10BBC000866ADFEDC87A90ED01AA81ED028A77EEF0
:10BBD000277A66EE836AC4EE863AC7EE274A89EE74
:10BBE000A67AC8EE267A37EE057A77EE857AB0EE39
:10BBF000006AB4EEC67AF1EE10FAF4EEC47AB8BF79
:10BC0000B0EE467AF1EE10FA08EE903A88BFF0EE08
:10BC1000447AFDEEE77ABDEEC77AF8EEE88A17EED1
:10BC2000907A17EE106A68EEA57A019BC5F8743A0F
:10BC3000A7EB0609C4ED003AC5F8806AC5F8847A16
:10BC400009F1010905F6A42499FBF3F9CCED006A8A
:10BC5000C1ED019A09F10109C1ED007AC0ED004A78
:10BC600005F58D55002A40F0E380DFED9F0ADFEDFA
:10BC70009F5A9FED9F2A9FED9F5ADFED9F2A9FEDD0
:10BC8000AA3ADFEDAA3A9FED9D4ADFEDA91A0BF122
:10BC9000980107EE902AB8EEE76A66EE207A37EE52
:10BCA000A57AFDEEC76A16EE903A2033402B00F2DB
:10BCB0001582F3EE026AB4EEE66AF1EE10FA0CDDDC
:10BCC000DFED974ADFED956AB0EE471AB4EEE61A5B
:10BCD000F1EE10FA37EE647AF6DCB4EEC57AF1EEE6
:10BCE00010FA0CD5DFED8E4ADFED8E6AB0EE471A02
:10BCF000B4EEE61AF1EE10FA37EE247AF6D4B4EE8A
:10BD0000E57AF1EE10FA40F3EC81DFED7D6A36EE74
:10BD1000C77A67EE076AB0EE431AA6EEA21AB0EE33
:10BD2000630AA1EE260A67EE264AA4EE807A27EE81
:10BD3000047AFDEEE76A16EE903A2033402B00F2CB
:10BD4000CA81DFED706AB4EEE66AF1EE10FA40F3F4
:10BD5000F6819FED730A9FED711AF0EE676AF0EEBF
:10BD6000664AF4EEC14AF1EE10FA76EEC06AF6DCED
:10BD70009FED631AF4EEC14AF1EE10FA13D59FED70
:10BD8000681ADFED684AB0EE660AB4EEE40AF1EE36
:10BD900010FA76EE816AF6D4DFED5A6AB4EEE66AFE
:10BDA000F1EE10FA0CDD9FED5E6ADFED5C6AF0EEFD
:10BDB000674AF4EEE64AF1EE10FA77EEC67AF6DC60
:10BDC000F4EEC57AF1EE10FA0CD59FED556ADFED71
:10BDD000556AF0EE674AF4EEE64AF1EE10FA77EEB5
:10BDE000867AF6D4F4EEE57AF1EE10FA40F381812A
:10BDF000DFED436A76EEE77A67EEA76AF0EE434A34
:10BE0000E6EEA24AB0EE631AA4EEA61A27EEA66AE0
:10BE1000E6EE017A67EE847A0132242A81ED007A17
:10BE2000C1ED017A01F108017FF433AF9FED36AA2D
:10BE30004FF0000A019B44F80C7C44E9029344E96A
:10BE400005A64FF49072002120464FF040FC4FF4BD
:10BE50009072A018002104F515744FF038FCA5422B
:10BE6000E8D107EE908A294BB8EEE77ADFED287A21
:10BE700083ED00AAF7EE006A0122C6EE870A8BF86E
:10BE8000942029EE279AB8F1000F00F01F81DFED12
:10BE9000217A9FED1B1ADFED172A9FED145AC7EE8A
:10BEA000A81AA3F52C76A6F1140506F5117738EE3D
:10BEB000698A20EE880A9FED102ADFED0D6A2B4675
:10BEC00030460022F7EE005A36E000BF00247449E5
:10BED000F03C00209C534937398E633C00000C42F3
:10BEE0000AD7233C83F9223DC3B8B23DDB0FC93FDB
:10BEF00000000000DB0F49C092E741B972F97F3FB3
:10BF0000DB0F494000001042BC297E3F7C470020E7
:10BF100027D4D23600004842E84D0020E4CB164139
:10BF2000DB0FC940E4CB16C19730083C15A82ABEE8
:10BF3000DB0FC9BF000010C207EE902AF8EEE77AC7
:10BF4000B6EE007A77EE877AB0EE697AA7EE807A5D
:10BF5000F0EE477A29EE077AE0EC017AFDEEC77A37
:10BF600017EE901A2031402900F2CE80B4EEC17A4B
:10BF7000F1EE10FAF0EE477A0CDD1FED174A5FED97
:10BF8000194AB0EE676AB4EEE46AF1EE10FA77EEA1
:10BF9000C47AF6DCF4EEE27AF1EE10FA0CD51FED7D
:10BFA000204A5FED204AB0EE676AB4EEE46AF1EE33
:10BFB00010FA77EE847AF6D4F4EEC57AF1EE10FA40
:10BFC00040F3B38071EE677A67EEA74A1FED2A4A05
:10BFD0001FED2A6AA4EE824A67EEA43AA4EE246A10
:10BFE000F0EE654AE3EE867AB0EE656AE7EEE14A86
:10BFF000A7EEA16A84EE864AC5EE864A77EE057AF8
:10C00000FDEEE73A13EE901A2031402979D8B4EECC
:10C01000C57AF1EE10FA0CDD1FED3F3A5FED413AC3
:10C02000B0EE677AB4EEE37AF1EE10FA77EEC37A07
:10C03000F6DCF4EEE27AF1EE10FA0CD51FED483A98
:10C040005FED483AB0EE677AB4EEE37AF1EE10FABB
:10C0500077EE837AF6D4F4EEC57AF1EE10FA5ADD73
:10C0600071EE677A27EEA73A5FED513A1FED517AEC
:10C07000E3EE023A63EE278AA3EE237AF8EE003A63
:10C08000E8EE877A67EEA37A87EE867A01329045EA
:10C0900003F12803C3ED0B4A83ED0C7A83ED0E7A8E
:10C0A000C3ED0D4A83ED0F4AC3ED145AC3ED116A77
:10C0B000C3ED106AC3ED136AC3ED126A7FF43CAF9F
:10C0C000C835AF4206F114067FF4F3AE03B0BDEC01
:10C0D000068BBDE8F08FF0EE427A9DE6B0EE427A34
:10C0E00027E6B4EEE17AF1EE10FA48BF35EE477A72
:10C0F0000FE6F4EEE17AF1EE10FA48BF75EE677ADA
:10C100007AE6F0EE667ABFE7B7EE004AF0EE444A10
:10C11000B0EE446A72E71FED7A7AF4EEC77AF1EE78
:10C1200010FA48BF72EEE77A9CE71FED7F6AF4EEE3
:10C13000C67AF1EE10FA48BF72EEE77A44E75FED97
:10C14000836AB4EEE66AF1EE10FA48BFF0EE676A71
:10C150003FF515AE34E600BF10B5204B84B0C824BF
:10C1600003F5DA7103F275122128CDE9022183F873
:10C17000744118D00CD802281ED0082825D102A856
:10C18000019009F0C1FF0198FFF774F904B010BDE8
:10C1900029281AD102A8019009F0ACFE0198FFF7F6
:10C1A00069F904B010BD02A8019009F0EDFE0198F4
:10C1B000FFF760F904B010BD02A8019009F0F4FF88
:10C1C0000198FFF757F904B010BD02A8019009F0DB
:10C1D00053FF0198FFF74EF904B010BDF03C00206A
:10C1E000036870B55E6A26B133460522BDE870402B
:10C1F000184704460D464E1D00E023689B68204604
:10C2000098470028F9D0236815F8011B1B682046C1
:10C210009847B542F1D170BD0A44914217D010B48D
:10C220000139541E11F8013F08225840430010F014
:10C23000800F08BF400083F0D50314BFD8B2C0B24E
:10C24000013AF3D1A142EDD15DF8044B704770473C
:10C250002DE9F047164D0746002095F9BD9105F5EB
:10C26000E27684B007EB010805F2644504464FF01E
:10C27000B60A3368ABB193F83830142B11D019F1EA
:10C28000020F01D04B450CD1002269463046CDE962
:10C290000244CDE90078ADF808A08DF80E4029F0F1
:10C2A0001DFBE036B542E4D104B0BDE8F08700BF25
:10C2B000E84D002030B583B04D1C009303688572B3
:10C2C000C2729C690023A04703B030BD2DE9F04144
:10C2D0000C4F0124A0231825E6B2FF2B0BDCC5F17F
:10C2E0001B0103F10108D7F86404DBB23246C9B27E
:10C2F000FFF7E0FF4346013DEFD10134052CEAD1C1
:10C30000BDE8F081E84D002070B4447941BB03687A
:10C310004FF400524FF40076202502213CBB1A8CCA
:10C3200022F001021204120C1A841A8B188C22F0CB
:10C33000F30280B2120420F00A00120C014342F012
:10C34000010241F001011A8319841A8B22F00C02B8
:10C350001204120C1A831A8B92B270BC1A837047A3
:10C3600000220368164615461146002CD7D0042C2F
:10C3700021D0082C38D0198C21F480510904090CE3
:10C3800019849C8B1D8C45F6FF7040F6FF412840B8
:10C390002140024342F4805241F4807199831A840F
:10C3A0009A8B22F440621204120C9A839A8B92B2F6
:10C3B00070BC9A8370471A8C22F010021204120C7F
:10C3C0001A84188B198C89B240F6FF4221F0A00123
:10C3D00002400D4342F4807245F010051A831D841B
:10C3E0001A8B22F44062B3E71A8C22F48072120492
:10C3F000120C1A84998B1A8C21F0F30192B2090461
:10C4000022F42062090C324342F4807241F00101AF
:10C4100099831A849A8B22F00C02C4E70B88F0B43B
:10C4200033BB028C4C880E898B88C98822F00102AC
:10C430001204120C0284058B028CADB225F0F305B8
:10C4400092B22B4322F00A0243EA061322439BB224
:10C4500042F0010203830284038B23F00C031B04CC
:10C460001B0C0383038B9BB21943F0BC0183704701
:10C47000042B048C2CD0082B4E888A880D89C988FF
:10C4800051D024F480542404240C0484838B078C1E
:10C490002C0344EA022440F6FF421A4045F6FF739B
:10C4A0003B4043EA063322439BB292B243F48053AB
:10C4B00082830384828B22F440621204120C8283F2
:10C4C000838B9BB243EA01239BB2F0BC838370470A
:10C4D00024F010042404240C4D880F898A88C9880C
:10C4E0000484068B038C12029BB242EA073423F0C9
:10C4F000A00340F6FF42324043EA051322439BB2B9
:10C5000092B243F0100302830384028B22F4406250
:10C510001204120C0283038B9BB243EA01239BB2E9
:10C52000F0BC0383704724F480742404240C048436
:10C53000848B038CA4B29BB224F0F30423F4206315
:10C54000224343EA062342EA05129BB243F4807376
:10C5500092B282830384838B23F00C031B041B0C95
:10C560008383838B9BB21943F0BC8183704700BFE8
:10C570002DE9F04F824C94F8DE8694F8E9A687B056
:10C5800016460B22054689464046114602959DF8FF
:10C5900040701D4633F0FAFBC245834640F0B08040
:10C5A0000390404637F0E2FE17F00803024601937D
:10C5B00000F09A80BBF1000F00F092809BF807100A
:10C5C000890700F18D80C4F8ACB4C4F8A804C4F89D
:10C5D000A40410B140F60B31C18005F0020ADFF867
:10C5E000B881029B674A84F86C5408F58071002575
:10C5F0005846C4F89434C4F880144FF4807331461C
:10C60000C4F86824C4F87434C4F87834C4F8706486
:10C6100084F86D74C4F89894C4F87C84C4F8885481
:10C62000C4F88454C4F89054C4F88C54C4F8C05668
:10C6300084F8C456A4F8B85628F01AF8D4F8AC0414
:10C6400007F00101FFF760FE4F4A504BD4F8AC04ED
:10C65000C4F8CC56C4F8D026C4F8C836BAF1000FD6
:10C6600025D0D4F8B07417B33A6803689A421ED044
:10C6700001233146384684F8C53627F0F9FFD4F84F
:10C68000B00408F50572294632F0E2FFD4F8AC0494
:10C690002A4608F5077132F0DBFF019B93B93C484D
:10C6A00027F0FEFF3A48012128F032F80AE0394A23
:10C6B000002302F1080184F8C53632F0C9FF019B5E
:10C6C000002BECD0324827F0F7FF314807B0BDE827
:10C6D000F08FCDE90403039B13B1D9798B0716D5ED
:10C6E000002007B0BDE8F08F15F00103F1D105F08F
:10C6F00002018A46BAF1000F22D1D4F8ACB46EE739
:10C700000B220C21504633F041FB039049E7504681
:10C7100037F02CFE039AC4F8AC2415F0020ADDE9C8
:10C720000423C4F8A40405F0020123D0904219D0D8
:10C73000C0B140F60C3CA0F806C0BAF1000FDCD046
:10C74000B8F1000FCCD0C4F8A82483B9BBF1000F16
:10C75000C6D0C4F8ACB412B140F60B33D3805FFA44
:10C7600081FACAE7B8F1000FBAD0C4F8A824C4F817
:10C77000B0B4F0E70028DCD1DDF80CB02FE700BF43
:10C78000E84D002008B80508A50803082947030854
:10C7900050520020B05400209C520020F0B5C54BF0
:10C7A000C54EC64DC64C0822C3F88820336B83B0F3
:10C7B00043F00103336307464FF4C052284640F26A
:10C7C00002336946CDE90023FBF71AFC6A6AC4F814
:10C7D000DC7C22F470426A626A6ABA4BC4F8E03CBC
:10C7E00042F420426A626A6AB748C4F8F80622F442
:10C7F00070226A626A6AB548C4F8FC0642F42022D4
:10C800006A62726CB24DC4F8085742F48042726496
:10C81000726BB048C4F8100742F0800272630222C3
:10C8200084F80027AC4FAD4AAD49C4F814771C33E7
:10C830004FF0A046C4F8E43CC4F80467A94BC4F820
:10C84000182705F5487506F51666C4F85057C4F85C
:10C850005437C4F81C670123DFF8B4C2C4F84CC7CE
:10C8600007F51077A5F5E465A2F5A062A6F58C663C
:10C87000C4F85877C4F80C57C4F8C42784F80337B1
:10C8800005F5A0754B61C4F888671946A03684F891
:10C890000A38954BC4F8905702F59072A7F5BC671B
:10C8A000A035C4F89C67914EC4F89427C4F89877D3
:10C8B00002F52A6207F5D457C4F8A037C4F8A45784
:10C8C00003F569534FF050250020ACF5BC6CC4F85B
:10C8D000C827C4F8CC7702F5A04207F5A047C4F8F2
:10C8E000D067C4F8D43706F5A046A3F54853C4F87A
:10C8F000D85704F5DF65C4F8DC27C4F8E467C4F84A
:10C900000438C4F88CC70246C4F8E0772B4684F894
:10C910000C08402683F81C21A3F822210132042AA6
:10C92000C3E9496083F81D1183F81F01C3F8300182
:10C9300003F12803EED1002211462B46402083F854
:10C940007423A3F87A230132042AC3E9DF0183F8B0
:10C95000751383F87713C3F8881303F12803EED116
:10C960004FF0A04362489A6822F001029A60DA68A8
:10C9700042F04002DA60FBF7FBFD94F80137002239
:10C98000212161F317420BB142F4801294F8FB1697
:10C99000D4F8043701299A6300F0DF80DA68D4F80C
:10C9A0000468D4F80807C2F3076121F0600141F080
:10C9B000400161F31F620021DA603160026861F3B7
:10C9C000CC22026094F80327012A00F0B3801021E2
:10C9D0004848FCF7A9F84748FCF78CF8D4F8080752
:10C9E00094F8F93600224FF0FF3102614261816113
:10C9F000C26153B305F114073F4E114607EB83079D
:10CA00004FEA830C4FF0FF0E56F8042F1368002BEB
:10CA1000ACBF00234FF09043B74213601161C2F8DE
:10CA200008E0F1D105F15003344963440027FF26A3
:10CA300051F8042F1568002DACBF00254FF090452C
:10CA40009942156017619660F2D1036994F8FB165C
:10CA500043F48073012903615CD0D4F8042728488B
:10CA60000023936100294FF0FF336FF08041516143
:10CA70005360516114BF00231023906143F470137D
:10CA80009069D4F8E01C43F4605343F00803034377
:10CA900093619368096843F0010393608847194BD9
:10CAA000194ADA606846194B0093FDF743FC03B05E
:10CAB000F0BD00BF00E100E000380240000002408D
:10CAC000E84D0020B80200200804010040004001A9
:10CAD0000008005000090050200900504009005093
:10CAE000003C0140400B0050C00500500030005099
:10CAF000EC540020E0540020F45400203055002075
:10CB00000008008000ED00E00005FA054302000186
:10CB1000000B0050D4F80427144B03636FF08041DE
:10CB2000134D00234FF0FF3093615161506051610C
:10CB30009561A3E701680F4A0F4E41F003010160C0
:10CB4000802159629E62C3F80421E022C3F80821C3
:10CB5000C0F24002C3F80C2139E79A6822F03E0186
:10CB600041F02A0161F307029A6017E7030181008F
:10CB700000080080A0004000800020002DE9F04760
:10CB80009AB0DDE9226ADDF8909004460D4617461A
:10CB9000984602E0206834F0CBFB206834F0D0FBEC
:10CBA0000028F7D10146642201A84EF090FD264BE3
:10CBB0008DF80450CDF85CA00293002D3FD0AB1E41
:10CBC000012B3ED9042D14BF002203221F4B0396D4
:10CBD0001B6B8DF805201E440123CDE905940496B6
:10CBE0008DF85B3037B14246394607A84EF00EFD4E
:10CBF0008DF85A80164E96F82E9D00231893B9F1A1
:10CC0000000F19D196F82D0D642202FB006001A9D6
:10CC100000F553604EF0FAFC012386F82D9D86F84E
:10CC20002E3D236843B143463A46294620461AB072
:10CC3000BDE8F0470DF0B0BC1AB0BDE8F0870522A2
:10CC4000C4E70222C2E700BFD45A0020F82B00201C
:10CC5000E84D00200C480D4BD0F8B01D10B40C4C22
:10CC6000C0F8A03D8A1E2231B0F8CE3D1B01A4FBC6
:10CC700003C3DB08A3F5B06322F8023F9142F3D16E
:10CC80005DF8044B704700BFE84D0020E532020814
:10CC9000CDCCCCCC70B5084C251D2E4614F8010B1C
:10CCA0002CF052FA28B1037805F8013BB442F5D1D3
:10CCB00070BDFF23F8E700BFD85B00202DE9F047E7
:10CCC0001D4F012607F10805B2464FF03C094FF011
:10CCD000000817F8010B37F049FB044690B180F8C3
:10CCE0000690C671FB7803F07F02012A18D013F07A
:10CCF000800F20460DD185F8048037F0FFFD85F8C0
:10CD000005802C600136052E05F10805E1D1BDE84E
:10CD1000F08785F804A037F0F7FD85F805A0F0E767
:10CD20001B0605D40121204633F02CFAFB78DEE700
:10CD300037F0EAFDF6E700BFE05B00202DE9F04F99
:10CD4000DFF8FC91DFF8FCA183B009F10C060124A7
:10CD500019F8018BB8F1000F00F0C6804FEA1815E2
:10CD6000013D032D08F00F0200F2C1800AEB4503DC
:10CD7000B3F8400040FA02F717F0010700F0D28044
:10CD800001239340013B184055444BF0AFFF95F809
:10CD90004830664F184407EBC00704237761FC71E5
:10CDA000BB71002302E0152B00F09E8003EB4302D1
:10CDB0005F49895C41454FEA430B03F10103F2D11E
:10CDC0005C4B1A4492F8A518002900F0AD8040464B
:10CDD00032F060FF0546284632F0A2FF0378002BB0
:10CDE00040F08280534B5B44042283F8E54883F88B
:10CDF000E428002D78D0002F5DD03B68287A03F11D
:10CE00003F4202F57E020AEB92224FF0010C92F8AB
:10CE10004C2002F01F015209032A0CFA01F171D0D3
:10CE2000042A67D0022A75D0B7F804E0BEFA8EF261
:10CE3000C2F11F02C2F3CC0103EB810102F0070231
:10CE40000F6A92004FF00F0C0CFA02FC27EA0C0755
:10CE50000F620F6A90403843002208624FF0010BC6
:10CE600011460BFA01FC3CEA0E0001F101011ED152
:10CE700018680327974020EA07001860D3F800805D
:10CE80000220904040EA08001860986820EA0700F5
:10CE9000986098689860586820EA0C005860586854
:10CEA0005860D86820EA0700D860D868D860102990
:10CEB00002F10202D5D1204B204AB3F8201EB3F86C
:10CEC000223E0091002001340190B2FBF3F3304682
:10CED0009BB22946E4B227F079FD0123092C737433
:10CEE00006F118067FF434AF03B0BDE8F08F0027D9
:10CEF000776156E7DFF850C0DCF830200A43CCF801
:10CF0000302091E7DFF840C0DCF840201143CCF836
:10CF1000401089E7DFF830C0DCF844201143CCF83A
:10CF2000441081E777613CE70D4654E7083500205F
:10CF30009C340020F82B0020E84D002040420F00D8
:10CF40000C5C002070B70508003802402DE9F04164
:10CF50002A4C2B4DB4F8F46EA5F8A46C82B0EEB94F
:10CF600094F8F00E37F002FA94F8F12EC5F8A80CF8
:10CF7000003A18BF012285F8A62C48B194F8F21E99
:10CF80002B22002914BF11210121C28033F0FAF8AD
:10CF9000002002B0BDE8F0413AF066BB94F8F08E94
:10CFA000002240462B2132F0F1FE0746404637F082
:10CFB000DDF9F8B1F7B12B22C5F8C00CC280397A7F
:10CFC000FDF7FAFD4FF000080E4AB2FBF6F3C3F38B
:10CFD0004F0000909BB23946CDF8048005F6AC4076
:10CFE000A4F8F66E27F0F2FCD5F8AC3CC3F800804C
:10CFF00085F8BD8C02B0BDE8F08100BFE84D00208F
:10D00000F82B002040420F002DE9F84F254C94F8F2
:10D01000043F84F8F83E04F6FB67002604F6187413
:10D020005FFA86FB0BF101085FFA88F8012117F817
:10D03000010F42460E448A4632F0A8FE4FF0000926
:10D04000054640B3387804F80E9C04F80D9C04F8AB
:10D050000FBC04F810AC44F8045C37F087F918B141
:10D0600080F806A080F80780297AFDF7A5FD0E4A12
:10D070000021284632F018FC0C4B23600C4B221D7B
:10D0800021462846C4E9013932F0E2FA6979286874
:10D090004A4627F037FC082E04F11C04C0D1BDE835
:10D0A000F88F00BFE84D002040420F003D490308C3
:10D0B00089FA020870B541F224032D4C2D4E2E4DF5
:10D0C00016F8C80C002241F22801E25041F22C036C
:10D0D00065500221E252C4F8E82FC4F8EC2FC4F8DE
:10D0E000F02F32F053FE002841D0244B0268054651
:10D0F00003F1C000597C11B159688A422BD0183312
:10D100008342F7D1002316F8C80CC4F8145F84F8E2
:10D11000083F37F02BF908B10223C380297AFDF7C5
:10D120004BFD2846164A002132F0BEFB154A16492F
:10D13000C4F8181F0026111F2846144BC4F81C3FC2
:10D14000C4F8206F32F084FA697928683246BDE865
:10D15000704027F0D7BB138D0D490E4A9BB2D2F811
:10D16000982A0133B2FBF3F381F85831CAE770BD56
:10D17000E84D0020E05E002000FFFF00DC330020CF
:10D1800040420F00045D0020B1FA020851FC020881
:10D1900098010020F82B00202DE9F04FD24DD34C00
:10D1A00085B007460E4605F2E470C02200214EF01D
:10D1B0008EFA14F85C3C002B00F0E88014F85B3C1D
:10D1C000002B00F0018195F86437012B72D0022BFF
:10D1D00000F00681C64BDFF83CC303931F46BCE852
:10D1E0000F000FC7BCE80F000FC795F85AE795F876
:10D1F00056379CE80700DFF820C344F878CCBEF12E
:10D20000000C18BF4FF0010C072B87E8070004F84B
:10D2100059CC00F23881042B00F24681DFF8FCB2D1
:10D22000ABF17E034FF00008029346454FF0030137
:10D230003EDD029B13F801AB029305EB0A030AF1F2
:10D24000010993F85B775FFA89F938464A4632F06C
:10D250009DFD034638461F46002B00F01D8137F028
:10D2600085F8CBF8140020B14FF00303837180F8E8
:10D27000079095F8572795F856375FFA88F1002AF6
:10D2800000F00881FA7982F0010200923846524695
:10D2900008F1010848F0F2FD002800F0FD804FF091
:10D2A0000103B8F1080F8BF811300BF1180BBCD14A
:10D2B000039B69E0DFF868C28E4FDFF8608244F8B4
:10D2C000546CBCE80F000FC7BCE80F000FC79CE808
:10D2D000070095F8563795F85AC704F8143C002310
:10D2E000BCEB030C87E8070018BF4FF0010C9B460E
:10D2F00007F1940019464FF4407204F859CC04F831
:10D30000583C07F5657A4EF0E2F9A8F17E090296DD
:10D310005E4654F8543CB34240F3AC8019F8013BEC
:10D320002B4493F85B77384632F0B6FD8346384697
:10D3300037F01CF895F857370746002B00F09D8012
:10D340009BF8073083F0010B0BF0010114F8590C26
:10D35000013104F85A1C08B18BF0010B002F00F0CA
:10D36000B380B87900285CD041285AD0624B634919
:10D37000634A44F8A83C029E44F8AC1C012304F81C
:10D38000583C44F8A02C0023C5F84C32D5F84C3258
:10D390005BB10022012183F82C6083F82D101A6301
:10D3A00083F82E2005B0BDE8F08F564E564C0FCEB8
:10D3B0000FC40FCE0FC496E80700A4F1200384E841
:10D3C0000700C5F84C32EDE795F85827003A384683
:10D3D00018BF01223146FBF7D7FEC5F84C02D5E74E
:10D3E00095F85A37002B3FF4F5AE95F85637082BD1
:10D3F0007FF460AFDFF81CC1DFF81CE1BCE80F0070
:10D40000A4F1900703970FC7BCE80F000FC79CE873
:10D410000700012387E8070004F8593C44F878EC3A
:10D4200034E0B888CAF80C704901B0FA80F041F0D5
:10D4300009010136C0F11F004FF00303CAF80400D0
:10D44000CAF814108AF810B0FE71BB71384632F079
:10D4500099FE1BF0010F384612D037F04FFADAF878
:10D460000C30C8F81430082E0AF1200A08F1180808
:10D470007FF44FAF029E1F4B86E79BF807B063E730
:10D4800037F042FAEBE7082B7FF4C8AE1F4B44F8A5
:10D49000503CC3E6FA79F8E6194B174A44F86C3C5D
:10D4A00044F8742C00236FE795F85937184A44F86C
:10D4B000502C012B05D0022B06BFBEFA8EF35B0960
:10D4C000002304F84C3CA9E6490141F009014FF062
:10D4D000FF33CAF81410CAF80430CAF80C708AF87E
:10D4E00010B00136B2E700BFF82B0020E05E00204C
:10D4F000505E00201C5E002085E7030889E70308D2
:10D500007DE7030838B80508985E0020FD7A040816
:10D510002D7B040864B80508E9150508DC330020F4
:10D5200090B805082DE9F84FD34F97F8C80D97F834
:10D53000C95D36F01BFF60B12D23C3802021044656
:10D5400032F020FE0A2033F04DFA20463AF0C0F8BF
:10D5500020B9CA4BD3F8F033DE0001D5BDE8F88F0F
:10D56000013D092DFAD897F8C75DD5B940202DF0B7
:10D5700065FB0028F2D090F9043097F8991D092B2B
:10D58000C8BF143B3B440A2993F8D45600F0B1813C
:10D5900093F8DF3697F8C62D002A08BF1D46002DE8
:10D5A000DCD0284636F0E2FE8046002800F0998163
:10D5B0002D23C380012132F0E5FD0121084637F01B
:10D5C000B1F9D8F80030B8F804201A833C2033F0C1
:10D5D00027FB0021012037F0A5F997F8C93D002B62
:10D5E00000F0CC80A64CDFF8A092A64D002694F85F
:10D5F000941CD4F8980CC94301F0010137F08AF962
:10D6000094F8941CD4F8A00C81F00401C1F38001BB
:10D6100037F080F9B8F1000F04D0D8F80030B8F82E
:10D6200004205A83D9F80430C3F30803002B40F0D8
:10D63000FF80EFF31183002B40F0FA80226BA96882
:10D64000236B9A42FAD1D4F8903C9942F6D8D4F898
:10D650008CCC4FF47A7000FB0CF35B1AB3FBFCF339
:10D6600000FB02324FF0100C4FF47A710120D9F810
:10D670000430C3F30803002B40F0BA80EFF31183AA
:10D68000002B40F0B580236BD5F808B0D4F830E01B
:10D690007345F8D1D4F890ECF345F4D8D4F88CACB9
:10D6A00001FB0AFEAEEB0B0EBEFBFAFE01FB03E331
:10D6B0009B1A772BDBD994F8941CD4F8980C01F0C2
:10D6C000010137F027F994F8941CD4F8A00CC1F3A9
:10D6D000800137F01FF9B8F1000F04D0D8F80030FE
:10D6E000B8F804201A83D9F80430C3F30803002BD8
:10D6F00040F0CC80EFF31183002B40F0C780226B09
:10D70000A968236B9A42FAD1D4F8903C9942F6D892
:10D71000D4F88CCC4FF47A7000FB0CF35B1AB3FB9B
:10D72000FCF300FB02324FF0100C4FF47A71012031
:10D73000D9F80430C3F30803D3BBEFF31183BBBBA9
:10D74000236BD5F808B0D4F830E07345F8D1D4F89D
:10D7500090ECF345F4D8D4F88CAC01FB0AFEAEEBA8
:10D760000B0EBEFBFAFE01FB03E39B1A772BDFD9FE
:10D7700097F8C93D01369E42FFF639AF97F8C73D8D
:10D78000002B40F0A680D7F8C83D03F0FF13B3F597
:10D79000803F7FF4E3AE394BD3F8F03313F080537E
:10D7A0007FF4DCAE87F8C93DBDE8F84F46F02CBEEB
:10D7B000EFF3118A8CF31288D5F808B02B68DB03DD
:10D7C00044BFC4F8880CD5F808B0236BD4F888ECB3
:10D7D0005FFA8AFA8AF31188D4F88CAC734401FB9F
:10D7E0000AFEAEEB0B0EBEFBFAFE01FB03E3BCE749
:10D7F000EFF3118A8CF31288D5F808B02B68DB039D
:10D8000044BFC4F8880CD5F808B0236BD4F888EC72
:10D810005FFA8AFA8AF31188D4F88CAC734401FB5E
:10D820000AFEAEEB0B0EBEFBFAFE01FB03E33FE785
:10D83000EFF31181102383F31288D5F808C02B6809
:10D84000DA0304D50123C4F8883CD5F808C0236B5B
:10D85000D4F8882CC9B281F31188D4F88C0C4FF419
:10D860007A711A4401FB00F3A3EB0C03B3FBF0F352
:10D8700001FB0232F6E600BFE84D0020E05E00202A
:10D88000F82B002010E000E000ED00E0EFF3118144
:10D89000102383F31288D5F808C02B68DA0304D567
:10D8A0000123C4F8883CD5F808C0236BD4F8882C31
:10D8B000C9B281F31188D4F88C0C4FF47A711A44F0
:10D8C00001FB00F3A3EB0C03B3FBF0F301FB02320B
:10D8D00029E7322033F0A4F94046002132F052FC0F
:10D8E00051E7012132F04EFC0121084637F01AF8C9
:10D8F0006CE6074CD4F8D43B5C057FF52FAE08F0FE
:10D90000D5FE00287FF42AAE002D7FF44AAE25E62E
:10D91000F82B00202DE9F041214E224F96F8F733E5
:10D9200087F8943C06F57D7607F6984500244FF07D
:10D93000050816F8010B20BB28600134032C05F103
:10D940000405F6D197F8941CD7F8980CC94301F058
:10D95000010136F0DFFF97F8941CD7F89C0C81F09A
:10D960000201C1F3400136F0D5FF97F8941CD7F8B7
:10D97000A00C81F00401BDE8F041C1F3800136F054
:10D98000C9BF36F0F3FC013401212860E3B210B1C5
:10D9900080F80680C371286832F0F4FBCEE700BF40
:10D9A000E05E0020F82B00200B6810B414681B1BED
:10D9B000036054684B681B1B43608B6892685DF87A
:10D9C000044B9B1A836070472DE9F047041E0D46F7
:10D9D00012DB092C26DC824A0B468248A0FB04108D
:10D9E000C00800EB8000A4EB40000021125C1A701C
:10D9F00059702846BDE8F08764422D23092C01F8B0
:10DA0000013B24D8764A774BA3FB0403DB0803EBE6
:10DA10008303A4EB43030020D35C48700B702846BB
:10DA2000BDE8F0876F4B632CA3FB04264FEAD606B4
:10DA300021DC6B4A0B466B49A1FB0601C90801EBCF
:10DA40008101A6EB4101515C03F8011BC5E7654A62
:10DA5000632CA2FB04364FEAD60637D8604A614BE6
:10DA6000A3FB0603DB0803EB8303A6EB4303D35CB2
:10DA700001F8013BC7E7A3FB0627B4F57A7F4FEA1D
:10DA8000D7070DD2564A0B465649A1FB0701C908D4
:10DA900001EB8101A7EB4101515C03F8011BCAE7CF
:10DAA000A3FB072842F20F7294424FEAD80836D8F7
:10DAB0004B4A0B464B49A1FB0801C90801EB810108
:10DAC000A8EB4101515C03F8011BDDE7A2FB06371F
:10DAD000B4F57A7F4FEAD7070CD2414A414BA3FBFA
:10DAE0000703DB0803EB8303A7EB4303D35C01F8D5
:10DAF000013BB4E7A2FB073842F20F739C424FEAA6
:10DB0000D80821D8364A374BA3FB0803DB0803EBC0
:10DB10008303A8EB4303D35C01F8013BDEE7324A01
:10DB2000A3FB080994424FEAD90921D82C4A0B4695
:10DB30002C49A1FB0901C90801EB8101A9EB4101B5
:10DB4000515C03F8011BB5E7274BA2FB08099C4277
:10DB50004FEAD90921D8224A224BA3FB0903DB084B
:10DB600003EB8303A9EB4303D35C01F8013BCAE752
:10DB70001E4AA3FB090394424FEAD30A21D80B465D
:10DB80001849174AA1FB0A01C90801EB8101AAEB58
:10DB90004101515C03F8011BCAE7144BA2FB0902C7
:10DBA0009C424FEAD20A13D80E4B0D4AA3FB0A033C
:10DBB000DB0803EB8303AAEB4303D35C01F8013BCF
:10DBC000CAE70A22BAFBF2F046F010FA0346D7E79A
:10DBD0000A22BAFBF2F046F009FA0146E4E700BF78
:10DBE000182F0608CDCCCCCC9F8601003F420F00F9
:10DBF00070B4344890F8F833A3F13001092957D8AC
:10DC000000F57E74224600F2074012F8015FA5F18C
:10DC10003001092904D88242F7D1002070BC704736
:10DC2000141B022C4ADD2848002101E010F8013BBA
:10DC300001EB810103EB4103161A303B022E04462F
:10DC400003F0FF01F2DC214B03FB01F1A2424FF094
:10DC500000030DD903EB830314F8016B5B00303B29
:10DC60003344A24203F0FF03F4D1194800FB03F34D
:10DC70002E2D06D01748A0FB032301EB930070BCA8
:10DC80007047013204200024157804EB8404303DF1
:10DC90006400092D00F1FF30A4B202D82C44A4B2D4
:10DCA000013210F0FF00EFD1642202FB0433E1E700
:10DCB00000211D4600F57E720B46D9E7064C002177
:10DCC000C4E700BFE05E0020D96200208096980083
:10DCD00040420F00ABAAAAAAD862002038B5044679
:10DCE0000D460A460068FF214DF0F1FC21682944E9
:10DCF000216038BD83B50C46164605462BF0DAFA8E
:10DD000020462BF0D7FA0021204B0846002E08BFF2
:10DD10001E4636F007FE0021012036F003FE28469D
:10DD200033F00EFBB0B10121002036F0FBFD284698
:10DD300033F0FEFA0746204633F0FEFA0028FAD008
:10DD40003946204633F000FB3846B04700210846EC
:10DD500036F0E8FD204633F0F3FA0028DFD0012149
:10DD6000002036F0DFFD204633F0E2FA0146284677
:10DD7000019133F0E1FA01990028F8D0284633F0F8
:10DD8000E3FA0021084636F0CDFDC8E7B591030857
:10DD9000F0B50023C1E90033C1E902330B61026829
:10DDA000DFF88CC089B004ADC2F385572E4647FA20
:10DDB00003F0C007344604D513F80C0004F8010B37
:10DDC00026460133062BF2D11748C2F3032404443C
:10DDD000002394F8544133708DF8184000F5AE7C60
:10DDE000C2F305370DF1190647FA03F0C0073446B0
:10DDF00004D513F80C0004F8010B26460133062B5A
:10DE0000F2D100233370C2F3834406ABCDE9013471
:10DE1000084602F00F0305490095C2F3031247F0CC
:10DE200023F909B0F0BD00BF70B70508402F060800
:10DE3000BCB8050870B5094CD4F80824054662B191
:10DE40000026D4F808042D2101363AF0E5FFAE4251
:10DE5000F7DBBDE870403BF015BA70BDE05E002016
:10DE600038B50F4C94F8131401F03F018B1C024697
:10DE700001F10A0584F8113484F80E5404F20C40C0
:10DE800084F80F24083118F00DFF254485F80A04A2
:10DE900094F80E341C44000A84F80B0438BD00BF0B
:10DEA000E05E002070B51D4C0968D4F8545B1C4E30
:10DEB000D4F8504BD6ED577ADFED1A6A491B00EEC5
:10DEC000901A0168F8EEE00A091B60EEA70A00EE5E
:10DED000101A20EEA07AB8EEC00A1C46A0EE007A16
:10DEE000B1EE400AF1EEC77A67EEA67AFCEEE77A69
:10DEF000C2ED007A47F0A2F99FED0B7ADFED0B7AC5
:10DF0000E0EE077AFDEEE77A17EE902A002ABCBF12
:10DF100002F50C42A032226070BD00BFF82B002039
:10DF2000980100202C7D8E3FA00CB34500A00C462C
:10DF300038B50B4C00250122802120462CF06AFECA
:10DF400030B194F904002CF097FE08B1006838BD98
:10DF50000135042D04F10C04EDD10020F7E700BFDA
:10DF60001463002038B5041F00F1080554F8043F7D
:10DF7000D81780EA430013F04DF9A542F6D138BD19
:10DF8000F8B5C44CDFEDC47AD4F8682494F8D034E2
:10DF9000B4F8D27407EE102A2DED028BB8EE478A42
:10DFA00028EE278A002B60D1D4F8DC3494F8ED24D5
:10DFB000002B40F3FC8007EE902A9FEDB86ADFED5E
:10DFC000B86AF8EEE77AB7EE007AA7EE867AF0EE56
:10DFD000477A07EE103AF8EEC78AB7EE087A87EE6E
:10DFE000270AC6EEA87A20EE270A4BF069FE0F2812
:10DFF000B8BF0F2094F8D13485B2A4F8D254002BC6
:10E0000000F03C81AF4234D0B4F8D4349FEDA56A1F
:10E0100094F86C6407EE103A07EE905AB8EE477A1F
:10E02000F8EE677AC6EE076A86EE277A76EE887A89
:10E0300037EE087AC8EE276AC8EE077AB6B39A4B6D
:10E0400094F8D624B4F8D854C3ED047AC3ED087A12
:10E05000C3ED0C7AC3ED106AC3ED147AC3ED187AE0
:10E06000002A49D0BDEC028BF8BD94F8D134002BC6
:10E0700072D094F86C64002E40F0F880B4F8D43478
:10E08000DFED886A07EE907A07EE103AB8EE676A1D
:10E09000B8EE477AC6EE877A86EE867A77EE887A89
:10E0A00037EE087AC8EE276AC8EE077A7E4B94F8F6
:10E0B000D664B4F8D85400225A609A60DA605A6183
:10E0C0009A61DA615A629A62C3ED047AC3ED087A02
:10E0D000C3ED0C7AC3ED106AC3ED147AC3ED187A60
:10E0E000DA625A639A63DA635A649A64DA645A6544
:10E0F0009A65DA65002E65D1D4F8DC3494F8ED2405
:10E10000002B40F3948007EE902A9FED646ADFEDC8
:10E11000646AF8EEE77AB7EE007AA7EE867A07EE41
:10E12000903AF8EEE77AB7EE086A86EE070A86EECE
:10E13000A77A20EE070A4BF0C3FD0F28B8BF0F20C7
:10E1400080B2A4F8D804002E3BD0A8428AD0002880
:10E1500074D1BDEC028BF8BDD4F8DC3494F8EE2415
:10E16000002B40F38E8007EE903AF8EEE78A3D46AA
:10E1700007EE902A9FED496ADFED496AF8EEE77AEB
:10E18000B7EE007AA7EE867AF0EE477AB7EE087A15
:10E1900087EE270AC6EEA87A20EE270A4BF090FDFC
:10E1A0000F28B8BF0F2080B2A4F8D4042AE794F84F
:10E1B000D1340F25A4F8D254002B7FF423AF284686
:10E1C000F2E7054694F8EC3484F82538002D3FF446
:10E1D00049AF07EE905A9FED336A344BF8EE677AF9
:10E1E000D3ED006A86EE277ABDEC028B0022012176
:10E1F000C3F8042384F82418C3F80823C3F80C23B5
:10E20000C3F81423C3F81823C3F81C2337EE267A67
:10E21000C3F82423C6EE877AC3F82823C3F82C2337
:10E22000C3EDC47AC3EDC87AC3EDCC7AF8BD0F2034
:10E23000A4F8D80446B30F2D3FF414AF07EE900AAC
:10E24000DFED186A194BF8EE677ABDEC028B86EEAB
:10E25000A77AD3ED006A37EE267AC6EE877AC3ED49
:10E26000C47AC3EDC87AC3EDCC7AF8BD94F8D6343D
:10E27000B4F8D854002B7FF4F5AE3DE794F8EE24C3
:10E2800076E73D460F208FE794F8EC3484F8253884
:10E2900005469EE7E05E0020BD378635CDCCCC3DFF
:10E2A000002474494E2DA63D4C630020D06300200D
:10E2B0001D4991F8F823A2B3F0B400260546334671
:10E2C000304637461BB991F8F8432D2C23D02E2A1F
:10E2D00019D0CA1800EB800092F8F843A4F130027C
:10E2E000092A4FEA40009CBFA0F13002A0180E2B73
:10E2F00014D80133CA1892F8F823002AE2D106B1E3
:10E300004042F0BC70470133002DF8D0CA182A44AF
:10E3100082F8F873DDE701231E46EBE70020F0BC2E
:10E3200070470020704700BFE05E00201FB503ACBF
:10E330008DF80C30009400238DF80D3009F054F85E
:10E3400004B010BD10B5FBF7F1FF1121044631F008
:10E3500019FF204636F0D2FAC82032F061FC204680
:10E36000BDE8104036F0D0BA704700BF704700BF1C
:10E37000704700BF704700BF70B501F07F0505EB27
:10E38000850400EBC404282101FB05010126C4F823
:10E3900030310023C4E94A2284F81C5184F81D61FD
:10E3A000C4F8343101F58E711DB9FAF725F9002052
:10E3B00070BDFAF795F9002070BD00BF2549D1F86E
:10E3C00078380F2B04D05A1CC1F8782800207047E9
:10E3D00070B5214C94F820590023C1F87838F5B96C
:10E3E000D4F80829D4F80C39B2F5006F19D09A4244
:10E3F0002CD01AD9C2F50063402B18D9403B02F14A
:10E400004005C1F87C38012384F82039C4F8085944
:10E4100092B2402311490A448121FFF7ADFF002049
:10E4200070BDC4F808598BB12A469B1AE4E74FF037
:10E43000000502EB0306C1F87C580CBF0221012144
:10E44000C4F8086992B284F82019E3E7002384F83D
:10E450002039E4E7E05E0020001B00202424002097
:10E46000ACE700BF70B51E4C94F82039012B03D0E7
:10E47000022B0AD0002070BD01461A48D0F87C3823
:10E4800053B984F82039002070BD00231A46812139
:10E49000FFF772FF0023F4E7402BD4F8082910D9C6
:10E4A000403B02F14005C0F87C38C4F8085992B2EC
:10E4B00040230D4C084622448121FFF75DFF0020D8
:10E4C00070BD4FF0000503EB0206C0F87C5808BF92
:10E4D0000220C4F8086992B208BF84F82009E8E76E
:10E4E000001B0020E05E002024240020012905D02C
:10E4F00008B50321FAF718FB002008BDB2E700BFFA
:10E5000010B5002304220446194680F811211A464A
:10E51000FFF732FF2046FAF751F8002010BD00BF88
:10E5200010B5044629B990F81131032B0DD0002005
:10E5300010BDD0F8E4359B69002BF8D090F812217B
:10E54000032AF4D19847002010BDD0F89013D0F8DA
:10E550007C33994214D9C078D4F880230128A1EBE8
:10E56000030104BFD218C4F880238B4228BF0B4696
:10E57000C4F890139BB220460021FAF769F9D6E758
:10E58000D0F8E4351B691BB190F81221032A03D09F
:10E590002046FFF7B5FFCAE79847F9E738B51346B5
:10E5A00002250A46C0E94E3380F811510021FFF7D9
:10E5B000E3FE002038BD00BF10B50C7814F06004F5
:10E5C00013D0202C0AD14B78023B092B18D8DFE856
:10E5D00003F01B21171717171717272E224901229F
:10E5E000FFF7DCFF0024204610BD4B78062B24D01B
:10E5F0000A2BF3D01D4B8A78C3F88828204610BD1B
:10E60000F9F7ECFF0224EEE719490122FFF7C6FFF4
:10E610000024E8E717490122FFF7C0FF0024E2E7E2
:10E620004B88124A1B0AC2F884380024DBE70F4BE0
:10E630008A78C3F880280024D5E74B881B0A222B50
:10E640000CD0212B04D021462246FFF7A7FFCAE7B2
:10E65000CA880949092A28BF0922F6E7CA88074952
:10E66000362A28BF3622F0E768670020E05E0020E7
:10E67000646700206067002042030020F802002049
:10E68000F8B50B7813F060050C46064611D0202D26
:10E6900016D1CD88D5B11B062AD52A461F496078E8
:10E6A000F9F71EFEE2881D493046FFF777FF002587
:10E6B0000AE04B780A2B16D00B2B0ED0062B03D179
:10E6C0003046F9F78BFF02252846F8BD0222607814
:10E6D0001144F9F705FE2846F8BD8B78DBB9104BDD
:10E6E000C3F88C58F0E70F490122FFF757FFEBE71B
:10E6F0000D4B4A780D4FC3F8D42003230021C0E905
:10E70000E45580F8113107F144022B463D640D4673
:10E71000FAF79EF8D8E7F9F761FFD5E73C2C00201F
:10E72000E05E00206C67002098010020F82B00209C
:10E730000B7803F00303012B03D0022B04D000203D
:10E7400070478B881BB937E78B88832BFBD097E703
:10E75000F0B5012190F8D17590F8D36590F8CFC548
:10E7600090F8CE5590F8D03590F8D22580F8111158
:10E7700090F8CC1585B005EB0C2503EB072302EBD5
:10E78000062201F01F06AFB292B290F8CD558DF877
:10E7900008109BB2012E0446ADF80A70ADF80C309B
:10E7A000ADF80E20C0F840218DF8095017D0022E88
:10E7B0001FD036B101F08001F9F7A6FE002005B0A8
:10E7C000F0BD092D0FD8DFE815F0BF00AC000E003A
:10E7D000D5000E00EA0085000E007700540090F886
:10E7E0001221032A2FD02046F9F7F8FE002005B0A9
:10E7F000F0BD01F060012029DAB234D0012D00F023
:10E800002081032D00F00681002DD7D190F8121140
:10E81000022900F0DF800329E5D11B0600F14B81BE
:10E8200002EB820200EBC20393F87633002B00F078
:10E830004D81BF4B0122C3F8A028BE4920460222C9
:10E84000FFF7ACFEBAE7DAB2012ACCD8D0F8E4354B
:10E8500002A99B689847BDF80E30002BAED1204628
:10E86000FFF74EFEAAE7D0F8E43502A99B68984767
:10E87000A4E7F9B2AE4D012985F89018B3D890F805
:10E880001231022B00F02781032BACD1002900F0BC
:10E89000868190F810110129E1D0D0F8E4355B6849
:10E8A000984795F8901884F810112046F9F7FEFD66
:10E8B0002046FFF725FE81E7012A94D190F8123116
:10E8C000022B00F01781032B8DD100F58871FFF723
:10E8D00065FE73E73D0A022DADF8062000F0508179
:10E8E000032D00F00B81012D7FF47DAFD0F8EC35C6
:10E8F00080781B680DF106019847BDF80620002AB4
:10E900003FF45CAFBDF80E30002B3FF457AF9A4296
:10E9100028BF1A4601462046ADF80620FFF73EFE06
:10E920004CE790F81231023B012B3FF65CAF012F10
:10E930007FF444AFD0F8E43500229B68C0F818217A
:10E9400002A9204698478AE790F81231023B012B32
:10E950003FF649AF764BD0F818210021C3F898183C
:10E9600012B10222C3F89828734920460222FFF709
:10E9700015FE23E7012F00F09880022F7FF41EAFD1
:10E9800013F0FF0F7FF41AAF02691B0A023B5268B3
:10E99000032B00F21D81DFE803F0393531241A43DF
:10E9A0007FF421AF90F81231032B3FF41CAF0369C1
:10E9B00007F07F0580F81451196867F30A120A43BB
:10E9C0001A60FFF79DFD002D00F0E580022384F81A
:10E9D0001231F3E651063FF4F1AE1146F9F794FD1A
:10E9E000ECE6052363F30612514B012184F816115E
:10E9F0002046C3F89C28FFF783FDDFE6042363F37A
:10EA00000612F1E7032363F30612EDE7022363F333
:10EA10000612E9E790F81231022BDBD0032B7FF4CA
:10EA2000E2AE27B9550602D01146F9F76DFDD4F8CC
:10EA3000E43502A99B68204698472046FFF760FD11
:10EA4000BCE690F812110229C4D003297FF4CBAEA2
:10EA5000002F7FF4B3AE12F07F013FF400AF180631
:10EA600000F1A78002EB820304EBC30304EB8100F7
:10EA700083F8767383F8741383F87573282303FB84
:10EA80000243416D03F55D73DA780B68023A6FF368
:10EA90005553012AD4F8E42598BF43F080530B6006
:10EAA0002046936802A99847D9E6D0F8E435C0F823
:10EAB00018719B6844E702F07F0202EB820200EBD0
:10EAC000C20393F81E31002B7FF4B3AE184B002223
:10EAD000C3F8A028B1E600293FF4C1AE0121032309
:10EAE00080F8101180F81231F9F7E0FC2046FFF7AA
:10EAF00007FD63E61149FFF751FD5FE6FDB2052D05
:10EB00003FF671AEDFE805F0342C241C0B03D0F87F
:10EB1000EC3580789B690DF106019847EDE6D0F859
:10EB2000EC3580785B690DF106019847E5E600BF9A
:10EB3000E05E002080670020786700207467002076
:10EB4000D0F8EC3580781B690DF106019847D4E6C2
:10EB5000D0F8EC358078DB680DF106019847CCE6FB
:10EB6000D0F8EC3580789B680DF106019847C4E633
:10EB7000D0F8EC3580785B680DF106019847BCE66B
:10EB8000D0F8E43580789B6A0DF10601984745700E
:10EB9000C4F8F005B1E6012384F812310EE6022232
:10EBA000D0F8E43580F8101180F812215B6898479E
:10EBB00055E6282202FB014304EB810083F81E7115
:10EBC00083F81C1183F81D51816903F58E735BE78F
:10EBD000012363F3061207E770B5044649B990F8BC
:10EBE0001131022B1BD094F81631012B0DD00020CF
:10EBF00070BDD0F8E4355B69002BF8D090F8122195
:10EC0000032AF4D19847002070BD2A4A2369D2F81C
:10EC10009C285A60002384F81631002070BDD0F87B
:10EC20003831D0F82451AB4217D9C278012AD0F834
:10EC30002821A3EB050308BF5219C0F8383108BFDB
:10EC4000C0F828219BB20021FFF796FB00231A464B
:10EC500019462046F9F7FCFDC5E7D0F83C31B3FB77
:10EC6000F5F605FB163666B99D420AD8D0F8402164
:10EC7000934206D233463246FFF77EFBC4F840612A
:10EC8000E4E7D4F8E435DB681BB194F81221032AD9
:10EC90000CD00023052284F8112119461A4620467B
:10ECA000F9F7D6FD2046F9F789FC9CE720469847FE
:10ECB000EFE700BFE05E0020214A038890429BB24C
:10ECC00012D002F5806290420ED0B0F1804F0BD08E
:10ECD000A2F58032904207D002F58062904203D0C4
:10ECE00002F58062904203D14A8823F070031343F7
:10ECF000144A904218D002F58062904214D030B489
:10ED000023F440730C894D6802F56C429BB2234397
:10ED100090420C880380C56204850DD18B7A0386EE
:10ED2000012330BC8382704703800B884A68C2622B
:10ED30000385012383827047034B9842EED0EFE7AF
:10ED400000000140001000400004014000B583B005
:10ED500009238DF80730F9F705FF8DF807009DF8B6
:10ED60000730012BF7D09DF8070003B05DF804FBD6
:10ED700082B0064B002201920193019B03EB8000BD
:10ED80000190019B186802B0704700BF50280040F6
:10ED900082B0064B002201920193019B03EB80009D
:10EDA0000190019B196002B0704700BF50280040DD
:10EDB0000023C0E90033C0E90233C0E90433C0E9ED
:10EDC0000633C0E90833C0E90A33C0E90C33836372
:10EDD000704700BF0B6870B4D1E90524CD682B43A0
:10EDE0001343D1E9072523431343D1E909422B43B8
:10EDF000D1E90D652343134304680B4A3343224092
:10EE00002B4313430360D1E90B3442690D6922F0AF
:10EE1000070223431343D1E9014243614560846003
:10EE200070BCC260704700BF3F801CF0026836496A
:10EE3000002310B422F00102212488420260036002
:10EE400043608360C3600361446138D02F4B9842B4
:10EE50002ED02F4B98423CD02E4B984240D02E4B78
:10EE6000984232D02D4B984241D02D4B984246D0FB
:10EE70002C4B984217D02C4B98423CD02B4B9842AD
:10EE800016D02B4B984224D02A4B984228D02A4B9C
:10EE900098421AD0294B984229D0294B98422ED01B
:10EEA000284B984208D14FF03D5243F8AC2C03E078
:10EEB0004FF4746243F8202C5DF8044B7047224BEA
:10EEC0005DF8044B3D229A607047204A43F8642C59
:10EED000F2E74FF474125DF8044B43F8382C704796
:10EEE0004FF074625DF8044B43F8502C7047184A99
:10EEF00043F87C2CE0E73D2243F8082CDCE7154A78
:10EF000043F8942CD8E700BF10600240286002400C
:10EF100040600240586002407060024088600240D9
:10EF2000A0600240B86002401064024028640240C1
:10EF300040640240586402407064024088640240A9
:10EF4000A0640240B8640240006002403D0000201E
:10EF5000400F002000003D202DE9F04FDFF8ACA36A
:10EF60002DED028B9AF8B818002297B0CAF8A8289D
:10EF7000CAF8AC28CAF8B028CAF8B428CAF8A42835
:10EF800019B19AF8B9288AF8A4289AF8BA281AB1B7
:10EF90009AF8BB288AF8B3289AF8BE281AB19AF8CA
:10EFA000BF288AF8AE289AF8BC281AB19AF8BD286A
:10EFB0008AF8A9289AF8C03805935A1ED3B257B2D6
:10EFC00003937B1C00F0AA80C54AC64E52F83790C6
:10EFD000029602EBC70200231279019308EE102A71
:10EFE0001D46344698462678394630463AF0ACF805
:10EFF00083463046BBF1000F1ED035F0B7F9EA1D4D
:10F000001321D2B220B14FF0000E827180F807E0D8
:10F0100031F0B8F820783AF0C1F84FF0070308F162
:10F02000010223714FF0010384F802806070CDF873
:10F0300004B05FFA82F8E3700135042D04F1050491
:10F04000D1D118EE100A029ECDF81080FBF750F9CE
:10F05000A549A64A4868024042F440324A600FB9C6
:10F06000019B5BB9A24C4820FBF742F920460221E4
:10F0700048F0D0FFA26842F00102A2609A489C4A80
:10F080004168BAF8C24841F400014160516821F476
:10F0900080515160916B21F4401141F480119163D2
:10F0A000D16841F46001D160956B85F44011C1F3E2
:10F0B000015101EB81011F2000FA01FC25EA0C0C33
:10F0C000112505FA01F141EA0C019163D16841F083
:10F0D000E061D160956BC5F30151C1F10401C9B282
:10F0E00001EB810188404FF0120C25EA00000CFA78
:10F0F00001F108439063E4B1BAF8C418CAF8CC48E7
:10F10000A1B1BAF8C628CAF8D01862B1019B7948F3
:10F11000521A90FBF2F2CAF8D4286BB917B0BDECC2
:10F12000028BBDE8F08F744A1288EFE7734A1188AA
:10F13000E7E7734A1488DFE74846049948F06AFF16
:10F14000684B012003F114080723F278441CE4B251
:10F1500052B375783279A5F10A0101EB410105EB53
:10F16000450C092D03FA01FE03FA0CFB02FA01F12A
:10F1700040F2A080D9F80C2022EA0E0E41EA0E01DE
:10F18000C9F80C10421E02EB82021F21062801FA68
:10F1900002FC05FA02F273D8D9F8341021EA0C0106
:10F1A0000A432046C9F834200536B045CDD1D9F8F8
:10F1B0000820039942F40072C9F80820D9F8082001
:10F1C00042F48072C9F80820D9F80820574442F068
:10F1D0000102C9F8082097F9C828022039F00EFA70
:10F1E000044600289AD04668304639F07DFA454AF0
:10F1F000431E242101FB032393F8D851002D8DD108
:10F20000059983F8D911062283F8D821002885D0E2
:10F21000304639F069FA46F079FD6068FFF706FE7E
:10F2200007A8FFF7C5FD049EA26837480792012E84
:10F230008CBF4FF4806300230D9309F14C034FF40E
:10F240008072CDE90A56089309904FF40033606844
:10F250000C9507A94FF400674FF40056CDE9102331
:10F26000CDE90E76FFF7B6FD6268136843F001033F
:10F270001360D9F8083043F08043C9F808304DE7EF
:10F28000C11FA0F10D0201EB81014FF01F0E02EB37
:10F2900082020C280EFA01FC0EFA02F005FA01F1C6
:10F2A00013D8D9F8302022EA0C0211432046C9F8BD
:10F2B000301079E7D9F8101002FA0CF221EA0B0BA2
:10F2C00042EA0B02C9F810205CE7D9F82C1005FAC5
:10F2D00002F221EA00010A432046C9F82C2063E724
:10F2E000D4B805088467002000230140E030FCFF0B
:10F2F00000200140803801002E7AFF1F2C7AFF1F6A
:10F300002A7AFF1F98010020B8670020E05E0020E5
:10F31000024A536A23EA00005062704700380240F4
:10F32000024A136A23EA0000106270470038024064
:10F33000484B98422ED0B0F1804F32D0464B984285
:10F3400036D0464B98421ED0454B984237D0454B5D
:10F3500098423BD0444B98423FD0444B98424BD0CC
:10F36000434B984240D0434B98424CD0424B98423A
:10F3700051D0424B984256D0414B98425AD0414BC3
:10F3800098425ED07047404A136A43F00403136208
:10F390000420C5E73C4A536A43F00103536201204D
:10F3A000B6E7394A136A43F0010313620120B7E755
:10F3B000354A136A43F0020313620220B0E7324A6F
:10F3C000136A43F0080313620820A9E72E4A136A60
:10F3D00043F0100313621020A2E72B4A136A43F094
:10F3E0002003136220209BE7274A536A43F48033AB
:10F3F00053624FF480308BE7234A536A43F0020391
:10F400005362022084E7204A536A43F40033536274
:10F410004FF400307CE71C4A536A43F48023536264
:10F420004FF4802074E7184A136A43F040031362D4
:10F43000402075E7144A136A43F08003136280206A
:10F440006EE7114A136A43F4807313624FF48070BD
:10F4500066E700BF000001400004004000080040D3
:10F46000000C004000100040001400400004014067
:10F4700000400140004401400048014000180040A5
:10F48000001C0040002000400038024010B5044637
:10F490000068FFF74DFF0D4BD3F8982A204652081D
:10F4A0004FF6FF7130F000FA20460021FCF72CFFE8
:10F4B0000749084A41F248132046CA5001F58A51CB
:10F4C000BDE810400022083130F0C2B8F82B00200F
:10F4D000E05E002015D4010838B5124BD3F8984AE5
:10F4E000054600686408FFF723FFB4FBF1F3B3F5AA
:10F4F000803F03D3012CFAD96408F6E7224699B27B
:10F50000284630F0D1F90849084A41F24413284608
:10F51000CA5001F58A51BDE838400022043130F06C
:10F5200097B800BFF82B0020E05E002095F5010899
:10F530002DE9F04FCCB2002185B0074608461646AB
:10F5400035F0F0F90021012035F0ECF934F0ECFE53
:10F55000022E09D0042E44F6C01818BF4FF4964866
:10F56000072C06D900200AE0FF2C4FF41648F7D1EB
:10F570000326C34D95F8543023B90020A86505B083
:10F58000BDE8F08F032E0FD0BE490C44002294F842
:10F590005B07032130F0FAFB0028EED0BA4BC3F82A
:10F5A0002409C3799A07E8D4B74C95F8540041F27E
:10F5B0003F130022E654032130F0E8FBC4F8280D85
:10F5C0000028DAD04FF48062B04BC4F8E038C4F8B9
:10F5D000EC280323C4F8F02841F23012A4F8E438F0
:10F5E0000023A35441F22C124FF0010924F8029099
:10F5F00041F2381204F62811A35041F23C12C4F82B
:10F60000F418A35241F23E1204F62C51032EA354D7
:10F61000C4F8E888C4F80C39C4F80039C4F8FC38D8
:10F62000C4F8F818C4F80839C4F8043904F50E6AA7
:10F630000ED0D4F824B99BF8040034F097FEC4F837
:10F64000200958460FF04CFF494650460FF05CFF2A
:10F65000322031F0E5FA012E09D1D4F8280D4146C7
:10F66000FFF73AFFD4F82409FFF710FF0AE0022E53
:10F670003AD1D4F824090FF022FFD4F8280D4146DE
:10F68000FFF72AFFC5F858A04FF0060A022E10D047
:10F69000A86D31F055FE60B10121002035F042F92E
:10F6A000A86D31F04DFE0146002840F0848035F011
:10F6B00039F9384631F044FE80B10121084635F071
:10F6C00031F94FF0050B4FF00008384631F038FEA5
:10F6D0000146002877D1012035F024F9042ED7D037
:10F6E000052031F09DFAD1E7032E5CD1DFF8A89117
:10F6F00067484FF0000B89F800B0594640224BF0A4
:10F70000E6FF8DF80FB0DFF87CB19DF80F30072BC6
:10F7100009D9604801210FF0F7FED4F8280D4146C1
:10F72000FFF7DAFEAEE79DF80F3003EB43030BEB78
:10F73000C30393F8F5377BB39DF80F3003EB430316
:10F740000BEBC303D3F8F83733B39DF80F305B44AA
:10F7500093F85B0700B30022032130F017FB019000
:10F76000D0B10FF0ACFE9DF80F3099F80010019A5F
:10F7700003EB43030BEBC30305EBC100D3F8F837EE
:10F78000C365D379DB0748BF012301F1010148BFFD
:10F7900080F8603089F800109DF80F300133DBB23B
:10F7A0008DF80F30B1E7042E7FF46CAFD4F8240944
:10F7B0000FF085FE51E7A86D31F0BAFD01463846DD
:10F7C00031F0C2FD6CE7384631F0B2FD95F8AA3051
:10F7D000014683B9242803D14FF0010385F8AA30EC
:10F7E000012E04D13846019131F0AEFD0199A86D8A
:10F7F00031F0AAFD69E7012B06D14D280CBF022389
:10F80000002385F8AA30EBE7022B06D13C280CBF79
:10F810000323002385F8AA30E2E7032B10D10A283E
:10F8200002D985F8AA80DBE7042385F89D0085F8D6
:10F830009C8085F89F8085F89E0085F8AA30CFE7E8
:10F84000042B09D195F89E3085F8AB00434085F82C
:10F850009E3085F8AAB0C3E7052BC1D195F89C303E
:10F8600095F89D9095F89E004B4517D25A1C2B4455
:10F87000484085F89E0085F89C2083F8A010AFE7EB
:10F88000D86F0020F82B0020E05E0020DCB80508CF
:10F8900034700020C0670020207000208842C0D152
:10F8A00095F8AB3085F8AAA0F42B99D1B9F1000FE7
:10F8B00096D12421384685F8AA9031F045FD4D2196
:10F8C000384631F041FD3E21384631F03DFD494694
:10F8D000384631F039FDF421384631F035FDF42158
:10F8E000384631F031FD032E1BD0D4F8240943797A
:10F8F00001689D080223AB40DB439BB20B828D89DC
:10F900002B408B81007920210FF0C8FDD4F8240909
:10F910004A4649462FF09CFED4F824391868FFF770
:10F9200007FD0022D4F8280D11462FF091FED4F8DF
:10F93000283D1868FFF7FCFC012020E6224A936866
:10F9400003F00C03042B10B421D0082B22D01F4B42
:10F9500003601D4C1E4AA168C1F30311114491F8C4
:10F96000FC13CB404360A168C1F38221114491F89C
:10F97000FC1323FA01F18160A1685DF8044BC1F327
:10F9800042310A4492F8FC23D340C3607047114BC4
:10F990000360DEE75468516852686302C2F388125C
:10F9A0004CBF0C4B094B01F03F01B3FBF1F303FBE0
:10F9B00002F3054A5268C2F3014201325200B3FB1E
:10F9C000F2F30360C5E700BF003802400024F400F2
:10F9D0009801002000127A002DE9F04FB34CD4F8C2
:10F9E00004375A69D2078BB002D50BB0BDE8F08F4F
:10F9F0005A699B6912EA030AF7D0CAF307431AF45B
:10FA0000002F009340F00281009B5D0743D41AF061
:10FA1000020F5FFA8AF503D0D4F8043702225A6144
:10FA2000BAF1000FC0F211821AF4006FCAF307276F
:10FA300040F084812E0708D59D4B9E48D3F818349A
:10FA40009847D4F8043708225A61ED0600F1E9819D
:10FA5000F80600F1A981B90600F12E81009BDA06B3
:10FA600009D5934B9348D3F828349847D4F80437F2
:10FA70004FF480125A61009B9B06B6D58C4B8D4883
:10FA8000D3F82C349847D4F804374FF400125A6155
:10FA90000BB0BDE8F08FD4F808279369D269134002
:10FAA0001FFA83FBBBF1000FB1D0DFF80882CDF85D
:10FAB0000CA045464FF0000909E05FEA5B0B09F135
:10FAC000010908F1040805F1280500F0DA811BF0AE
:10FAD000010FF2D0D4F808175FFA89F708694A6B6A
:10FAE00004EB8703FA40D3F81037D2019B68D2B2F7
:10FAF00002431A40D007D3B216D54B6BD8F8182062
:10FB0000012000FA09F023EA00034B63684B6948BF
:10FB1000D3F81034012191603946984794F8FB6678
:10FB2000012E00F0FC8101231A0703D5D8F8182014
:10FB300008239360DE0603D5D8F8182010239360BD
:10FB4000580603D5D8F8182040239360990703D5A9
:10FB5000D8F81820022393601A06AED5D5E94C6078
:10FB6000D5F82431D8F818C0311A8B42DCF81820A7
:10FB700028BF0B46033392B2B2EB930F9DD9D4F852
:10FB80000827323704EB8703CDE901989046994660
:10FB9000B04238D2BEB3D5F8241194F8FB36D5F86C
:10FBA0002821371AB94228BF394601F1030E4FEA1E
:10FBB0009E0E83B98FB20337BF10D9F800A70AD0C1
:10FBC000013352F8040BCAF800009F42F8D1D5E97E
:10FBD0004C60D5F82821DCF8183008440A44B042BB
:10FBE000C5F82821C5F834010AD195F81C11D8F8B8
:10FBF0003420012707FA01F122EA0102C8F8342073
:10FC00009BB29E45C4D3DDE9019856E7D4F8083786
:10FC10009D69DB691D402D0C3FF4F6AE04F5DF66EF
:10FC2000DFF88CB0B046B146002708E06D0807F158
:10FC3000010706F1040608F128083FF4E5AEEB07DA
:10FC4000F4D5F9B204EB8102D4F80837D2F84C2786
:10FC500092685B691A40D007D3B218D594F8FB06B6
:10FC6000726D01239842936007D11269D8F87C33F2
:10FC7000C2F312029B1AC8F88C33DBF80C344846E6
:10FC8000984794F8FB36012B00F0578101239A071F
:10FC900002D5726D022393601B07C7D5DBF81434BD
:10FCA00048469847736D08229A60BFE7E84D0020E8
:10FCB00098010020E0540020D4F80837D4F8101739
:10FCC0009A680868C2F34102022A08BF03224FF073
:10FCD000000514BF65F30A0062F30A0008605A6861
:10FCE00042F480725A6006A8FFF728FED4F8042771
:10FCF000D4F80807D368BF49079D6FF38D23D360FD
:10FD00008068C0F34100014491F89C11032900F080
:10FD1000CF80B949B9480126294484F8FA6681425E
:10FD20004FF04006A4F8FC6600F215810E2161F345
:10FD30008D234FF40051D36051618FE6B04B94F89E
:10FD40000A28D3F82034AF4800218DF817108DF819
:10FD500017209847D4F80817D4F8042794F80237E6
:10FD600088684FF400615161002B3FF463AEC30714
:10FD70007FF560AE94F80D38012B7FF45BAE9DF8F3
:10FD80001730032B7FF456AED4F804389E491A6816
:10FD900042F001021A601A6842F003021A600B690D
:10FDA00043F006030B6145E6D4F8082795485368ED
:10FDB0004FF0000823F0010341465360F8F7B4FE0A
:10FDC00094F8F966414656B1904BFF2203EB860644
:10FDD00053F8045FD86BAA609E428260F8D1D4F8D1
:10FDE000083788484FF0FF329A614FF00112DA610C
:10FDF0000B2262F3070162F30708C3F8148019614C
:10FE00001A686FF30A121A60F8F7D8FBD4F80427BF
:10FE10007B4B7C48D3F81C344FF480515161984798
:10FE200019E6D4F804379A6922F010029A611A6A26
:10FE3000C2F34340022802F00F0144D0062823D029
:10FE40009A6942F010029A6102E694F802373BB1D7
:10FE5000D4F80428136823F0030161F30703136047
:10FE6000D4F8082766495368D1F82414654823F06C
:10FE7000010353608847D4F804374FF000425A61B9
:10FE8000D2E5DDF80CA0C2E501EB8101D4F8C8573A
:10FE900004EBC1012E68D1F8840AC4F8C46CC2F323
:10FEA0000A1202442868C4F8C80CC1F8842AC7E7BB
:10FEB00000214FF4007084F8FA160921A4F8FC061A
:10FEC00061F38D2335E747F6F0701042B8D001EBAF
:10FED0008100C2F30A1204EBC00002F1030C5FEAD6
:10FEE000AC0CD0F8785AD4F8C8E74FEA810818BFAC
:10FEF000002006D00130DEF8006045F8046B844530
:10FF0000F8D1414404EBC101D1F8785AD1F8840A00
:10FF100015440244C1F8785AC1F8842A90E7B9F12F
:10FF2000000F7FF400AE94F80938042B7FF4FBAD8A
:10FF30003448F8F743FB3346F6E5002F7FF4A6AECE
:10FF400094F80928052A7FF4A1AE48460193F8F7F2
:10FF500035FB019B9BE62E48A5F57401A1F51051D8
:10FF6000814203D80D2161F38D23E2E629492A4815
:10FF70002944814203D20C2161F38D23D9E627481D
:10FF8000A5F18C71A1F54341814203D80B2161F3A6
:10FF90008D23CEE6224923482944814203D20A21F7
:10FFA00061F38D23C5E6204920482944814203D2CC
:10FFB000092161F38D23BCE61D48A5F1B771A1F5B8
:10FFC0005851814203D2082161F38D23B1E61949CA
:10FFD00019482944814203D2072161F38D23A8E601
:10FFE000164917482944814234BF0621052161F38F
:10FFF0008D239EE670B70508401E1BFF3F420F0091
:020000040801F1
:1000000098010020E054002000ED00E0F4540020AE
:10001000DFC810002013FBFE20D61300FF69180074
:1000200000D3CEFE40771B00C05BB3FEC091210021
:1000300040AC2700C01D6AFE40E13300803C36FE24
:10004000E09C41000D4B93F8E22A12F0010F0C4A9C
:1000500003D0012382F8AC30704792F8AC2062B92B
:10006000D3F82C2B4AB193F8D82A104493F8D92A04
:1000700083F8D80A114483F8D91A7047F82B002066
:10008000D86F002010B50E4C40F0080284F83C24D4
:1000900094F9DA20022A06DD420704D583071CBF43
:1000A000012384F8E23005210648F8F777FE06219F
:1000B00084F83D04BDE810400248F8F757BE00BF81
:1000C00098010020D005002010B5F8F7FFFDA8B377
:1000D0001B4C94F9DA30012B30DD59B3022B2DD0B3
:1000E00094F8E2309BB971B180230521154884F85A
:1000F0004234F8F753FE062184F84304BDE810406B
:100100001048F8F733BEBDE810400420BAE70029D4
:1001100014BF0020042094F8DD301A0748BF40F0D7
:1001200002005B0701D411B108B940F00100BDE83D
:100130001040A7E7022BD3D10420ECE710BD00BF8D
:1001400098010020D6050020F8B5224C04F244475F
:10015000030A84F8490405460621384684F84834E1
:10016000F8F71CFE94F8DD3084F84A04DB072AD443
:10017000B4F8DE20AA4226D1174DD4F84434C5F88D
:10018000AD30C3B285F8B33041F26F714FF6FF73F3
:100190008A4218BF0123134405F1AD06C3F30722B9
:1001A0000621304685F8B12085F8B230F8F7F6FD23
:1001B000072185F8B3003046F8F7D8FD052104F291
:1001C0004B40F8F7D3FDBDE8F84004480721F8F7A5
:1001D000CDBD00BF98010020D86F0020DC050020B5
:1001E00008B5F8F773FD48B1A1F59C53083BB3F58A
:1001F0007A7F03D2BDE808400846A5E708BD2DE98F
:10020000F047C44DD5F89C3A002B3BD0C24EC34CAE
:1002100006F1DA07D5F89C0A31F092F8A0BBB5F8E0
:10022000C02A092A0CD9B5F8C21A64234B43B3FB80
:10023000F2F3452B40F3AC81A5F8C00AA5F8C20A39
:1002400094F8ED30012B00F0D181022B00F0EC810D
:1002500033B9B3480521F8F789FD012384F8ED305F
:1002600095F8CE3A2E6B002B00F0E881D5F8D03A05
:10027000F31A782B40F2E281D5F8D40AF9F776F92F
:10028000C4F8F060BDE8F087D5F89C0A31F050F86A
:1002900094F8B4308046052BBCD8DFE803F003099E
:1002A000181E3947AA28B5D1012384F8B430B1E724
:1002B000552803D1022384F8B430ABE7B5F8C43A2B
:1002C0000133A5F8C43A002384F8B430A2E703232D
:1002D00084F8B50084F8B4309CE7132884F8B6009D
:1002E000C4F8D00008DDB5F8C63A0133A5F8C63A1F
:1002F000002384F8B4308DE718B9052384F8B430AE
:1003000088E70023C4F8D430042384F8B43081E7AC
:10031000D4F8D430E218013382F8B700D4F8D020F2
:10032000C4F8D43093427FF475AFE6E7D4F8D03008
:100330007C4803F1020A4FFA8AF1F8F72FFD804555
:1003400094F8B59040F01A8126201EF099FB58B120
:10035000002385F8CE3AB5F8C23A0133A5F8C23A7F
:10036000002384F8B43055E795F8CE3A4B451AD1BE
:10037000002385F8CE3A09F1FF33102B00F2F88004
:10038000DFE813F01F007F007F00E0007F00F60031
:10039000F600F6001F00F600F600F600F600F60084
:1003A000F600F6001F00B9F1090F02D0B9F1110FE4
:1003B00001D1012BDCD0B5F8CA3A0133A5F8CA3A0D
:1003C000D9E7BAF1060F5CDDB9F1010F06D0B9F13A
:1003D000090F0CBF4FF002094FF0030994F8BA005F
:1003E00094F8BB1094F8B92094F9B7E094F9B9C027
:1003F00094F8B83086F8DA9041EA002109B2900703
:1004000086F8DBE086F8DDC0A6F8DE1006D512F02F
:100410000C0F14BF0122002286F8E220B9F1030F6D
:1004200013D1BAF1090F2CDD94F9BD20082AA8BF19
:10043000082222EAE27286F81021002043B29A4292
:1004400000F101005EDC94F8BC30D5F8A8A00020D3
:1004500002469BB2524590466ADB95F8C83686F84C
:10046000DC00232B0DD109EB890303EB83030CEB99
:100470008303A5F8CC36A5F8CEE6A5F8D016A5F8E6
:10048000D206294929480A224BF0F9F810B1002375
:1004900084F8E230244B3A681A607A685A603A89E4
:1004A0001A8194F8E23043BB96F8E23095F8D82AE6
:1004B00084F8E420002B14BF0223012384F8E230E7
:1004C00096F8DD3095F8DA0A84F8E80013F00103B5
:1004D0001CBFB2FA82F35B0995F8D92A84F8E520AB
:1004E000D9B2B5F8DC2A84F8E310A4F8E62013B1F9
:1004F0000AB1A4F8EA2084F8EC100FF0BBFB0FF06F
:10050000B9FB28E705EB4308234493F8BF30A8F86C
:10051000323B93E7F82B002098010020D86F002091
:10052000E30500208D700020B070002072020020D2
:1005300005EB48080132B8F8AC8052B2984508BFC4
:10054000104687E7BAF1040F9BDD94F8B72094F8C2
:10055000B83043EA022359041AB204D5C3F30D0399
:10056000A6F8E0308DE7002AF8DBA6F8DE3088E751
:10057000B5F8CC3A0133A5F8CC3AECE619F0010F06
:100580007FF4EEAEB5F8C83A0133A5F8C83AE7E60D
:100590003A4BD3F85024B3F85414012A1DD141F238
:1005A0005632914203D14FF0FF32C3F85024D3F8B2
:1005B0005024D5F89C0A02EB820202EB820201EB86
:1005C000420189B2A3F8541403681B6998470023B9
:1005D000A5F8C03AA5F8C23A32E60132E7D1B1F542
:1005E000965F04BF0122C3F85024E0E7234E96F93A
:1005F000DA70002F3FF434AE022F11D14FF4804057
:10060000FFF7A2FD84F8ED7096F9DA30012B7FF741
:1006100027AE96F8DD30C3F3400386F8E2301FE6DC
:10062000032384F8ED30EFE7144BB3F8E030002BF0
:100630003FF416AE032384F8ED3011E695F8C020A0
:1006400095F8C1309A4204D0F8F7BEFFC4F8F060C4
:1006500018E6D4F8F030F31AB3F57A7FBFF412AE8F
:10066000D5F8D03AF61A952E7FF60CAE044805213F
:10067000F8F77CFBBDE8F047F8F7A6BF980100202B
:10068000E305002010B5134CD4F82C0B00B394F8FC
:10069000D81A59B194F8D92A0EF050FCB4F8DC3AC3
:1006A00083421ABFA4F8DC0A01210021B4F8DE2A33
:1006B00062B141F288339342B8BF13469A4205D0E3
:1006C000A4F8DE3ABDE8104043F09EBE0029F9D1FF
:1006D00010BD00BFF82B002010B4014404460020D8
:1006E00014F8013B08225840430010F0800F08BF67
:1006F000400083F0070314BFD8B2C0B2013AF3D16F
:100700008C42EDD15DF8044B704700BF10B54FF43B
:10071000806084B02AF092FA50B3164B90F904002E
:1007200093F8F430144A002B18BF08234FF4E1313A
:100730000124CDE90143009100234FF480612AF0A8
:10074000DAFA0E4BFF22C3F84802003818BF012026
:1007500083F8D42683F8E42683F8F42683F8042764
:1007600083F8142783F8242783F8342783F8442751
:1007700004B010BDD86F002045900008F82B002071
:100780002DE9F04F384CD4F8D43B13F0006383B01C
:100790005CD094F8FCC060455CD3FF2856D1334B45
:1007A00093F8EA30002B4DD0DFF8C8B00022CBE937
:1007B0003E22CBF80021BCF1000F52D004F2D46EDF
:1007C0000EEB0C139A461046154611461646174670
:1007D000CDF804C07346B3F802E0B3F80CC093F848
:1007E000009093F90180714462444F45D3E901ECD4
:1007F00038BF4F4610334645B8BF46469A4509B202
:1008000012B275446044E6D1CBE93F508BF8F870E2
:100810008BF8F960DDF804C091FBFCF192FBFCF26F
:1008200094F8C836ABF80421092B104A08BF9BF88E
:10083000F830ABF8FA104FF0000182F8EA1008BF68
:10084000A4F8D2360A4803B0BDE8F08F002003B008
:10085000BDE8F08F04F2D46404EB001003B0BDE8EF
:10086000F08F62466146DBE7F82B002098010020FC
:10087000D0700020D86F00202DE9F8434B4C42780F
:1008800094F8083102F00F05CBB9F5B92B460021D9
:1008900084F80C11EB1AD9B20E290CD844490B4438
:1008A00093F8781B39B102F0F002802A4AD0902ADE
:1008B0005FD0A02A0DD000273846BDE8F88300217C
:1008C000AB4284F80C11F6D8E4E784F808512B46C3
:1008D000DDE7412966D081F08003042B62D9084608
:1008E000F8F7CAFB031D0246DBB2324884F80C312C
:1008F00065F05F0584F80D51F9F734FB94F80C713D
:10090000002FD8D0BE1E16F0FF0024D1FF25A94627
:10091000022756B1DFF8A080464418F8011BD4F82E
:10092000300130F011FD4645F7D1D4F83001494689
:1009300030F00AFDD4F83001294630F005FD384684
:10094000BDE8F88365F07F050427022684F80D5181
:1009500084F80C713046184A4FF6FF71104412F8B3
:10096000015B491B904289B2F9D15FFA81F90D0A06
:10097000CFE7412914D081F08003042B10D9084619
:10098000F8F77AFB65F06F050627042684F80F0157
:1009900084F80D5184F80E1184F80C713046DAE7B2
:1009A0000420EFE7082304229FE700BFD86F002050
:1009B000F82B0020E6700020E47000202DE9F04FB5
:1009C000C31D83B0DFF838A1DFF8388103F4FC736E
:1009D00000AFDAF89067ADEB030DC7F800D03268CE
:1009E000DAF8883768449A420C4678606D465AD0E7
:1009F00098F834310DF10102591C03F00F0388F807
:100A000034118DF800303A60A0EB0209D6E90012EB
:100A10005FFA89F9521A09F107035FFA82FB03F4BE
:100A2000FC73CB45ADEB030D57D25A4668464AF0EE
:100A3000EDFD33685B4433605A466946384642F000
:100A40006DFEDAF89027DAF888373068117A70602E
:100A5000C21A4A40D2B28342336088F8352109D0A5
:100A60000133336013F8011C984282EA0102F7D186
:100A700088F835213B68591C39601A70D7E9003273
:100A8000D21A012A08DD00215A1C3A601970D7E9F0
:100A90000032D21A012AF7DC2846A04700200C3782
:100AA000BD46BDE8F08F98F83431B6F90C20591CDA
:100AB00003F00F0343F01003002A2A46B8BF43F0A7
:100AC000200302F8023B88F83411691C3960D6E92A
:100AD00000135B1A3A606B7096E74A4668464AF024
:100AE00095FD33684B4433604A466946384642F0C8
:100AF00015FE2846A04701200C37BD46BDE8F08F03
:100B0000F82B0020D86F00200F4B104AD3F8D812D2
:100B100030B4C3F8DC12013103F59C7003F5DC75C9
:100B200003F53274C3F8D81203F5E471C2F88C5798
:100B3000C2F89047C3E96E0030BCC3E9B211C2F8F5
:100B40008407C2F888177047D86F0020F82B002060
:100B50002DE9F04F784DDFF8E49185B0D5F8904756
:100B6000D4E900431B1B002B00AF04460E46904601
:100B700028DD002389F8E032FFF7C6FF0020A31923
:100B800004F1010BC5F88037C5F87CB72278D5F899
:100B90008C675109012940F0958002F00F0A12F08C
:100BA000100214D150B199F8E212013101F00F0195
:100BB000514500F0908089F8E02210461437BD4678
:100BC000BDE8F08F99F8E0020028D8D1D4E7A31C43
:100BD000C5F87C37E21C6378D5F88407C5F87C2714
:100BE000A4783060C218726063404FF0000C89F83E
:100BF000E132D5F87CB7D5F8803789F8E012348136
:100C0000A6F80CC0A3EB0B03DCB2121AE31DD2B2A0
:100C100003F4FC73A242ADEB030D69D2594668465A
:100C20007A604AF0F3FC7A6830460BEB02036946BF
:100C3000C5F87C3742F072FDD5F88437306899F8F2
:100C4000E1228342C6E9003009D00133336013F852
:100C5000011C984282EA0102F7D189F8E122D5F815
:100C60007C371B78934239D1B6F90830FA2B54D02F
:100C70003268D5F88437D9F8DC02D5F88C17C6E984
:100C80000032D5F89027D5F88837536000241481B6
:100C9000948107F10C0389F8E042FC602AF01AFC09
:100CA000013041D0FB680BB100209847D5F8903750
:100CB000D5F88827196801201437C3E90021BD46FB
:100CC000BDE8F08F00210846F8F70AFA0120143732
:100CD000BD46BDE8F08FD6E9000293E7002301206E
:100CE000B6F9081089F8E032F8F7FAF9012065E75B
:100CF0002246594668464AF089FC0BEB040330460D
:100D000022466946C5F87C3742F008FD00201437BA
:100D100089F8E2A2BD46BDE8F08FB8F1000FA7D078
:100D2000052388F80030A3E7D5F89027136802213F
:100D3000581C10601970B5E7F82B0020D86F002000
:100D40000B4B93F8B62B12B1B3F8882B4AB9B3F911
:100D5000383C084AD81782FB0323C0EBA30000B23B
:100D60007047D3F8D00B90FBF2F000B2704700BF91
:100D7000F82B002067666666F8B5184CC6B20546C3
:100D80003146D4F8E40230F0DFFA94F8E812D4F8EF
:100D9000E402C5F307274E40394684F8E86230F094
:100DA000D3FA94F8E812D4F8E402C5F307464F40AA
:100DB000314684F8E87230F0C7FA94F8E812D4F8B3
:100DC000E4022D0E4E40294684F8E86230F0BCFA69
:100DD00094F8E8124D4084F8E852F8BDD86F00202E
:100DE00070B50C4DC6B231460446D5F8E40230F079
:100DF000ABFA95F8E812D5F8E402240A4E402146F1
:100E000085F8E86230F0A0FA95F8E8124C4085F8D1
:100E1000E84270BDD86F002038B50B4C0023054662
:100E20002421D4F8E40284F8E83230F08DFAD4F8C2
:100E3000E402542130F088FAD4F8E4022946BDE8EF
:100E4000384030F081BA00BFD86F00202DE9F04360
:100E5000DFF860932DED028B99F8E94283B00E46DE
:100E60001546002C00F04482013C89F8E9429FEDD0
:100E7000CD8ACD4FDFF840833378002B62D099F8CC
:100E8000E942002C5ED135B12FF04CFE2B68C01A20
:100E9000002880F2F68399F8EA12002940F099833D
:100EA00099F8EB02062840F2E181C04A92F85D34DD
:100EB00092F85C449C4200F00A82D2F8581499F8E7
:100EC000ECC231F8134064440130013302F58B6207
:100ED000A4B2C0B2DBB2B4F5E06F89F8EB02537193
:100EE00000F0DB8100F2AC80B4F5806F00F0048389
:100EF00066D9B4F5A06F00F0CE823DD9B4F5A16FEC
:100F000025D8601EC0B2FFF73BFCC8B1B0F90C3069
:100F1000A74AADF8014092F87617D9F8F02203EB12
:100F2000830303EB830349089B0093FBF1F3102138
:100F3000CDF803308DF800106846904700233370D9
:100F4000002D99D103B0BDEC028BBDE8F083B4F560
:100F5000C06FF5D1964BB3F8B82B002A00F046834A
:100F600023F0A4FF10220024CDF8030006238DF8FF
:100F700000208DF8014025E2B4F5826F00F05A821E
:100F8000B4F5846F40F03A81894B93F84C2B91076C
:100F9000D6D5B3F8683BCDF80330102120220423C6
:100FA0008DF800108DF801208DF80230D9F8F0325C
:100FB0006846002498473470002D7FF45DAFC1E788
:100FC000B4F5067FBCD8B4F5007FC0F03081A4F53D
:100FD0000073182BB4D801A252F823F06113010852
:100FE0004F1301084F1301084F1301084F13010855
:100FF0004F1301084F1301084F1301084F13010845
:10100000410F0108410F0108410F0108410F01087C
:10101000410F0108410F0108410F01083513010874
:101020001F1301081F1301081F1301081F130108D4
:101030001F1301081F1301081F1301081F130108C4
:10104000B4F5116F00F0E3815DD8B4F5026F00F0E4
:10105000C48122D9B4F5036F00F07D82B4F5046F2A
:101060007FF46EAF524BD9F8F022B3F9383C03EB62
:1010700083035B001020CDF80330402108238DF856
:1010800000008DF801108DF802306846002490476A
:101090003470002D7FF4F0AE54E7B4F5E46F00F047
:1010A0007C81B4F5006F40F08980414A92F84C1B76
:1010B0008C077FF545AFD80740F1F682D2F8542B64
:1010C00082EAE273A3EBE27303EB5303A7FB031380
:1010D000DB08002AACBF43F0004343F0404310213B
:1010E00000240822CDF803308DF800108DF801405F
:1010F000D9F8F0328DF80220684698473470002DF8
:101100007FF4BAAE1EE745F230239C4200F0B9816D
:1011100021D945F240239C4200F0338245F250230E
:101120009C427FF40DAF224AD9F8F032D2F8D02B8E
:10113000CDF80320502110228DF8002052228DF886
:1011400001108DF802206846002498473470002D65
:101150007FF492AEF6E6B4F5376F00F01C826FF4C0
:10116000376C04EB0C03072B3FF6EAAEA4F17100D9
:10117000C0B2FFF705FB00283FF4E2AE90F9013062
:10118000CDF8033010238DF80030ADF80140D9F8C8
:10119000F0326846984700233370002D7FF46CAE20
:1011A000D0E600BF0000C8421F85EB519801002027
:1011B000F82B0020D86F0020C5B3A291B4F5E26FE0
:1011C0007FF4BEAEC74B93ED130AD3ED007A20EE49
:1011D000270A002420EE080A48F072FD1023072297
:1011E000CDF803008DF800308DF801308DF8022025
:1011F000D9F8F03268469847347080E740F20143EE
:101200009C427FF49DAEB9F90C33CDF80330102128
:10121000012204238DF802308DF80010D9F8F03245
:101220008DF801206846002498473470C4E6B4F570
:10123000807F00F01A81B4F5887F7FF481AEAA4BDD
:10124000D9F8F022B3F93A3CCDF80330012110234C
:101250008DF800308DF801308DF8021068460024BA
:1012600090473470002D7FF407AE6BE601309F4A43
:10127000C0B292F8651492F864348B4222D04B1CB1
:10128000DBB24900D2F86044994A645A89F8EB020B
:10129000B4F5E06F53717FF425AE924B93ED120AD3
:1012A000D3ED007A20EE270A002420EE080A48F049
:1012B00007FD10220723CDF803008DF800208DF8DC
:1012C00001407FE0002182F865140123DAE78648B7
:1012D00099F8EC3290F8FC0082F85D140133DBB22F
:1012E0000130834289F8EC3200F06F810120C0E7C1
:1012F00000283FF4BCAD0378303B012B3FF6B7AD7F
:10130000013009F2E9220621FFF722FC99F8E932BF
:1013100089F8EA02002B3FF4AAAD3470A7E5A4F1E6
:101320001100C0B2FFF72CFA00283FF409AEB0F963
:10133000023025E76C4B93F8772B002A40F0988118
:10134000B3F8900BCDF803001023022265E0601E75
:10135000C0B2FFF715FA00283FF4F2AD43680FE77B
:10136000614B6449D3F8C83BD9F8F02281FB0301F3
:10137000DB17C3EBA10300241021CDF803300223B7
:101380008DF800108DF801408DF8023068469047C6
:101390003470002D7FF470ADD4E5524B93ED140AF8
:1013A000D3ED007A20EE270A002420EE080A48F048
:1013B00087FC102320228DF80030CDF8030007238E
:1013C0008DF801208DF802306846D9F8F032984740
:1013D0003470002D7FF450ADB4E5434B93F84C2BA3
:1013E00092077FF5ADADD3F8583BCDF8033010210F
:1013F000202208238DF802308DF80010D9F8F03241
:101400008DF801206846002498473470D4E523F015
:101410003FFD10230922CDF803008DF800308DF830
:1014200001308DF80220D9F8F03268460024984740
:101430003470C1E52C4AD2F83C3C13F0200440F053
:10144000D880D2F8D43B190640F121811023042220
:101450008DF803408DF804408DF805408DF8064066
:101460008DF800308DF8013042E6D9F8F432CDF82D
:1014700003301022002401238DF800208DF8014054
:10148000A0E7194AD9F8F032B2F9362CCDF803208A
:101490003021102250E6FF20FFF772F900283FF4B8
:1014A0004FADB0F90C301049D9F8F02291F8761709
:1014B00003EB830303EB83031020490800249B0004
:1014C00093FBF1F305218DF80000CDF803308DF882
:1014D00001408DF80210684690473470002D7FF46B
:1014E000CBAC2FE5D4370020F82B0020980100204A
:1014F000F80500206766666699F8F8320133DAB2BB
:10150000042A00F0B88042F2107389F8F82203FB35
:1015100002F3D9F8FC22002A00F0A88002338B4A9B
:1015200092F8E21AB2F8D82BC80748BF0433D107A3
:1015300048BF0A33940748BF1433D00548BF283347
:10154000510748BF6433520648BF03F57A63102140
:1015500000240422C6E57D4B93F84C2B92077FF5BF
:10156000EFACB3F85E1BD9F8F0224FF4F36303FB42
:1015700001F3A7FB03135B091020CDF803303021E2
:101580007CE5724AD9F8F032B2F9342CCDF8032058
:1015900040211022D0E5FF20FFF7F2F800283FF4A9
:1015A000CFAC90F90130CDF80330102170220B231D
:1015B0008DF802308DF80010D9F8F0328DF8012046
:1015C0006846002498473470F6E489F8EC1201204C
:1015D0004FE65F490620FFF7F1F9002389F8EA0298
:1015E000337003B0BDEC028BBDE8F083D3F8D00BB1
:1015F000B8E4B2F8623B92F84C1B643BC3EB437017
:10160000C3EBC00388FB03401844DB17C3EB202364
:101610000933092BA8BF092323EAE37303EB8303F0
:1016200011F0020F03EB830314BF4FF47A70002014
:101630009B00CC0748BF00F5FA6092F8641BD9F80C
:10164000F0229BB203440B44042010218DF80200C9
:10165000CDF803308DF800108DF801106846002495
:1016600090473470002D7FF407AC6BE4013356E7EC
:1016700023F00EFC66E6012389F8F83242F210737B
:1016800047E7347003B0BDEC028BBDE8F08392F8FD
:10169000763B002B3FF454AC99F80033032B4FD822
:1016A000DFE803F0443A2B12D2F8502B82EAE273BF
:1016B000A3EBE27303EB5303A7FB0313DB08002A3E
:1016C000B8BF43F080430AE5D9F80823537A907AEB
:1016D000D17A03F1407303EB0023002203EB0143B3
:1016E00089F8002310220421CDF803308DF8002062
:1016F0008DF801208DF8021058E4D9F804138A7D82
:10170000087C897A120402EB00220A44591C89F8E9
:10171000001302EB0363E5E7D9F804134A7DC87BA5
:10172000497A120402EB00220A44EFE7D9F80413C5
:101730000A7D887B097A120402EB00220A44E5E75D
:101740005A1C89F800231B06CCE700BFF82B0020A9
:10175000891C01082DE9F04782B0054602AF184602
:101760001C460E46904646F07BFD083020F00700F0
:10177000ADEB000D0DF1080A013CD14614F8013F14
:101780005BB989F800304246CDF800A031462846C2
:1017900036F0E8FFBD46BDE8F087184642F028FA6B
:1017A000C3B2A3F120023F2A88BF202309F8013BDE
:1017B000E4E700BF10B5114C94F8023723B9104B81
:1017C0004FF480225A6110BD0E4A136823F00603BD
:1017D000136046F011FD94F80237002BEFD0D4F8D7
:1017E00008379B68DB07EAD5D4F80428136823F090
:1017F000030161F307031360E1E700BFE84D002038
:10180000003C014010ED00E008B501210320FDF788
:10181000BFFA72B644F00AF82DE9F04F8DB0D04C03
:10182000DFF85493CF4D00904FF0000854F80B0CA4
:10183000002800F0FF802FF083FD0646002800F00E
:10184000DF81D9F8303044F8073CE0260023C64F4A
:1018500004F8033CA4F10B0B06FB08F654F80B0C40
:101860002FF06EFD002800F0E58054F80B0C2FF0EF
:101870005FFD14F8023C5A1E82460B2A0DD8DFE8A1
:1018800012F020003B004700540084009C00E4005C
:101890001801380143017D01950124280DD0009ADB
:1018A00042B9B24A92F86624824240F08581012210
:1018B00004F8032C0D2BD1D186E0012304F8023C5F
:1018C000CCE700234D28C4F8C53084F8CD3084F827
:1018D000CE3004D0582808D004F8023CBEE70222DB
:1018E00004F8022C84F8C430B8E7032304F8023C5F
:1018F000022384F8C430B1E704233C2804F8023CF6
:101900000BD0BAF13E0F0CD0002304F8023CA5E73F
:101910000A233C2804F8023CF3D1002304F8013CDC
:101920009CE7012304F8013C98E7D4F8C500BB19F3
:101930000344421CC4F8C52083F8CFA194F8CD001D
:10194000022A8AEA000184F8CD1087D12378C02BBF
:10195000DAD86278FF2A08D1052BD5D9012384F87B
:10196000C430072304F8023C78E7A4F8C120002221
:101970009342C4F8C93014BF0523062384F8C3205A
:10198000C4F8C52004F8023C68E7D4F8C500BB19C8
:101990000344421CC4F8C52083F8CFA194F8CD00BD
:1019A000D4F8C9308AEA00019A4284F8CD107FF455
:1019B00055AF062304F8023C50E794F8CD3083423B
:1019C000A2D10D2304F8023C14F8017C002F40F052
:1019D000F980674B08940FCB04AE86E80F00D4F86B
:1019E000C930D4F8D100ADF82C7023440993B4F871
:1019F000C130ADF8283094F8C3308DF82A30012377
:101A00008DF82E30324603AB08A9039729F062FD0A
:101A100048B1049B059394F8C420564B0493314677
:101A2000584623F05BFF039E002304F8023C002E7F
:101A300040F0DE8008F10108B8F1030F04F1E00482
:101A40007FF4F4AE0DB0BDE8F08FD4F8C500BA193C
:101A50000244431CC4F8C53082F8CFA194F8CD20CD
:101A600094F8CE0001938AEA020284F8CD20514610
:101A7000D52242F06FFB019B84F8CE00072B7FF448
:101A8000EDAEB4F80530C02B3FF63EAFB4F80320FE
:101A9000A4F8C120A27884F8C32000229342C4F89D
:101AA000C93014BF08230923C4F8C52004F8023C38
:101AB000D4E6D522014694F8CE0042F04BFB94F8D0
:101AC000CD3084F8CE008AEA0303D4F8C50084F848
:101AD000CD30BB190344421CC4F8C52083F8CFA104
:101AE000D4F8C9309A427FF4B9AE092304F8023C15
:101AF000B4E694F8CD30434084F8CD3094F8CE303D
:101B000083427FF401AF54E7D4F8C500BA19024408
:101B1000431CC4F8C53082F8CFA194F8CE000193DD
:101B2000D522514642F016FB019B84F8CE00052BCE
:101B30007FF494AEB4F80120B4F80330A4F8C120C7
:101B4000227884F8C32000229342C4F8C93014BF1D
:101B50000B230C23C4F8C52004F8023C7EE600BF2A
:101B6000B74F0020D86F0020E84D0020E05E002035
:101B700010B90508B80A0120F82B0020D52201462B
:101B800094F8CE0042F0E6FA84F8CE00D4F8C5000E
:101B9000BB190344421CC4F8C52083F8CFA1D4F874
:101BA000C9309A427FF45AAE0C2395E694F8CE30B1
:101BB00083427FF4A9AE04E7232804BF022204F87D
:101BC000032C77E6012F4FF0000602D004F8026CD8
:101BD00030E7D4F8C93008942344099308A8B4F82E
:101BE000C130CDE90A66ADF828301FF005F9EDE700
:101BF00054F80B0C27F05EFB54F80B0CB04719E7B8
:101C000014F8033C002B3FF415AFD9F8302054F8FA
:101C1000071C521A632A7FF60DAF012B28D0022B26
:101C20007FF408AF54F80B3CC5F81C33C5E9C43346
:101C30000122402389F8422B85F820330D4A0E4BB0
:101C4000C5F8182385F821030C4A0D48C3F8082469
:101C5000C5F8642337F01AFB4FF4005029F0AAFAB4
:101C6000084837F009FB85F8686385F86963E1E6A1
:101C7000FFF7CAFD21E70308E05E0020F0720020B4
:101C8000762F0608AC2F060800B583B00268074B14
:101C90008188CDF8012032221B68ADF805108DF83F
:101CA00000206846984703B05DF804FBC872002026
:101CB0005E2810B50ED05D2804D00B4BBDE8104057
:101CC0001B681847084C2368984723683D20BDE8E7
:101CD00010401847044C5D202368984723683E2035
:101CE000BDE81040184700BFD88B00200B2812D841
:101CF00010B401EB4103084C01EB83032344184467
:101D00000379934204D021440023027181F87C308E
:101D10005DF8044B70477047D88B0020084B5A88F9
:101D20001B88801A9B1AC00090FBF3F00628A8BFFE
:101D3000062020EAE070C0F19600C0B2704700BFF4
:101D4000A4370020094B03EB4002B2F88610084A82
:101D5000127802EAD122520707D0D3F80421511C8D
:101D6000C3F80411134483F808017047D88B00208E
:101D70000006002010B5164B42681B7803F00303E1
:101D8000032B21D1134B1B88DBB1134B1349B3F940
:101D90004631B1F904100A2491FBF4F15B1A1B01DE
:101DA00003F5B95314334FF4B471B3FBF1F3C3F13A
:101DB000080303F00F0360331370436800225A7066
:101DC00010BD05231370F8E72D231370F5E700BF4E
:101DD0004437002060370020D88B00202C380020AA
:101DE000436872221A70436873225A7043687422DF
:101DF0009A7043680022DA7070470F4B4268B3F95B
:101E000004300A2193FBF1F31B0110B503F5B9531C
:101E10000A4C4FF4B4711433B3FBF1F303F00F0326
:101E2000E118E35813604B6853600B7A13724368F0
:101E300000225A7210BD00BF2C38002058B9050886
:101E4000044B93F84D3113F0FD0F14BF9E209D20DD
:101E5000704700BFD88B0020094B93F84D3113F029
:101E6000FD0F06D142F210735843064B90FBF3F07E
:101E70007047242358434FF47A7390FBF3F0704774
:101E8000D88B002040D20600064B07EE900A93F84C
:101E90004D31B8EEE70A1BB9DFED037A20EE270AD1
:101EA000704700BFD88B002048F95140831E00F1D5
:101EB0007A02EA2123F8021F9342FBD14E2243F615
:101EC0004913C280CE2243850281CD232322838001
:101ED000A0F87220A0F87830704700BF08BB1F48F8
:101EE000B0F8B43103F001036BBB30B490F8B841E3
:101EF000ACB11B4A02F1F00502E00133A3420ED05F
:101F000052F8041B4904F8D590F8A41200EB8101A3
:101F1000D1F83C1245F823100133A342F0D130BC74
:101F200070470E48B0F8B421032A4FEA52030BD988
:101F30000A68A0F8B43102F5C332A03203F00103FD
:101F40000A60002BD1D070470B6803F5C333A03370
:101F500048F205020B60A0F8B4217047D88B00202E
:101F6000948D00202DE9F04100283AD12D4A92F8B5
:101F7000B80180B32C4A2D4B92F804E092F905C0C9
:101F800092F90680CEF1FF07AEF17F06FFB2F6B2FE
:101F900003EB800003F1F002002403E0834202F12E
:101FA000040218D053F8041B8904F7D5E1B2A1EB61
:101FB0000C0181EAE175A5EBE175012D0DDC71B134
:101FC000414514BF394631468342D17004F10104C2
:101FD00002F10402E6D1BDE8F0810821F4E7714680
:101FE000F2E7114B1A79F02A09D802F10F000D4AD5
:101FF00018710B6803F582431A330B60B7E7094A7F
:1020000093F9054092F8BA017F2584421D719879B1
:1020100005DB4042C0B2987120445871E9E7002CBA
:10202000FADAF6E7D88B002000060020948D002015
:10203000F0B5384E78B196F82C33002B46D0364A9E
:10204000013BDBB286F82C331378DC0741D4334BE9
:102050000A681A440A6096F8B8414CB3304B2E4FC8
:1020600003EB840403F1F001002503E09C4201F13D
:1020700004011DD053F8042BC2F303200628F5D128
:102080003878C00715D596F82C0396F8BBE100EB1D
:10209000050CBCFBFEF00EFB10C00128CCBF0020DD
:1020A000012058B99C4205F1010501F10401E1D17B
:1020B000F0BDE84300F001000028F3D0C2F38342F2
:1020C00006EB8202D2F83C220A60EBE796F8BB31BD
:1020D000B5E7D6EDCF7A134B134CFDEEE77A6420CB
:1020E00017EE902AA2F57A7200FB02F283FB02300F
:1020F000D317C3EBA01303EB4303C3EB031384FB1E
:102100000302DB17C3EB62130533084A92FBF3F3B8
:102110009EE700BFD88B0020DA360020400D030078
:10212000948D0020D34D62101F85EB5140420F006B
:10213000F0B4524C002868D194F87803002856D0A7
:102140004F4BD3ED007AB3EE097AF4EEC77AF1EE95
:1021500010FA4EDCBBEE097AF4EEC77AF1EE10FA13
:102160004CBF08270027D3ED017AB3EE097AF4EECD
:10217000C77AF1EE10FA3EDD47F0010794F8B85146
:10218000ADB3404ADFF808C102EB850502F1F0006B
:1021900014E094F97B63B142ACBF0221002194F9B1
:1021A0007C63B3421CDB41F004010F421CBFDCF82E
:1021B00024300360954200F1040018D052F8043B2B
:1021C000D903F7D594F97A6303F00F01B142C3F351
:1021D0000313DEDC94F97C63B3424FF00101E2DAD1
:1021E00094F97D63B342D8BF41F00801DDE7F0BC4C
:1021F00070470427B7E7BBEE097AF4EEC77AF1EE31
:1022000010FA48BF47F00207B8E794F8793363B390
:102210001B4B1D4DD3ED007A93ED017A0A6894F8BB
:102220007803F0EEE77AB0EEC77AF4EEC77AF1EE13
:1022300010FAB8BFF0EE477AFDEEE77A80F00100C1
:1022400017EE903A193B03EB4303C3EB031385FBF3
:102250000365DB17C3EBE51305330C4DB5FBF3F357
:102260001A440A6084F8780368E70B6894F87803E6
:1022700003F5433303F5A0730B605FE7D88B0020B1
:1022800094370020948D0020353AFC4440420F00E2
:1022900058B90508F0B40B4F97F8B86186B107F547
:1022A000DE72054607F52B77002352F8044B35EA1A
:1022B000040004BF086847F823000133B342F4D197
:1022C000F0BC7047D88B002030B42A4B60B92A4844
:1022D000027DCAB993F8A5322849203301EB830166
:1022E00030BC4FF4A060D5E793F87E23F2B1013AF9
:1022F000214883F87E230A6802F5C32202F5207282
:102300000A60027D002AE5D01D4A12689106E1D5D7
:102310001C4A93F87E13127892071AD511BB93F8D2
:10232000A7321649203301EB8301D9E7124893F80D
:102330007F43057DA54205D8042483F87F2383F8D5
:102340007E43D8E70134012283F87F4383F87E235C
:10235000D1E70029BED193F8A6320849203301EB1A
:102360008301BDE793F8A3320449203301EB8301D5
:10237000B6E700BFD88B002048370020948D00209E
:10238000343800204437002010B41E4A48B91E4C8F
:1023900092F880030B6823440B6098B15DF8044BFE
:1023A000704792F8813303B3012B16D092F8800363
:1023B0000B68164C80F00100234482F880030B6008
:1023C0000028EBD192F8A33211495DF8044B203379
:1023D00001EB83014FF440705CE792F880030D4CF1
:1023E00080F0010082F88003D4E70B685DF8044BAD
:1023F00003F5742303F5107301200B6082F880034A
:10240000704700BFD88B002040420F0048E8010011
:10241000948D002020A107003C4AA0B992F8823395
:102420006BB192F883138A081341DB070AD501F0D8
:102430000101032A06D8DFE802F05048403892F83C
:10244000853353BB704792F88333013303F00F0396
:1024500082F883333BB192F88233086800F5C330C9
:10246000A0300860DCE72A4882F88233437A002BE8
:1024700044D12848C07818B143F0040382F882336D
:1024800025480078C00730D592F884030028E4D0AE
:1024900043F0080382F88233DFE792F892331F4952
:1024A00001EB83014FF40030F4E61C4B03F13002E2
:1024B000002914BF19461146F4E7194B03F118021D
:1024C00000290CBF19461146ECE7144B03F1080232
:1024D000002914BF19461146E4E7104B03F1180216
:1024E000002914BF19461146DCE70E480068002891
:1024F000CAD043F0010382F88233C5E792F88133F2
:10250000002BB6D0022382F88233B2E7D88B0020AA
:10251000A4370020DC360020DA36002070B9050828
:1025200080B90508D472002090F8603043B9426940
:102530000121072082F84430A2F8460082F84810B2
:10254000704700BF034A0123E021C37382F895134B
:1025500018467047D88B00204FF0FF30704700BFFF
:10256000704700BF704700BF0020704770B4067A04
:10257000AEB1427A0B4800212025002352B1142B22
:1025800005DC072903DCC45C202C18BFC5540133CB
:102590009342F4D101318E4200F11500EDD10020BB
:1025A00070BC70476F8F002010B50024C473FFF714
:1025B000DDFF034B012283F89523204610BD00BFA9
:1025C000D88B002070B403980378BBB10D4C02EB9C
:1025D0004205C5EBC5052544142901F1010408D8BD
:1025E000072A294405D891F897639E4218BF81F8BD
:1025F000973310F8013FE1B2002BEDD1002070BC01
:10260000704700BFD88B002014299DF800000ED819
:10261000072A0CD8074B02EB4202C2EBC2021A4453
:10262000114491F89733834218BF81F89703002033
:10263000704700BFD88B0020027A407A02FB00F07E
:10264000704700BF027A407A02FB00F0704700BF7B
:10265000002070474FF0FF30704700BF034B93F8E6
:102660006125027293F8623543727047D88B00205F
:1026700000207047012070470120704700207047FC
:10268000027A407A02FB00F0704700BF00207047DA
:102690000123C373184670470123C373184670475C
:1026A0004FF0FF30704700BF002070470120704797
:1026B00000207047F8B507460026F5B20024E0B2C6
:1026C000202229460134FFF711FB0C2CF7D10136EB
:1026D000092EF2D11B4D4222012420460021FFF792
:1026E00005FB15F8012F0134E4B2002AF5D197F962
:1026F0000F302BBB144D14464D22E0B20221FFF7E0
:10270000F5FA15F8012F0134002AF6D10F4D2B22CE
:10271000022420460321FFF7E9FA15F8012F0134BE
:10272000E4B2002AF5D10A4D2B22022420460421CE
:10273000FFF7DCFA15F8012F0134E4B2002AF5D1D5
:102740000020F8BDB42F0608C02F0608D02F0608B9
:10275000DC2F060810B50024C473FFF7ABFF20463A
:1027600010BD00BF70B5049C23786BB115460E1BDD
:102770003019082DC0B21A46294601D8FFF7B6FA1B
:1027800014F8013F002BF3D1002070BD08B51346AB
:10279000082B9DF8082003D808461946FFF7A6FA2B
:1027A000002008BD027A407A02FB00F0704700BFAB
:1027B0000020704700207047914201D0012A01D9C2
:1027C000002070470129FBD808B5074BC1EB011069
:1027D000C2EB021203EB421103EB40104FF4F07214
:1027E00048F014FF012008BD5839002001299DBF81
:1027F000024B012083F8641500207047D88B00201D
:1028000001298CBF00200120704700BF4FF0FF302E
:10281000704700BF00207047034B1B68186A0038E0
:1028200018BF0120704700BF1C3D002030B41D2997
:102830009DF808000DD80F2A0BD8074B074D93F8C9
:1028400064451E23C4EB041413FB021202EB441272
:102850005055002030BC7047D88B002058390020DC
:10286000014B1889704700BF000600200020704708
:1028700000207047074BB3F8BA16B3F8BC260346DE
:1028800010B4054C1C6001205DF8044B19815A817D
:10289000704700BFD88B0020A8B90508024B01463D
:1028A000D3F8D4062EF050BDD88B00202DE9F84384
:1028B0000546184C8846D4F8D80629782EF044FDF1
:1028C0006978D4F8D8062EF03FFD0026A84405F11B
:1028D0000209374619F8011BD4F8D8060E44F6B29F
:1028E0002EF032FD3744C845FFB2F3D1D4F8D806F4
:1028F00031462EF029FDD4F8D80639462EF024FDB5
:10290000EB7884F8F7364FF48073A4F8F836BDE816
:10291000F88300BFD88B002070B5214D95F8FC36A8
:10292000EA181C4692F87C208AB11E4E09225C1CD3
:10293000A6FB04135B0803EBC303E31AE918DCB23C
:1029400091F87C1009B1013AF1D185F8FC46026892
:102950001549561C06600C2616700268561C066047
:10296000002616700268561C066003EB430603EB54
:102970008603147019440D2240F0D0FE95F8FC1621
:10298000084B4A1CA3FB02035B08294403EBC30367
:102990000120D31A81F87C0085F8FC3670BD00BF99
:1029A000D88B0020398EE338DC8B00202DE9F041F4
:1029B000294D2A4A2B682A4C2E89B4F8FE7682FBD0
:1029C0000352DB17C3EBA2031FFA83F8474582B01B
:1029D0000D4603D1B4F80037B34233D002680190FA
:1029E000511C34230160137002680023511C0160E4
:1029F0001370414640F0F6FE0198314640F0F2FE79
:102A0000019847F6FF7140F0EDFE019847F6FF711F
:102A100040F0E8FE019847F6FF7140F0E3FE0198B0
:102A200047F6FF7140F0DEFE01980221FBF756F9F0
:102A30000120A4F8FE86A4F80067C4F8045702B089
:102A4000BDE8F081D4F80437064ACB1A9342C5D8C2
:102A5000002002B0BDE8F081C037002067666666DE
:102A6000D88B002080841E00026810B57F21541C82
:102A70000460117002680024511C01600E21147062
:102A8000FBF72CF9012010BD2DE9F041694F6A4D8B
:102A9000D7F8008084B0044640460E460CF09FFCF8
:102AA00085F80807B8F1000F0AD00DF1090202A954
:102AB00040460CF0C6FA002840F08D8095F80807D3
:102AC0000023ADF808308DF80A301A46431EDBB2F9
:102AD0000021FF20FD2B8DF80C20ADF80E108DF895
:102AE0000B0003D9002004B0BDE8F0819DF8083048
:102AF000042B00F09580052B00F09880032B00F04C
:102B00009780022B00F08B80012B08BF042100F07E
:102B100087809DF8093038689DF80A10013B0DF157
:102B20000E028DF809300CF0F5F995F80837032BF3
:102B300073D0042B0CD1414A9DF80A0001210023D7
:102B400001E012F8011F81426DD20133082BF8D148
:102B5000D5F80C27029B3A4F9A420DF108084FD046
:102B600023680D22591C21601A7023680022591C09
:102B700021601A7023689DF80820591C21601A7082
:102B800023689DF80920591C21601A7023689DF85C
:102B90000C20591C21601A7023689DF80A20591CCA
:102BA00021601A70BDF80E10204640F01BFE23680D
:102BB0009DF80B20591C216020461A700721FBF755
:102BC0008DF898E8030087E803000120C5F8146732
:102BD00004B0BDE8F08101A940460CF029FA0028B4
:102BE0003FF46CAF40460DF10A010CF027FA0028C3
:102BF0003FF464AF019B95F8080703F0010265E715
:102C00007A68D8F804309A42AAD1D5F814370D4A18
:102C1000F31A93427FF666AFA2E70B4A8CE70321D3
:102C20008DF8081075E78DF80A3091E70121F7E774
:102C30000221F5E724370020D88B0020CFB7050804
:102C4000E492002080841E00C7B705082DE9F04FEC
:102C5000C14B1B68804613F0800083B000F0708188
:102C6000BE4B187810F0020000F06A81DFF80CB358
:102C70009BF81430052B40F26881DBF80030B84D2A
:102C80000093002BB8BF5B42A5FB0342B548B64991
:102C9000920D00FB0233C3EB03139B0085FB03453E
:102CA00002EB8202DC1702EB8202C4EBA55400FBAC
:102CB000043304EB8204A4B281FB0321DB17C3EBD2
:102CC000A111BCB10025A94F2E46A7FB0432D208A2
:102CD00002EB8203A4EB4303E8B2A4469BB280005C
:102CE0008340BCF1090F94B246EA030605F10105E1
:102CF000EBD8340489B2B9B100259C4F2E46A7FB0E
:102D00000132D20802EB8203A1EB4303E8B28C4606
:102D10009BB280008340BCF1090F91B246EA0306E2
:102D200005F10105EBD83443DBF804E08C4D8D4E02
:102D30008D498EEAEE70A0EBEE70A5FB0032920D8D
:102D400006FB0200C0EB0010830085FB035002EB82
:102D50008202DD1702EB8202C5EBA05506FB0533AC
:102D600005EB8205ADB281FB0321DB17C3EBA1119B
:102D7000C5B10020DFF8F4C10646ACFB0532D2082D
:102D800002EB8203A5EB4303C7B2A9469BB2BF0087
:102D9000BB40B9F1090F95B246EA030600F1010004
:102DA000EBD8350489B2C1B10020DFF8C0C10646B6
:102DB000ACFB0132D20802EB8203A1EB4303C7B2A2
:102DC00089469BB2BF00BB40B9F1090F91B246EAF8
:102DD000030600F10100EBD83543DBF80830634A05
:102DE0000193002B1846B8BF5842A2FB0030604E3A
:102DF0006049030AA6FB0363DB0901FB03F1C1EB96
:102E0000D00189B2B9B1002691463746A9FB0132FB
:102E1000D20802EB8203A1EB4303F0B28C469BB2D3
:102E200080008340BCF1090F91B247EA030706F125
:102E30000106EBD8B9B2BBF81070DFB10026DFF89D
:102E40002CA1B446AAFB0732D20802EB8203A7EBFF
:102E500043035FFA86F938469BB24FEA890903FAC1
:102E600009F3092897B24CEA030C06F10106E9D8E8
:102E70001FFA8CF7BBF812303C4AA2FB0306F60897
:102E8000632E28BF6326092B63D900209346814611
:102E9000ABFB0632D20802EB8203A6EB43035FFAD8
:102EA00080FAB4469BB24FEA8A0A03FA0AF3BCF1ED
:102EB000090F96B249EA030900F10100E8D85FFA68
:102EC00089F9009B019A002BCCBF392338231616B1
:102ED000BEF1000F26F07F0635DD274A33439645C5
:102EE00043F00206C8BF43F00606D8F800301622A9
:102EF000581CC8F800001A70D8F800300022581C7E
:102F0000C8F800001A70404640F06CFC214640466C
:102F100040F050FC2946404640F04CFC40463946C3
:102F200040F060FCD8F800305A1CC8F8002083F844
:102F30000090D8F800305A1CC8F8002001201E70FC
:102F400003B0BDE8F08F1E43CFE7002003B0BDE81B
:102F5000F08F4FF00009B4E7CC3700204437002051
:102F60006BCA5F6B806967FFD34D6210CDCCCCCC50
:102F7000C55A7C0AA0860100FFC99A3B4837002049
:102F80002DE9F047AB4B1B68064613F0800084B078
:102F900000F09D80A84B187810F0020000F0978098
:102FA000A64F397D052940F29780632900F292806F
:102FB0000024DFF89CC289B22546ACFB0132D2085E
:102FC00002EB8203A1EB4303E0B28E469BB280008A
:102FD0008340BEF1090F91B245EA030504F10104F3
:102FE000EBD8EDB2BB68964A82FB0312D917C1EB4E
:102FF000623189B2002900F018814FF0000CDFF82F
:1030000050E26446AEFB0132D20802EB8203A1EB30
:1030100043035FFA8CF088469BB280008340B8F18E
:10302000090F91B244EA03040CF1010CEAD8E4B2AE
:10303000FB8984494FF4F36707FB03F7A1FB0737CC
:10304000C7F38F1742F20F739F4249D8CFB10020C8
:10305000DFF8FCE18446AEFB0732D20802EB8203C4
:10306000A7EB4303C1B2B8469BB289008B40B8F1CD
:10307000090F97B24CEA030C00F10100EBD81FFADC
:103080008CF7714BD3E9002313433ED14FF0FF3847
:1030900033681722591C31601A7033680022581C9B
:1030A000306039461A70304640F09CFB414630464D
:1030B00040F080FB33685A1C32601D7033685A1C24
:1030C000326030461C700621FAF708FE012004B079
:1030D000BDE8F087992585E7002004B0BDE8F087BA
:1030E0000021DFF86CC10F46ACFB0302D20802EBF3
:1030F0008200A3EB40039BB28B400431102947EAC6
:10310000030793B2F0D1BFB2BBE701A840F0AEFF16
:103110009DF80810002900F08A804FF0000CDFF8BD
:1031200030E1E046AEFB0132D20802EB8203A1EBB4
:1031300043035FFA8CF089469BB280008340B9F16B
:10314000090F91B248EA03080CF1010CEAD84FEAE2
:1031500008289DF80910E1B10020DFF8F4E084466A
:10316000AEFB0132D20802EB8203A1EB43035FFA0C
:1031700080F98A469BB24FEA890903FA09F3BAF14A
:10318000090F91B24CEA030C00F10100E8D848EABB
:103190000C089DF80A104FEA0828E1B10020DFF87A
:1031A000B0E08446AEFB0132D20802EB8203A1EB11
:1031B00043035FFA80F98A469BB24FEA890903FA12
:1031C00009F3BAF1090F91B24CEA030C00F10100C6
:1031D000E8D848EA0C08BDF80C301C49632BA1FB69
:1031E00003214FEA08184FEA51117FF651AF002032
:1031F000DFF85CE08446AEFB0132D20802EB8203CA
:10320000A1EB43035FFA80F98A469BB24FEA890932
:1032100003FA09F3BAF1090F91B24CEA030C00F179
:103220000100E8D848EA0C0832E70C4600E7884677
:103230008FE700BFCC3700204437002048370020FC
:1032400089B5F814D34D6210F09200201F85EB5120
:10325000CDCCCCCC044B93F8B1310BB121F018BEDE
:10326000024B1888704700BFD88B00208837002099
:1032700002683B4B70B505467E21501CB3F9003007
:10328000286011702968374C03EBC30384FB0302E9
:10329000481CDC17002328600B70FF20C4EB62047D
:1032A000FDF76EFA2034304BA4B200284DD01B78C5
:1032B000B0F90C1023BB2D4BA1F57A729A4246D877
:1032C0002B48B0FBF1F189B2284640F065FA294B52
:1032D000DB7A7BB121F0DCFD0146284640F05CFA48
:1032E0002146284640F058FA28460821FAF7F6FC0D
:1032F000012070BD204B2846198840F04DFAEFE7B9
:103300001E4B1E78002ED6D01D48002300EB8302F2
:1033100001339289B3421144F8DB1A4B9FED1A6ACC
:1033200093F8223007EE103A07EE901AB8EEC77AFB
:10333000F8EE676AC6EE077A67EEA67AFCEEE77AE1
:1033400017EE901AB1FBF6F1B5E71B7813B94EF6FC
:103350009C21B9E7094B1E78002EF8D00146D3E72F
:10336000E472002067666666875E00201783930319
:10337000008793036437002088370020F42C002056
:10338000F89200204C3300200000484310B5194C3F
:10339000A379D3B194F82230DFED176A07EE903AA3
:1033A000F8EEE77A154B86EEA77AC0B203EB800001
:1033B000B0F82C3707EE903AF8EEE77A67EE277A06
:1033C000FDEEE77A17EE900A10BD0D4B1B6813F067
:1033D00000630CD0C0B2FDF7D3F98089642310FBE1
:1033E00003F094F822305B0890FBF3F0ECE718460A
:1033F000EAE700BF4C33002000004843D88B002090
:10340000CC37002008B5FFF7C1FF3C2390FBF3F059
:1034100008BD044B0449B3F90A304068012241F069
:1034200023BE00BF000600206A2F0608064B07498E
:103430001A88074B40681B68534342F2107293FB93
:10344000F2F241F011BE00BF88370020FA340608BE
:10345000C0370020054A064992F8A53792F8A427FC
:1034600040680133013241F0FFBD00BFD88B00201E
:10347000FF3406080B4B4068B3F904300A2293FB73
:10348000F2F31A0102F5B9524FF4B4711432B2FBDF
:10349000F1F2C2F1080202F00F020349603241F07A
:1034A000E3BD00BF2C38002005350608034A044957
:1034B00092684068072341F0D7BD00BFC0370020A5
:1034C0000C35060807B5144A406892F8B517B2F8EB
:1034D000B637012909D1009392F8B8370F497B22FA
:1034E00041F0C2FD03B05DF804FB022906D10C498E
:1034F0007B2203B05DF804EB41F0B6BD0A225343D2
:1035000040F2FF32B3FBF2F39BB2092B054928BF0F
:1035100009237B22EDE700BFD88B00201235060877
:103520003B3606081C3506081F4B1A6812F02002AD
:1035300013B501461AD01D4B1A7812F0010215D0AE
:103540001B4B1A7812F0020210D01A4BDB89632B46
:1035500020D964205843FEF77FFC00281ADD164B63
:103560001B684FF47A725A4392FBF0F2134B48688F
:1035700093F84D31541E002B42F20E710CBF7E2386
:103580007D238C4208D800930D49072341F06CFD40
:1035900002B010BD0022E9E70A49072202B0BDE8E7
:1035A000104041F061BD00BF34380020DA36002001
:1035B0004437002048370020C0370020D88B002037
:1035C000223506082B35060813B54468FEF738FC8B
:1035D0000F4B1B789B07024612D50E4B93F8C3176F
:1035E0000D4B59B19889FEF737FC0C490092034600
:1035F0007022204641F038FD02B010BDD889F2E7B4
:10360000009007492D237022204641F02DFDF3E75D
:1036100044370020D88B0020483700201536060894
:1036200035350608034B0449D3F8C827406841F0F4
:103630001BBD00BFD88B00203C350608044B1B780F
:10364000DB0703D40349406841F00EBD704700BF5B
:10365000DA3600204035060807B5094A0949B2F9AB
:1036600006300193B2F904300093B2F90230406899
:10367000B2F9002041F0F8FC03B05DF804FB00BF94
:10368000C432002049350608084BD3F8D827002A51
:103690000BDD074B03EB8203D3F8D8202AB1054B8F
:1036A0000549DB68406841F0DFBC7047D88B0020DB
:1036B00058B90508000600205D3506081FB5938837
:1036C0000293937801935378009313780A46034941
:1036D00041F0CAFC05B05DF804FB00BF6535060883
:1036E000024B03491A6840681432E7E7DC72002095
:1036F00078350608024B03491A6840680832DDE74E
:10370000DC7200207C350608024B03491A684068C9
:103710000E32D3E7DC72002080350608F0B5194F71
:1037200097F86135934283B022D997F862658E424B
:103730000D461DD90898144644F092FD731B834230
:1037400007F5886C06FB0454A8BF034664441A4678
:1037500008990193204647F092FF97F86035019A47
:103760001843002814BF0123002387F8603502D1D5
:10377000002003B0F0BD0899204647F047FF002025
:1037800003B0F0BDD88B0020F0B587B005AF04467C
:103790000D46164607499DF830200393384641F000
:1037A00063FC039B0097324629462046FFF7B6FF8D
:1037B00007B0F0BDE82F06081E4B1F499A68B1F804
:1037C00048319FED1E7A406807EE902AF8EEE76ACE
:1037D00007EE903AF8EEE77A67EE877AF4EEE76A5A
:1037E000F1EE10FA02D8164941F03EBC934202DADB
:1037F000144941F039BC9B1A07EE903A01F2DC7390
:10380000B8EEE77AD3ED007A0F4AF8EE677A3C21FA
:1038100067EE277A87EEA67AFDEEC77A17EE903A22
:10382000B3FBF2F3B3FBF1F201FB1233074941F0B2
:103830001BBC00BFC0370020D88B0020CDCCCC3DB6
:10384000843506088A35060840420F009035060880
:10385000244A00234361D2F85C1141F45C5130B535
:1038600041F02C010124C2F85C114471D2F85411CA
:1038700004FA03F50133112B41EA0501F8D121F4D3
:10388000F0314FF42063C2F85411C38040F6012395
:103890000381154B0360142303718023037642F6E2
:1038A00014035022114903824FF6FF734383A0F89B
:1038B000562003F58C036FF07E42C0E91612C361F7
:1038C0000B4A40F2012303844FF0A0640023C0E9B7
:1038D000184280F8223080F8333080F84430A0F865
:1038E000683030BDD88B002098086400C4FF00FF0A
:1038F000180B3C0008B5A0F10103B3FA83F30228CA
:103900004FEA531301D0184608BD0F201BF02AF8C8
:1039100028B9054B1B7803F00103184608BDBDE824
:1039200008400F201BF0ACB8DA36002010B5044672
:1039300013201BF0A5F8A0B10A4B606893F8E127AB
:10394000032A4FF0100202D1D3F8EC3723B9BDE8B7
:103950001040054941F088BBBDE81040034941F0E3
:1039600083BB10BDD88B00209A350608E82F0608C7
:1039700038B5802200F180040021054647F0A7FEFB
:1039800000212046382247F0A2FE0C49002351F8BE
:10399000232044F8232001330E2BF8D108491E229E
:1039A00005F1C00047F032FE06490B2205F1E400A4
:1039B00047F02CFE032385F8EF3038BD70B90508B9
:1039C000B8BA0508D8BA050810B50A4C4FF4907279
:1039D00004F58860202147F07AFE074B1B6801221E
:1039E0002D33002084F86325C4F8F03784F860058F
:1039F00010BD00BFD88B0020282C00200022C273ED
:103A0000E2E7234B1B885A0510B5446805D52046CC
:103A10002049BDE8104047F07EBE180505D5204678
:103A20001D49BDE8104047F076BE590605D5204631
:103A30001A49BDE8104047F06EBEDA0705D52046AA
:103A40001749BDE8104047F066BE9B0705D52046E4
:103A50001449BDE8104047F05EBE25201BF010F869
:103A600028B120461049BDE8104047F054BE0F4B26
:103A700093F8F4372BB120460D49BDE8104047F0CC
:103A80004ABE20460B49BDE8104047F044BE00BF87
:103A9000D03700209E350608A3350608A83506084D
:103AA000AD350608B2350608B7350608D88B0020B4
:103AB000BC350608C1350608074B93ED6E7AD3ED89
:103AC0006B7AB4EEE77AF1EE10FA03DD0349406851
:103AD00047F021BE704700BFD0630020C6350608FE
:103AE00010B50C46A0B9184A184892F8F517236883
:103AF0000344236001B110BD92F8A332144920336E
:103B0000BDE8104001EB83014FF48060FEF7C2BBBB
:103B100011F0E6FC32280ADD23680B4A03F5742312
:103B200003F510730121236082F8F51710BD064AD2
:103B300092F8F517142881F00101CCBF054806481A
:103B400082F8F517D3E700BFD88B002040420F0062
:103B5000948D002020A1070048E8010010B504461C
:103B60001DF05AFC0349034604226068BDE810407A
:103B700041F07ABA6A2F0608032811D8DFE800F06E
:103B80000A0C0206074BD3F8F8077047064B1B7860
:103B9000DB0701D42CF0C6BF024BD3F8DC0770471B
:103BA00000207047D88B0020DA36002037B5044655
:103BB0002A4800EB4303B3F84E5105F00F0049B11A
:103BC000022804F101011DD8002814BF9C239B2367
:103BD00023700C460AB3C5F30315FFF7CDFF3C2154
:103BE000012D1F4BB0FBF3F3B3FBF1F201FB1233DA
:103BF00015D0022D23D01B49204603B0BDE830402C
:103C000041F032BA032806D1174B1B7803F00103A9
:103C1000653BDBB2DCE72023DAE71546DDE7642508
:103C200042F21071B0FBF1F1B1FBF5F005FB1010A1
:103C300000900E49204641F017FA03B030BD0A2526
:103C40000B49B0FBF1F1B1FBF5F005FB1010009052
:103C50000849204641F008FAEFE700BFD88B002062
:103C600040420F0090350608DA360020C9350608B4
:103C7000A0860100D8350608037840680122053B7C
:103C8000114693E7F0B52B4B2B4E1C68317887B06B
:103C9000074620460BF0BAF97178054620460BF02E
:103CA000A1F900220592B2788DF8132003466CB179
:103CB000039005A920460BF0BBF9327A039B2AB189
:103CC0000DF1130120460BF0B9F9039B9DF8131079
:103CD000ECB1E1B1194A1268914218DC184A02EBC2
:103CE0008102D2F82048039326201AF0C9FE0599D4
:103CF000039B70B911F0010F14BF502200228907F5
:103D0000786808D50F4941F0AFF907B0F0BD0E4C07
:103D1000E9E74422F3E732B1CDE900420B492A46F4
:103D200041F0A2F9F1E70A4900942A4641F09CF9D2
:103D3000EBE700BF24370020D0360020A02C002065
:103D4000D88B0020E73506088A390608EF350608C3
:103D5000FB350608F8B50446417882782C4823786C
:103D600090F86951302B05F1FF352A4B4FEA850554
:103D70002B444FF47A770BBF93F88B5193F88D5106
:103D800093F88C6193F88E6100EB8505D5EDCC7AC4
:103D9000FDEEE77A00EB860017EE903AD0EDCC7A94
:103DA00040F2CF75FDEEE77AAB4217EE900AA8BF5E
:103DB0002B46B3F57A7FB8BF4FF47A73A842A8BFF9
:103DC0002846A3F57A73B842C3EB0313B3FBF7F3AA
:103DD000C3F10E03B8BF3846DBB24FF0030CB3FBA0
:103DE000FCFC0CEB4C0EA3EB0E03A0F57A706244C6
:103DF000C0EBC0000833B0FBF7F73944DBB2D2B2F6
:103E0000C9B22046FAF792FA00232373F8BD00BF27
:103E1000D88B002058B905082DE9F04790F802909A
:103E200090F8018009F1020704460026FFB2002540
:103E300008EB060A032E1BD108F10301022DC9B2BB
:103E40000ED10B233A462046FAF770FA0135052DBC
:103E5000F0D10136072EEAD100232373BDE8F087A5
:103E600009EB05021623D2B22046FAF75FFAEDE716
:103E7000022DEBD117233A465FFA8AF12046FAF772
:103E800055FAE3E770B504466FF00205A278617851
:103E900052FA85F207391323D2B2C9B22046FAF793
:103EA00045FAA2786178EEB2324407311323D2B2D8
:103EB000C9B220460135FAF739FA042DE6D1617806
:103EC000A27806390323C9B22046FAF72FFA61789F
:103ED000A27806310223C9B22046FAF727FA002356
:103EE000237370BD2DE9F8432B49054691F85831ED
:103EF00091F85921294891F86711B0F9004000293B
:103F000002EB820214BF4FF0FF31012152004C43FB
:103F1000C2F1000803EB830344454FEA430303DB8C
:103F20009442A8BF1446A046B0F902205C424A431E
:103F3000A24203DB9A42A8BF1A4614461BB11922BB
:103F4000544394FBF3F4293C4FEA88066FF00307CF
:103F50004FF00909002E3346B8BF06F13F03C4EB0A
:103F6000A313512B0FD893FBF9F101EBC1029B1A5C
:103F7000AA780A446978803B3944DBB2D2B2C9B22C
:103F80002846FAF7D3F90137052FA6EB0806E1D149
:103F900000232B73BDE8F883D88B00202C38002039
:103FA00010B5044611F0D8FA642202FB00F3C3F303
:103FB0008F23632B60680449BDE8104028BF63234A
:103FC000012241F051B800BF3B3606082DE9F84305
:103FD000054616F035F81D4EDFF8749007460024AC
:103FE0004FF0880833786968A342214403DC00233A
:103FF0000B70BDE8F88337B3D6ED427AFDEEE77A71
:1040000009EB840317EE900AD3ED007AFDEEE77A10
:1040100017EE902AD6ED437AFDEEE77A121A17EEE4
:10402000903AD2001B1A92FBF3F3C3F188030B7092
:104030002046FFF7ABF9B0F57A7F02DA6B685322BE
:104040001A550134CEE781F80080FAE7F42C0020FD
:104050001C94002013B5374BC1789A68364B02295F
:104060009B89044641D0032945D0012905D19A1ADC
:104070009A42A8BF1A4622EAE272D3B19A1A9A4229
:10408000A8BF1A4622EAE27207EE902A0B20B3FB81
:10409000F0F307EE103AF8EEE77AB8EEC70A87EECB
:1040A000800A45F0C7FDFCEEC07ACDED017A9DF89F
:1040B000043062688A211170012261689342ACBFAA
:1040C0008B208D20885401320C2AF6D162688F2112
:1040D00011735A1E092A03D8626813448E225A703B
:1040E000636800225A7302B010BD9A1A9A42A8BFA0
:1040F0001A4622EAE272ABB107EE902AB8EEE70A5E
:10410000DFED0E7A20EE270A07EE903AF8EEE77A16
:1041100080EE270A45F0D4FD64280346A8BF642337
:1041200023EAE37306496068072202B0BDE8104045
:1041300040F09ABFC0370020A43700200000C842DA
:1041400004360608084B93F84D3107EE900A4BB938
:10415000F8EEE77A9FED057A9FED050AA7EE870A4C
:1041600045F0AEBD704700BFD88B00206766E63FC4
:10417000000000420D4B1B681B0137B514D50C4CD9
:104180004568D4F8643893F90100FFF7DBFF94F831
:104190004D210849002A0CBF0D220E220346009231
:1041A00028467A2240F060FF03B030BDCC370020B3
:1041B000D88B00200B3606080B4B13B54468B3F9B7
:1041C0000000FFF7BFFF094A094992F84D21002A74
:1041D0000CBF0D220E220346009220467A2240F0A8
:1041E00043FF02B010BD00BFE4720020D88B002056
:1041F000143606082DE9F0472DED028B82B0924669
:104200009DF834809DF8302007460C469946002BD7
:1042100052D0022B14BF0A25642507EE905AF8EEFF
:10422000E77A27EE808A002A48D0B0EE480A45F0A7
:1042300047FD07EE900AF8EEE77AF0EEE77AFDEE3A
:10424000E77A17EE906AB6FBF5F205FB12660CB141
:104250003C700124B5EEC08AF1EE10FA05D552EAA1
:10426000060302D02D233B5501349AF80010154B5C
:104270003819002914BF5146194640F0F5FE25189B
:10428000B9F1000F0AD010494A46684640F0ECFEEA
:1042900078193246694640F0E7FE0544B8F1000F50
:1042A00002D007F805800135002328467B5502B06F
:1042B000BDEC028BBDE8F0870125AEE7F0EE487A51
:1042C000BBE700BF1D36060822360608194B1B68DF
:1042D00013F0200F13B5446825D0174B1B789B07AC
:1042E00021D5164BB3F90000FDF7CEFDDFED147AB2
:1042F000144B154A93F84D3120EE270A2046B5EEAF
:10430000C00AF1EE10FA4CBF76217521002B0CBFCC
:1043100099239F23019301230093B0EEC00AFFF776
:1043200069FF02B010BD2D232370436800225A702C
:10433000F7E700BF3438002044370020323800202F
:104340000AD7233CD88B0020A97606081FB5184B46
:104350009FED187A1B88184A9FED180A92F881235E
:10436000446807EE903AF8EEE77AF4EEC77AF1EE99
:1043700010FAACBF01230223022A27EE800A14D0D0
:104380008DED030A029320F083FDFDF7C7FC029B2D
:104390009DED030A014601220620CDE90020084ACE
:1043A0002046FFF727FF04B010BD9721F3E700BFB9
:1043B0008837002000007A44D88B00200AD7233C9D
:1043C000A9760608114BB3F86838B3F57A7F07B5BC
:1043D000406806D20E49012203B05DF804EB40F0BC
:1043E00043BE07EE903A5722F8EEE77A00239FED9E
:1043F000090ACDE900320123074A27EE800A19464F
:10440000FFF7F8FE03B05DF804FB00BFD88B002077
:104410002A3606086F12833AA976060873B5194E34
:1044200096F8F436052B0546406807D016491F2339
:104430001E2202B0BDE8704040F016BE134C144975
:10444000237D00931E221F2340F00EFE96F8A2311A
:10445000ABB16B68DFED0F7A20221A54638A0E4AE3
:1044600000EE103A441CB8EEC00A6868012300212F
:10447000CDE9003120EE270A2044FFF7BBFE02B051
:1044800070BD00BFD88B00203236060848370020A8
:10449000393606080AD7233CA976060807B5012352
:1044A0004722CDE900320549054A91ED000A4068EE
:1044B0000021FFF79FFE03B05DF804FB4494002049
:1044C000A976060807B50B4BDFED0B7A93ED000AD2
:1044D0000A4A00219A23B8EEC00ACDE9001320EE63
:1044E000270A0223B0EEC00A4068FFF783FE03B03C
:1044F0005DF804FBC03700200AD7233C413606088C
:1045000013B5044620F0C4FC0E4B646893F8813365
:10451000022B00EE100A13D0FDF700FC0146DFED80
:104520000A7AB8EEC00A00230622CDE9003220EE56
:10453000270A064A02232046FFF75CFE02B010BDA0
:104540009721ECE7D88B00200AD7233CA9760608F0
:1045500013B50378134ADFED147A144C1A2B0CBFF1
:10456000B2F90220B2F9002000EE102AB8EEC00A1B
:104570001A2B20EE270A4FF001034FF00002CDE97D
:104580000032B5EEC00A0CBF15211421F1EE10FA6D
:10459000074A406848BF2246B0EEC00AFFF72AFE2D
:1045A00002B010BD2C380020CDCCCC3D45360608DD
:1045B0004B360608174B1B689A0613B5446820D57E
:1045C000154B1B789B071CD5144BC27893F84D31C3
:1045D000002B134B18680CBF0F210C21FDF754FC66
:1045E0000123DFED107A0093D31A01910E4A20EED9
:1045F000270A18BF01237F212046FFF7FBFD02B0E9
:1046000010BD7F23237043682D225A704368002217
:104610009A70F4E73438002044370020D88B00200B
:10462000CC7200200AD7233CA976060813B50446AD
:1046300008461146FDF728FC174B93F84D31002B27
:104640000CBF4FF4A5534FF47A7307EE903AF8EE8F
:10465000E77A08BF7E22F4EEC07A16BF7D220F23D0
:104660000C23F1EE10FA13DC80EE270AF2EE047A46
:10467000B4EEE70AF1EE10FAACBF01230223019277
:10468000002200922046054AFFF7B4FD02B010BD9B
:104690001A460023F3E700BFD88B0020A97606084E
:1046A00010B40C4B44681B7803F00303032B06D1B2
:1046B000094B204619885DF8044B1122B6E71123F7
:1046C000237043682D225A70436800229A705DF867
:1046D000044B70474437002060370020094B406886
:1046E0001B7803F00303032B07D1074B7122D3F888
:1046F00070186423B1FBF3F198E704492D2371226C
:1047000040F0B2BC44370020D88B00203735060873
:104710002DE9F04FCE4907780E784468C578172FF9
:1047200091B00CBF4FF0980E4FF0890E16F00406B2
:10473000099004D0C74B172F0CBF5E681E68DFF8C6
:104740003CC386EAE673A3EBE673022DB3FBFCF2EF
:104750000CFB123300F0A281032D15D0012D03D1E3
:104760004FF47A71B3FBF1F3002EBBBF2D216170C2
:10477000601CA01C84F800E0B749B84C002D08BFAD
:10478000214640F071FC1BE122461E2302F8023B49
:104790001F2363700B7813F0040300F07581AD4D97
:1047A000686843F0B7FE9EA3D3E9002343F01CFFE3
:1047B000824628688B4643F0ADFE99A3D3E90023D7
:1047C00043F012FFA64B002206460F4644F092F932
:1047D00008B9A34F0026A34B00223046394644F0C7
:1047E0007FF908B99F4F00269E4B0022304639467C
:1047F00044F06CF940B9304639468BA3D3E9002325
:1048000043F03AFD06460F46DFF874924FF0000879
:10481000954B00225046594644F058F9002840F084
:10482000EA80DFF85C924FF00008904B002250467F
:10483000594644F05FF9002840F0E6808C4B0BAA03
:1048400003F1100C18685968154603C50833634511
:104850002A46F7D11B882B80304675A3D3E9002365
:10486000394643F0C1FE74A3D3E9002343F006FDAB
:1048700044F050FA72A3D3E9002307468846504615
:10488000594643F0B1FE70A3D3E9002343F0F6FC90
:1048900044F040FA4FF00F0905460E460DF12C0A80
:1048A0004FF0FF3B052200233846414644F0CEF945
:1048B00005F00303069306F000430793DDE90601C4
:1048C000002871F100030BDA069B13F1FF33069306
:1048D000069B63F0030101314BF10003069107933E
:1048E000644B03EB8202069B1A44384692F89B31D4
:1048F00009F80A3005220023414644F0A7F9002DAB
:10490000884676F1000107462A46334602DAEA1C59
:1049100046F1000309F1FF399508B9F10A0F45EA9C
:1049200083754FEAA306BDD14FF0000A28463146F1
:104930001422002344F08AF94E4B1A44384692F868
:104940009B3110AA4A44069202F8143C41461422B4
:10495000002344F07BF9474B1A44384692F89B31C8
:10496000069A414602F8153C1422002344F06EF9E1
:1049700014220746884628463146002344F066F94B
:10498000A9F1020B05460E46BAF1000F7AD110AB21
:104990005B444FF02B02A9F1030903F8142C0AF130
:1049A000010ABAF1050FC1D10BAA631C04F10D0174
:1049B00012F8010B03F8010F9942F9D10023A373F8
:1049C000099B2D491B785A0901EB820103F01F0353
:1049D000012202FA03F31E4AD1F87408127802F099
:1049E0000602042A0CBF034320EA0303C1F874380B
:1049F00011B0BDE8F08F5046594642464B4643F051
:104A00003DFC82468B4603E75046594642464B469C
:104A100043F032FC82468B4607E700BFAFF30080CD
:104A200048AFBC9AF2D77A3E2D431CEBE236EA3E01
:104A30000000000084D77741000000D088C3E04127
:104A40000000000000405F410000000000F9D54177
:104A500044370020483700205936060851360608EA
:104A6000008056C000805640008066C000806640CE
:104A70007736060858B90508D88B0020809698002C
:104A800000807640D9468AE74FF02D31C4F80210F5
:104A9000516091602B22A272A37391E73C2101FB2C
:104AA00003F52046B5FBFCF40CFB14535943172FB8
:104AB000B1FBFCF500F801EB0CFB15130C49B3FB43
:104AC000F1F310D1002EB4BF5721452105912221C9
:104AD000CDE903312723CDE9004306490295082398
:104AE00040F0C2FA6CE7002EB4BF53214E21EDE72F
:104AF00040420F0061360608F8B52D4F0A24B7F979
:104B0000002092FBF4F484EAE473A3EBE4739BB219
:104B10005A2B054605D90A32CCBFB4236FF0B30334
:104B20001C1B244E96F8842332B9234B1B78DB07D9
:104B300029D417F0DFFE30BB96F88038B32B02D8AB
:104B400017F0D8FEF8B9B7F902100A2391FBF3F376
:104B500004B9C3B1002BB8BF5B4284EAE4709BB2D6
:104B6000A0EBE470B3EB400F6A6813DAB0EB430FCD
:104B700010DA092908DD002CCCBF6E2362231370E4
:104B80006B6800225A70F8BD002CCCBF6A236623E4
:104B90001370F5E7834205DD0929CCBF6023682344
:104BA0001370EDE7002CCCBF6C2364231370E7E790
:104BB0002C380020D88B0020DA36002030B585B0A4
:104BC000054601A83FF052FA044618B9287020465D
:104BD00005B030BD044A0123B2F9842801A9284652
:104BE00040F058FAF3E700BFD88B00204068E5E7B3
:104BF00073B50D4D0091044616460023024602216E
:104C0000286833F0AFFD094B009322462868002343
:104C1000142133F0A7FD28680096002322461621B0
:104C200033F0A0FD02B070BD4C520020BA780608E7
:104C30002DE9F04704468AB0E8B1B24B1868037A10
:104C40009C422246A8BF1A469C42B8BF0132A3EB41
:104C5000020303EBD373B4BF01210021C3F3470464
:104C600049B1A94B0093224600230221651C33F071
:104C700079FDEDB22C46DFF8E882A44FDFF8E4922C
:104C80000026454617F8013BD8F85C1101229A40EE
:104C90000A4230D0172B2ED8DFE813F0180034006A
:104CA0004D0077008D00B000D100F200120121010B
:104CB00066015B0078012D008A01A101B601C101E6
:104CC0009D00D101F50100021302E9010DF1080A6E
:104CD0005046FFF773FF18B98D49504640F0C4F9AC
:104CE0008848CDF800A0006800232246022133F056
:104CF00039FD0134E4B20136182EC3D120460AB082
:104D0000BDE8F087B5F84E21002312F00F021946D6
:104D100018BF012202A8FEF749FFB5F84E3103F093
:104D20000F027C4B03EB82032046D3F8C81102AA82
:104D3000FFF75EFFDDE7B5F85021012312F00F0207
:104D400018BF1A46002102A8FEF730FFB5F850310F
:104D5000E5E7D5F80808FDF797F895F84D31DFED50
:104D60006E7A6E4A002B0CBF0F230C230193012394
:104D700020EE270A0093002102A8FFF73BFA6849BA
:104D800002AA2046FFF734FFB3E7664B1B681906FB
:104D9000B1D5B5F9FC07FDF75FF80246FDF750F80D
:104DA0006149034602A840F05FF9604902AA204623
:104DB000FFF71EFF9DE75B4B1B681A069BD5B5F9F5
:104DC0000C1802A80022FFF731FC594902AA20461C
:104DD000FFF70EFF8DE7534B1B681B068BD5D5F8ED
:104DE0007018642302A8B1FBF3F10022FFF71EFC48
:104DF000504902AA2046FFF7FBFE7AE7B5F9FE37D5
:104E0000DFED457A454A00EE103AB8EEC00A4FF0A1
:104E1000060E0123CDE9003E20EE270A02230021E1
:104E200002A8FFF7E7F995F8B101434B434902AAFD
:104E3000002808BF19462046FFF7DAFE59E7B5F803
:104E40000038DFED357A354A00EE103AB8EEC00A88
:104E50004FF0060C0123CDE9003C20EE270A022387
:104E6000002102A8FFF7C6F995F8B101344B354986
:104E700002AA002808BF19462046FFF7B9FE38E706
:104E8000FEF7E8F907EE900AB8EEE70ADFED227ABE
:104E9000224A01230620CDE9003020EE270A022312
:104EA000002102A8FFF7A6F995F8B101264B274982
:104EB00002AA002808BF19462046FFF799FE18E706
:104EC00002A995F80408F8F77FFD214902A846F0E9
:104ED00006FC204902AA2046FFF78AFE09E71E4B7E
:104EE0009B7A002B3FF407AFB5F902280E499A23AD
:104EF00002A840F0B9F8194902AA2046FFF778FE47
:104F0000F7E600BF4C520020C936060808BB05086A
:104F1000D936060858B905080AD7233CA9760608E9
:104F2000E0360608CC370020ED360608F2360608D3
:104F3000FC3606080937060896360608893606083C
:104F4000AF360608A2360608B3360608BB36060892
:104F50000936060819370608A43700202237060844
:104F6000D88B0020C1370608654B9B7A002B3FF495
:104F7000C2AE644A64499268072302A840F074F8FC
:104F8000624902AA2046FFF733FEB2E695F8E13700
:104F9000002B3FF4B0AE032B3FF4ADAE5C4902A84A
:104FA00040F062F85B4902AA2046FFF721FEA0E626
:104FB000594B1B6899077FF59EAE01234722CDE927
:104FC00000325649564A91ED060A02A80021FFF721
:104FD00011F9544902AA2046FFF70AFE89E6B5F9FD
:104FE0001408FFF7AFF895F84D314749002B0246FA
:104FF0000CBF0D230E2302A840F036F84A4902AA3E
:105000002046FFF7F5FD74E602A9D5F81808F8F771
:10501000DBFC464902AA2046FFF7EAFD69E6B5F83F
:105020001C28434902A840F01FF8424902A846F054
:1050300056FB414902AA2046FFF7DAFD59E63F4BED
:105040001B689B007FF557AE3D4B1A8A4AB13D491C
:1050500002A840F009F83C4902AA2046FFF7C8FD23
:1050600047E63A4A38492046FFF7C2FD41E6B5F91E
:105070001E28374902A83FF0F7FF364902AA20460A
:10508000FFF7B6FD35E602A9D5F8C807F8F79CFC8E
:10509000314902AA2046FFF7ABFD2AE63C21D5F8AC
:1050A000CC37B3FBF1F302A8B3FBF1F201FB1233EF
:1050B0002A493FF0D9FF2A4902AA2046FFF798FD66
:1050C00017E695F84D31D5F8D02773B940F249610C
:1050D0007E23B2FBF1F202A80B493FF0C5FF02AA02
:1050E00049462046FFF784FD03E64FF47A717D239D
:1050F000B2FBF1F202A804493FF0B6FFEFE700BFB0
:10510000A4370020C0370020ED3606082E370608E9
:10511000373706083D37060834380020D093002082
:10512000A976060846370608523706085F3706088C
:105130002D740608093606086B370608CC370020A0
:10514000B844002074370608793706088237060805
:10515000613506088B37060898370608A637060813
:10516000AF3706082DE9F043744B1F6883B0002F5A
:1051700056D0FF238DF803308DF80230002877D108
:105180006F4B93F88628002A4DD093F8B851002D24
:1051900046D06C4A93F88C186B48536992F810808B
:1051A00000294FF0000103F0010C14BF4FF00F0E67
:1051B0008E4600F1F0020B460F4612E0984554D39C
:1051C000BCF1000F51D174461E260133DBB21680AC
:1051D0009770D4700131A94222D0062B02F104024B
:1051E0001ED050F8044B2404F4D5002BE6D17446AD
:1051F0007826EAE7012203EB82027169D2F83C22A9
:105200000192CA077CD593F88C38002B14BF0F236A
:10521000002301A94FF400408DF80730FDF73AF85C
:1052200003B0BDE8F083474EB3F8882841F2286107
:105230008A42DFD941F24F618A4263D941F27661F5
:105240008A4261D941F29D618A4262D941F2C561C7
:105250008A426FD941F2EB618A426DD941F21271F3
:105260008A4294BF0B220D22C5E700242646ACE7F4
:10527000344E0DF102020C4638460DF1030109F0DF
:10528000E0FE06F11001384609F0D8FE06F11401DF
:10529000384609F0CDFE9DF803909DF802804946FE
:1052A0004246384609F04AFE7569317C244B05F0C8
:1052B000010505EB410505EB091593F88628A3F8D0
:1052C000880805EB0825ADB202BBB3F88A28AA42CC
:1052D00021D0A3F88A580F22206893F88C5800F543
:1052E0004331013AD2B201F5A07185F0010083F893
:1052F0008628216083F88C08002A7FF446AF92E765
:10530000FF2386E7022276E7032274E7A3F88A5890
:10531000E2E704226FE7216893F88C08A3F88A2853
:1053200001F5433202F5A07280F00101226083F89A
:105330008C1879E706225EE70A225CE72437002012
:10534000D88B002000060020948D002038B504463C
:1053500002214FF4FA7032220123E17040F203156A
:105360000021E080A5802281A372217010202AF004
:10537000B1FC607038BD00BFF0B55C4C5C4DD4F83A
:1053800090282B68DFED5B6A5B4E2968C4F89018A3
:105390009B1A07EE903AF8EE677AB7EE007A67EE5E
:1053A000A67A3378F4EEC77AF1EE10FA88BFF0EE01
:1053B000477A04F6940213F0010383B0C2ED007A39
:1053C0000CD14E4A4E491278A4F84631D2070B80D0
:1053D0002FD4012384F8B43803B0F0BD01AB6A4682
:1053E00004F69C0104F69800F8F75CFD4348454933
:1053F000019B009A0078424FA1FB02C281FB03C1CE
:10540000DB17C3EB61135209C1073A80A4F8463198
:10541000DFD533782D68DB0761D594F8C3373A4E72
:105420008BBBF3890F2B30D8B068D4F8A038C11AE1
:1054300005E0354ED4F8A038B0682D68C11AD4F80C
:10544000B028C4F8A0084FF47A73AA1A03FB01F33A
:1054500040F2DC5193FBF2F31BB28B422B4AC4F8AF
:10546000B058A8BF0B469342B8BF1346D6E90021F7
:10547000A4F8AC380123C4F8A818C4F8A42884F808
:10548000B43803B0F0BDB389CCE7214901AB081FA4
:105490006A46F8F707FD94F8C337B0684BB9D4F8FB
:1054A000A038009AC11AD4F870381344C4F8703880
:1054B000C5E7D4F8A038DDED007AC11AF8EE677AB6
:1054C00007EE101A67EEA77AB8EEC77AE7EE077A0A
:1054D000B1EEE77AFCEEC77A17EE902AE3E70A4EC0
:1054E000D4F8A038B068C11AA9E700BFD88B002053
:1054F000282C00206F12833A44370020DA3600202F
:10550000603700201F85EB514837002024FAFFFF49
:105510008094002070B330B583B040F25514AA23B4
:105520000022ADF800408DF803308DF802108DF8A0
:1055300004200DF1010401AD55235A400821530008
:1055400012F0800F08BF520083F0310314BFDAB2AB
:10555000D2B20139F3D1AC4202D014F8013BECE7EE
:10556000AA2369468DF803208DF80430F6F738FE3B
:1055700003B030BD704700BFF0B590F860309BB00D
:1055800004467BB9416843694A7883F84420C87867
:105590008A78012142EA0022A3F8462083F84810C5
:1055A0001BB0F0BD466902E030682BF0C1FE3068E8
:1055B0002BF0C6FE05460028F6D12946642201A834
:1055C00046F085F81549164B164E1868D1F8BC38C8
:1055D000039391F8B8188DF85B5003441791049326
:1055E00011496369B578114F029740F2FF50CDE938
:1055F0000513ADF804005DB97078642202FB006009
:1056000001A9043046F002F8012263697570B27096
:105610001868FF211BB0BDE8F0407BE7D88B002065
:10562000282C0020145B002029250108D45A0020D2
:1056300090F8602062B910B50378032B29D0042BB1
:1056400012D0022B1C4C08D0002384F8C83810BD9F
:10565000194B002283F8C8287047012384F8C93801
:10566000002384F8C83810BD4368017E5B78124C73
:105670000120814203F00F0384F8C90810D00229E9
:10568000E2D1002BE0D0162084F8CA2825F0F8FBE0
:10569000DAE7094C002384F8C92884F8C83810BD1B
:1056A0002BB1152084F8CA1825F0EAFBCCE71620A8
:1056B00025F0E6FBC8E700BFD88B002070B50B4C87
:1056C00005460E46D4F8C8062BF036FE0028F9D061
:1056D000D4F8C80631462BF037FE2DB12878314674
:1056E000D5223EF037FD287070BD00BFD88B00205A
:1056F00070B50A4C4FF0FF3504F528762068E03489
:1057000040B190F83830142B04D02BF015FE8542B0
:1057100028BF0546A642F1D1284670BDAC4F0020F7
:1057200008B5054B93F8CB380BB1002008BD01211B
:105730000DF0F0FC002008BDD88B002010B50E4AFB
:105740000E4B92F8CC280E495C781B780978012A18
:1057500082B00CBF10220D2222441E330424027298
:1057600043728DF8044021B901210DEB0400F6F7D6
:105770006FFD02B010BD00BFD88B0020A04F0020ED
:105780003A370020F0B58BB00D46109E30461C46CF
:10579000174642F065FD134B8DF806502344032253
:1057A0009B798DF804201E28A8BF1E2003F03F031C
:1057B000220648BF43F0400302460546314602A890
:1057C0008DF807308DF8057045F020FF064B1B78EB
:1057D00013B100200BB0F0BD291D01A8F6F738FD6C
:1057E0000BB0F0BDA04F00203A37002010B584B0B8
:1057F00003AC00949DF818408DF80C4000248DF8FF
:105800000D40FFF7BFFF04B010BD00BF00B5094B4E
:1058100083B01B7804228DF804201BB1002003B054
:105820005DF804FB01210DEB0200F6F711FD03B05A
:105830005DF804FB3A37002000B5094B83B01B78B4
:1058400002228DF804201BB1002003B05DF804FB98
:10585000012101A8F6F7FCFC03B05DF804FB00BFD2
:105860003A37002000B5084B83B01B7801218DF832
:1058700004101BB1002003B05DF804FB01A8F6F78B
:10588000E7FC03B05DF804FB3A37002000B5074B96
:1058900083B01B7800208DF804001BB9012101A8FA
:1058A000F6F7D6FC03B05DF804FB00BF3A370020E2
:1058B000ECE700BF0B4B197049B101290CD003294B
:1058C000094814BFC722F722012133F0E1B9064885
:1058D0004722012133F0DCB903488722012133F04C
:1058E000D7B900BF563900201C3D0020184B70B5B9
:1058F0001D78044625BB09B9284670BD154E96F89B
:10590000A917D6F8D008003918BF0121F5F7BAFA5F
:105910000028F1D1104B1B78DB0713D50F4B96F8FD
:10592000D5181A7E96F8D43812F0400F14BF102202
:105930000D220A441E33012522726372284670BD6F
:10594000044EEBE7012042F049F941F04FFFE5E753
:1059500055390020D88B0020DA36002000060020C0
:1059600008B5064B1B78DB0700D508BD012042F0C7
:1059700035F9BDE8084041F039BF00BFDA360020F4
:10598000044B18780B4600B970471146D8B241F065
:105990007BBE00BF553900203FF0CABE0F2A07D892
:1059A00008B508461146029A3FF09EFE002008BD49
:1059B0000020704708B5054B93F8DF380BB1002085
:1059C00008BD42F08BF9002008BD00BFD88B002035
:1059D00070B5184C94F8D63894F8E05833B345F0C5
:1059E0000805154E84F8E058737EAB420AD0328920
:1059F0001248002145F06BFE114875762A460421B5
:105A000033F046F994F8D81894F8D7083FF0AEFE72
:105A100094F864350B48C3EB031300EB43104FF4C9
:105A2000F072202145F053FE002070BD05F0F7050F
:105A3000D7E700BFD88B002000060020BC940020D0
:105A40001C3D00205839002030B5A0F17D03012B0A
:105A5000044683B00D46104608D921462BF074FC4D
:105A600015B1288804442C8003B030BD7D210192FB
:105A70002BF06AFC019884F020012BF065FCEFE725
:105A800030B50F4B85B0D3F8C42A00230446C51D9A
:105A9000ADF80E3014F8010B01920DF10E01FFF775
:105AA000D3FFA542019AF5D10DF10E0011F0EEF8E9
:105AB000019A9DF80E000021FFF7C6FF05B030BD2A
:105AC000D88B0020044AD2F8C83A43F4DF2343F4C9
:105AD0008063C2F8C83A7047D88B0020013070B597
:105AE000094EC4B203E03FF09BFB013448B9E5B274
:105AF000152D21463046F6D9162D04BF034B93F8D9
:105B0000CC5A284670BD00BFA0960020D88B00203C
:105B100000B1D7E7044AD2F8C83A23F4DF2323F4CC
:105B20008063C2F8C83A7047D88B002070B5104E19
:105B300084B00446D6F8D00A0D4625F03FF80D4B48
:105B40001A795B79003A18BF01220BB142F00802C2
:105B5000CDE9015200234FF4964194F900000091E1
:105B60001A46082125F0C7F8C6F8D00A04B070BD5F
:105B7000D88B00206437002010B5064C03E0D4F821
:105B8000D00A2BF0D5FBD4F8D00A2BF0D9FB002893
:105B9000F5D110BDD88B002010B50D4CD4F8D43AF7
:105BA0001B791E3B012B0DD9D4F8D00A01213830C6
:105BB000FFF7BCFF0023C4F8D83A84F8DC3ABDE80C
:105BC0001040D9E7D4F8D00A01212BF0A9FBF1E766
:105BD000D88B002070B5094E054633685E200C4610
:105BE0009847336828469847E0B2FCF761F8C4F359
:105BF0000720BDE87040FCF75BB800BFD88B0020E1
:105C000003682DE9F041002B3C4D3D4F3D4EB8BFA0
:105C10005B42A5FB0321890D07FB0137C7EB071783
:105C2000BF00B37985FB0725FA170446C2EBA555DB
:105C3000002B56D101EB810101EB810105EB8101C4
:105C400009B2DFF8BC801320FFF7C4FF2E4908FB20
:105C5000057581FB0531ED17C5EBA11109B21B20BC
:105C6000FFF7B8FF2368254D002BB4BF53214E2109
:105C70002320FFF7AFFF6368B27983EAE376A6EBF0
:105C8000E376A5FB0631890D08FB0168C8EB08180F
:105C90004FEA880885FB08354FEAE873C3EBA55542
:105CA0002ABB01EB810101EB810105EB810109B206
:105CB0001220FFF78FFF124B134903FB058581FB71
:105CC0000531ED17C5EBA11109B21A20FFF782FFCC
:105CD0006368002BBDE8F041B4BF57214521222065
:105CE00078E7C1EB011105EB810109B2A9E7C1EB2E
:105CF000011105EB810109B2DAE700BF6BCA5F6BE6
:105D0000806967FF64370020D34D6210F0B5464CC0
:105D100094F8DD3A012B83B0054650D994F8DE0A99
:105D20004249434E94F8DF7A421CA1FB02C1184459
:105D300006EB800001F4FE7606EB9101521AD0F8D2
:105D4000D86184F8DE2A2FB1D4F8E01A04F6E422F0
:105D500091420DD06EB9374A0133A2FB031222F0F3
:105D6000010101EB52029B1A84F8DD3A03B0F0BD49
:105D7000314E94F8F83A93B9304B019348F2A501AB
:105D8000123B15226F46A4F8FC1A009384F8FE2AF1
:105D900029463846B04758B994F8DD3ADBE76F46F4
:105DA00038460DF0A7F829463846B0470028F3D00A
:105DB00094F8F81A59B138460DF016F8ECE71C4A79
:105DC00002EB8302D2F8D861002EC4D0D1E7009E46
:105DD0001B4A964214D9013A013E41F2210512F8BC
:105DE000013F81EA0321082311F4004F85EA4100B5
:105DF0000ABF490081B289B2013BF5D19642EED18A
:105E000038463DF0EFFC0F49009D6D1A152DA8BFD7
:105E100015252A4601F1180045F0F8FB94F8DD3A03
:105E200084F8295B97E700BFD88B0020CDCCCCCC81
:105E300058B90508ABAAAAAA19290108E9960020B1
:105E4000D7960020D496002070B50C4E054606F675
:105E50002E31D5223EF05CF92C686C6006F62C31B0
:105E6000641A182CA8BF18242960224606F644306C
:105E700045F0CCFB86F85C4B70BD00BFD88B002092
:105E80002DE9F84FDFF868B00024824689460BF50B
:105E90003667A04650260CE001352C44EFF3118301
:105EA00086F31288DBF8C02B944217DADBB283F357
:105EB00011880BEB0403601C93F8605B384429469F
:105EC0000022FAF745FE0028E6D049465046FAF788
:105ED00075FD40EA08005FFA80F8DDE70022DBB2DA
:105EE000CBF8C02B83F311884046BDE8F88F00BF84
:105EF000D88B0020F0B58BB004461F4B1F4A2049B9
:105F0000009302A81F4B3FF0AFF826680025731CD2
:105F10002360357023682922591C21601A70236878
:105F2000EA22591C21601A702368C822591C21607A
:105F300002A81A7042F094F9471C02A93A46206858
:105F400045F064FB236829461F440C2300E02768C2
:105F50007A1C013B22603970F9D12268511C216002
:105F6000137023680122991821601A7023689B1B03
:105F700033700BB0F0BD00BF83930020FC2E0608E9
:105F8000F42F0608EC2F060870B505682B4E002389
:105F90006A1C02602B7003682122591C01601A7070
:105FA0003378DB0704461DD5254B1B8859050FD5D3
:105FB000244920463DF0A0FB3378DB071CD523683D
:105FC0000022591C21601A7023685B1B2B7070BD66
:105FD0001A0523D4D80523D4D90723D49A0723D567
:105FE0001949E6E7194B1B6863B1194920463DF092
:105FF00083FB3378DB07E2D423682A22591C216013
:106000001A70DCE7134B1B681806CDD5124B1B78B2
:1060100003F00303032BC7D01049CAE71049C8E7B0
:106020001049C6E71049C4E7104B114993F8F4270B
:10603000104B002A18BF1946BBE700BFDA36002014
:10604000D03700209E35060800300608D4720020A4
:1060500004300608CC370020443700200C300608F6
:10606000143006081830060820300608D88B0020A7
:10607000C13506082830060838B50368204D591C7C
:1060800008222DED028B01601A7003689FED1D8AB6
:10609000591C1E2201601A70B5F9023007EE103A41
:1060A000B8EEC77A044627EE087ABDEEC77A17EE37
:1060B000103A99B23DF070FBB5F9003007EE103A96
:1060C000B8EEC77A204627EE087ABDEEC77A17EEFB
:1060D000103A99B23DF060FBB5F9043007EE903A02
:1060E000F8EEE77A204667EE887ABDEC028BFDEE8B
:1060F000E77A17EE903A99B2BDE838403DF04CBBD4
:106100002C38002058A08B4138B50368214A5D1C0B
:106110000A2105601970036808215D1C056019706B
:10612000D37A044663B31EF0B3FE1B490530A1FBCE
:106130000031C1F3CF0120463DF02EFB174D184929
:106140002B6881FB0321DB17C3EBA10189B2204639
:106150003DF022FB1EF0AAFEAD6823682A0C591CF4
:1061600021601A7023682A0A591C21601A7023685A
:106170005A1C22601D7023685A1C2260187038BD9A
:10618000084A054B11880531A3FB0131C9083DF0D0
:1061900003FBD3E764370020CDCCCCCCC037002044
:1061A000676666668837002003681122591C70B53F
:1061B00001601A7003681C4D1C4E5A1C02600222BA
:1061C0001A70044629683DF0CFFA696820463DF010
:1061D000CBFAE98901EBC10189003231A6FB01311B
:1061E000C1F34F1120463DF0D7FA298A01EB810116
:1061F000490089B220463DF0CFFA0D4A0D4B116897
:106200009942A8BF194621EAE171A6FB013149096B
:1062100001F57A7189B220463DF0BEFA23682A7DE5
:10622000591C21601A7070BD483700201F85EB5142
:10623000CC72002020A10700F8B50B4D0B4F06468D
:106240002946D5223DF064FF34687460A91E641AA3
:10625000402CA8BF40243160224607F6C43045F0E8
:10626000D5F987F8044CF8BD663E0020D88B002095
:1062700030B50B4B0B4D43F8405C83B0C822014650
:10628000A3F13B0403F83C2C68463A2201930094A6
:106290003DF044FA6846FFF7CFFF03B030BD00BFC2
:1062A000A43E0020C83E7BEA70B5404B404D1B68C1
:1062B000590582B004460BD495F8093C0F2B15D82C
:1062C0003C4A3D4902EB8303D3F8F4318B420DD0B5
:1062D00095F8083CDA0731D49B0705D5D5F80C0CA6
:1062E000201AB0F57A6F13D202B070BD334B019310
:1062F000C821A3F13F0203F8401C68460092FFF753
:10630000F9FD6846FFF798FF0FF02EF802B070BD58
:1063100095F8093CD5F8100C0F2B97BF254A264954
:1063200002EB8303D3F8F41103681B69984795F8CF
:10633000083C6FF3410385F8083CD5E71F4A95F800
:10634000091C1F480192C3F382030F2902F8393C4C
:1063500040F6C8238CBF0021012122F83C3C712368
:10636000A2F1400602F83A3C02F8381CA2F13703C9
:10637000A2F13E0142F8400C6846BA2200933DF07B
:10638000C7FE009B721C9B1A73706846FFF754FF90
:106390000EF0EAFF95F8083CC5F80C4C23F0030317
:1063A00043F0020385F8083C02B070BDCC370020F2
:1063B000D88B002058B90508A0680600A43E00202C
:1063C000C80032EC034B1B6A30EA030314BF012000
:1063D0000020704764370020AF4A38B508200023FA
:1063E0005371FFF7EFFF40B113684FF48064022050
:1063F0004FF482611C80507159804FF40020FFF7E8
:10640000E1FF38B1537911685C1C40F201405471CE
:1064100021F81300A1494B7A002B59D18B7A002B1C
:1064200040F00A814FF40070FFF7CCFF38B1537988
:1064300011685C1C4FF40460547121F81300984BF0
:106440001968880700F1B880490700F19880954BDA
:106450001B681B0657D45379934913714FF480304E
:1064600000234B715371FFF7ADFF28B10B6801207A
:106470004FF4047248711A804FF40040FFF7A2FFF6
:1064800038B14B790A685C1C4FF400704C7122F8EB
:1064900013004FF40030FFF795FF38B14B790A68CD
:1064A0005C1C4FF4A0604C7122F813004FF4802064
:1064B000FFF788FF38B14B790A685C1C4FF43760EE
:1064C0004C7122F813004B790B7100234B7138BDCE
:1064D0000120FFF777FF0028A0D04FF48030FFF7AE
:1064E00071FF38B9537910685D1C4FF4047455710D
:1064F00020F81340537910685D1C4FF411645571F6
:1065000020F813408AE74FF40050FFF75BFF38B1E3
:10651000537911685C1C4FF40360547121F8130027
:106520004FF48050FFF74EFF60B153791068591C4B
:106530001D46C9B24FF40064023320F81540537170
:1065400020F811404FF48040FFF73CFF38B15379F9
:1065500011685C1C4FF48460547121F813004FF4EF
:106560008060FFF72FFF00283FF475AF5379116863
:106570005C1C4FF40260547121F813006BE74FF478
:106580008060FFF71FFF38B1537911685C1C4FF42E
:106590008070547121F813004FF40060FFF712FF70
:1065A00000283FF454AF537911685C1C4FF4887095
:1065B000547121F813004AE78020FFF703FF38B138
:1065C000537910685D1C45F23024557120F8134052
:1065D0004FF48070FFF7F6FE38B1537910685D1CF8
:1065E00045F24024557120F813401020FFF7EAFED1
:1065F00038B1537910685D1C4FF4E064557120F890
:1066000013402020FFF7DEFE38B1537910685D1C7F
:106610004FF4E264557120F813404020FFF7D2FE9A
:1066200000283FF411AF537910685D1C4FF4E46407
:10663000557120F8134007E70220FFF7C3FE00283A
:106640003FF4F0AE4FF40040FFF7BCFE38B9537989
:1066500011685C1C4FF40070547121F81300042081
:10666000FFF7B0FE38B1537911685C1C4FF4C0607D
:10667000547121F813004FF48010FFF7A3FE002897
:106680003FF4D0AE537911685C1C45F25020547130
:1066900021F81300C6E600BFF8050020A43700204B
:1066A00034380020CC370020F005002003685A065B
:1066B00007D513F4057F04D007298CBF00200120E3
:1066C000704703F48253B3F5825F03BFC81FB0FA6B
:1066D00080F040090020704770B5BC4C94F8143C21
:1066E000012B84B000F04C8194F8210CFDF702F9E5
:1066F00094F8223C834205461FD0002800F0D78042
:10670000D4F8D43ACBB1B24A93F904005279002AB2
:1067100018BF08224FF4964100230325CDE901520A
:1067200000911A46082124F0E6FAC4F8D00A20B1F4
:10673000FFF732FA012384F8223C94F8233C012B22
:1067400000F0C280D4F82C6C3EB1A24B3046597890
:10675000FFF7ACFF002840F0F28094F8310CFDF711
:10676000C9F894F8303C8342054622D0002800F056
:10677000F680F6B1337A002B00F01781964A02EBCF
:106780008303D3F8F431924A96F904001279009306
:10679000003A18BF012200230221CDE901121A4656
:1067A000102124F0A8FA8D4B186010B1012384F851
:1067B000303CD4F8346C3EB1864B30465978FFF704
:1067C00075FF002840F0AB8094F8400CFDF792F87C
:1067D00094F8383C8342054623D0002800F0C78057
:1067E000FEB1337A002B00F0E3807B4A02EB830397
:1067F000D3F8F431764A96F9040012790093003AFE
:1068000018BF012202210023CDE901121A464FF4DC
:10681000007124F070FAC4F83C0C10B1012384F824
:10682000383C94F8410CFDF765F894F8423C8342FB
:10683000054630D088B36A4BD4F8446C4FF47A7272
:10684000C3F86C243EB34FF480524021304624F00C
:10685000E1F90546F8B95E4B96F904001B79002B67
:1068600014BF0921082103224FF4E133CDE90121AE
:1068700000932A462B464FF4805124F03CFAC4F88A
:10688000480C40B15749584A84F84C5C01230860D1
:10689000157084F8423C04B070BDD4F8480C24F064
:1068A0008DF9C4F8485C84F8425C04B070BDD4F83B
:1068B000D00A24F083F994F8233CC4F8D05A012B71
:1068C00084F8225C7FF43EAF94F8240CFDF712F8B4
:1068D000054600286FD0D4F8C43A002B7FF432AFBD
:1068E000D4F8282C002A3FF42DAF394992F904003E
:1068F0004A790979002A14BF08220022002908BF1A
:1069000042F0010203254FF46141CDE901520091AB
:106910001A46202124F0EFF9C4F8C40A12E794F8CB
:10692000383C002B7FF47DAFD4F81C3C002B3FF4A7
:1069300078AF0122C4F83C3C84F8382C71E794F815
:10694000303C002B7FF435AFD4F81C3C002B3FF4D7
:1069500030AF224901220B6084F8302C29E71F4E0A
:10696000306824F02BF9356084F8305C21E7D4F8E6
:106970003C0C24F023F9C4F83C5C84F8385C50E704
:10698000D4F8185C134B28465978FFF78FFE68B38C
:10699000D4F8D436002B7FF4A7AED4F81C3C002BDF
:1069A0003FF4A2AEC4F8D4369EE64FF49643EAE62E
:1069B0004FF461431EE7D4F8C40A00283FF4C2AE86
:1069C00024F0FCF8C4F8C45ABCE600BFD88B002001
:1069D00064370020805B002058B90508BC72002095
:1069E0000006002008710020E070002094F8200CC0
:1069F000FCF780FF0646D8B1D4F8D436002B7FF4DC
:106A000073AE002D3FF470AE0E4A95F90400127972
:106A1000B2FA82F252094FF416510225CDE9015221
:106A200000911A46042124F066F9C4F8D4065BE606
:106A3000D4F8D40600283FF457AE24F0BFF8C4F8C9
:106A4000D46651E664370020F8B5C44C94F8143C81
:106A5000002B00F0A181082024F0F0F8C4F8D40A3B
:106A600000283CD0082124F0DFF800260346BC496A
:106A7000BC4884F8213C0522C4F8546C31F046FE31
:106A800041F208530122B748A4F8583C84F85C2C22
:106A90000AF0CEF931462B22B34844F018FE48F6EE
:106AA0007C607D25E02331462B22A4F8640CAF489E
:106AB00084F8673C84F88F5C44F009FE48F67C213A
:106AC000A0224EF27B0384F8BB5C84F8966384F8C2
:106AD0003F54A4F8901C84F8932CA4F8943394F8B1
:106AE000233C002B00F02481102024F0A7F8102173
:106AF000C4F82C0C24F098F89D4D9E4B84F8310C72
:106B000040F23B113A2019806A7A18719F214AF2AB
:106B10001E409971002198601973002A40F0EF809F
:106B2000AB7A002B64D1944E33685A0700F1E080B1
:106B30009F0700F1D480180700F1CA808F4F386892
:106B4000C0F3C010FEF7E4FF0020FEF7C7FF0346C6
:106B50004FF4007084F8CC3A24F070F84FF40071D0
:106B6000C4F8340C24F060F8D4F8BC3C84F8400C31
:106B7000002B14BF0123002384F8C03C77D1D4F844
:106B8000103C002B14BF0123002384F8C93C36D1EC
:106B9000D4F8E82C0023C4F8C03B002A00F0BE80E3
:106BA000012284F8F83A84F8EC2C002374487549E3
:106BB000C4F8E83A062231F0A9FD40F609437048CE
:106BC000A4F8EC3A0AF034F94FF4805024F036F887
:106BD0004FF48051C4F8440C24F026F8002384F8C4
:106BE000410C84F8423CF9F78FFFBDE8F84073E5AB
:106BF000D4F8C83A43F00403C4F8C83A93E73168BC
:106C0000002311F0020184F8CA3C84F8CB3C40F028
:106C1000EB806B7A2BB10120FFF7D4FB002840F00A
:106C2000DD80AB7A002B40F0D3800820FFF7CAFB51
:106C300020B16318042283F8CC2C01313B681B0679
:106C400000F1F280092042F2090384F8D01C84F894
:106C500061054D494D48A4F8DC3C2025042284F808
:106C6000625531F053FD49480AF0E2F890E76B7A3B
:106C70002BB10120FFF7A6FB002840F0A580AA7ADF
:106C8000002A40F0DE803B68190600F1B6803168CA
:106C90004B070CD54FF48060FFF794FB38B1A31875
:106CA000082183F8C41C013284F8C82C67E7080760
:106CB00005D54FF40070FFF785FB0028EFD10905DB
:106CC000F2D54FF40060FFF77DFB0028ECD0E6E73B
:106CD000D4F8C83A43F48073C4F8C83A2EE7D4F81D
:106CE000C82A42F4601242F0C002C4F8C82A22E75F
:106CF000D4F8C82A42F40272C4F8C82A18E7D4F8B3
:106D0000C83AAA7A43F00201C4F8C81A002A3FF42C
:106D10000AAF43F03603C4F8C83A04E7D4F8F03CAD
:106D2000002B4CD0012384F8EC3C84F8F83A3CE783
:106D3000202023F083FFC4F8280C00283FF4D4AEB1
:106D4000202123F071FF124B124A1A6084F8240CA0
:106D5000FFF742FB012384F8233CC5E6D88B0020D3
:106D60008CBB0508289800203C98002068980020DB
:106D7000A4370020EC62002034380020CC370020FB
:106D8000BC96002034BC0508E0BB0508AC98002088
:106D9000C8720020815A0108042023F04FFFC4F874
:106DA000180C00283FF457AE042123F03DFF294A78
:106DB00084F8200C0123226084F8143C4BE684F80C
:106DC000EC3C84F8F83AFFE6012284F8C42C5AE738
:106DD0000620FFF7F7FA00283FF427AF63180222D6
:106DE00083F8CC2C013120E74FF46070FFF7EAFA0A
:106DF00070B3012184F8CC1C0BE74FF4A050FFF7CF
:106E0000E1FA20B1A318022183F8C41C01324FF427
:106E10000850FFF7D7FA00283FF439AFA318042130
:106E200083F8C41C013232E74FF45850FFF7CAFA16
:106E300000283FF407AF6318082283F8CC2C0131F7
:106E400000E70620FFF7BEFA0028BDD102461AE788
:106E50000146DEE69D2801082DE9F04FB24C89B0CD
:106E600005460F46164694F8819329F05BFE82464C
:106E7000002028703070D4F85481387018F0010F59
:106E800049D017F0FDFD002842D0A84B1A68002A0F
:106E90003ED0970104D5B2F1007F18BF02F17E42C7
:106EA000D4F8F41C9FEDA27AAAEB010307EE903A06
:106EB000F8EE677AF4EEC77AF1EE10FA05DCD4F852
:106EC000F80C01238340134212D111B91923C4F8DD
:106ED000F83CD4F8F83CC4F8F4AC012001331A2B88
:106EE00028BF002300FA03F11142F7D0C4F8F83CA0
:106EF000D4F8F82C8F4B904903EB82032846D3F843
:106F000030233EF0B1F80223337009B0BDE8F08FB2
:106F10000023C4F8F43CD4F8FC3C8BB3874B1B78BB
:106F2000D8072DD4D4F8003D9FED857A03F5921350
:106F300003F57863A3EB0A0307EE903AF8EE677A5D
:106F400067EE877AFDEEE77AB8EEE77A17EE903AC9
:106F5000F1EE0C7AB4EEE77AF1EE10FA06DB79493D
:106F600028463EF081F801233370CEE70A212846F7
:106F7000B3FBF1F201FB123373493EF075F8F2E70F
:106F800018F4007F0BD0714BDB7843B17049284671
:106F90003EF06AF80323337001233B70B5E718F025
:106FA000200F09D094F8843333B16A4928463EF063
:106FB0005BF801233370A8E718F4806F34D094F89D
:106FC000043D012B30D1644B1B68990727D5634BD7
:106FD000B3F90220B4F9143DD21A6FF463739A42E4
:106FE00018DB40F28D339A4217DC0A2392FBF3F24E
:106FF0005B4928463EF038F81AF00EFA594B1B68E8
:1070000093F863300A3B23EAE3739842ABDB012336
:107010003B70A8E76FF05902EAE75A22E8E75249C5
:1070200028463EF021F8E7E718F4005F0ED00EF096
:1070300057FA94F84C31834208D94C4928463EF01F
:1070400013F80223337001233B705EE718F4004FFE
:1070500008D0474BB4F9A021B3F90A309A4201DDB8
:107060004449EBE718F4804F07D00EF021FAB4F84A
:107070009E31834201D94049E0E718F0080F04D05F
:10708000B9F1020F01D13D4981E718F4006F0FD02B
:107090002A4B1B78DA070BD517F08AFC40B1384B26
:1070A0001B78DB0704D594F8513D0BB93549C5E78A
:1070B00018F4805F14D0214B1B78D80710D517F037
:1070C00077FC68B12E4B1B78D90709D4D4F8F83770
:1070D000A3F53713A3F5D863002B01DA2A49ADE7EE
:1070E0002A4B1B885A0601D52949A7E718F0800FBB
:1070F00054D0284BB3F9000094F8663198424DDB28
:10710000FDF720F894F84D212349002A0CBF0D22E9
:107110000E220346009228467A223DF0A5FF022364
:10712000337001233B70F0E6D88B0020D47200202E
:107130000024F44858B90508276E0608DA360020FE
:10714000ACC52737D0370608DB370608DC36002009
:10715000E8370608F2370608343800202C380020BB
:10716000FD370608DC720020073806080E380608CE
:10717000000600208F37060817380608243806084E
:10718000443700202E38060839380608D03700204A
:1071900044380608E47200204D380608694B1B6825
:1071A0001B017CD518F0400F79D06749029191F806
:1071B000008004AAC8F109084FEA580800231046C5
:1071C0002021984521D14044604944F0A4FA4FF071
:1071D000000A08F10308D346029B1B785B4502D9DD
:1071E000B8F10B0F15D908AB9844002308F8103CF0
:1071F000BAF1000F53D0564904AA28463DF034FF97
:107200000223337001233B707FE602F8011B013338
:10721000D7E75FFA8BF108460391F9F7B1FA4D4BC6
:10722000039993F800C031311CF0010CC9B234D07D
:10723000B4F962E1BEF1FF3F2FD08289642312FBD3
:1072400003F2454B93F822305B0892FBF3F39E4523
:10725000B4BF0B46522394F9602112F1800F04D081
:1072600090F901E09645A8BF5423BCF1000F08D067
:10727000B4F96421B2F1FF3F03D040689042A8BF47
:10728000432304AA994208F8023018BF0AF1010A00
:107290000BF1010B08F101089EE70B46DBE7D4F880
:1072A000548118F0040F0BD0B9F1010F08D12B490C
:1072B00028463DF0D9FE0223337087F8009024E67B
:1072C00018F4807F08D0234B1B78DA0704D5244BB1
:1072D0001B780BB92349B1E618F4803F0CD01D4B45
:1072E0001B78DB0708D5B4F848312BB11E4A9268E9
:1072F000934201DC1D49A1E618F0020F14D0154B92
:1073000094F881231B7803F0030313430CD11DF081
:10731000BFFD174B5B8A834206D9164928463DF0CC
:10732000A3FE01233370F0E518F0100F3FF4EDAD2C
:1073300094F8543D002B3FF4E8AD0F4928463DF04A
:1073400093FE10E6CC370020F42C0020A43506086C
:10735000276E0608DA3600204C3300205C38060819
:107360004C63002068380608C037002074380608CF
:10737000A43700207D3806088938060807B50023A1
:1073800000F10D020DF1070140688DF80730FFF79D
:1073900063FD9DF80730084A43B1D2F8743843F4CE
:1073A0000013C2F8743803B05DF804FBD2F87438E7
:1073B00023F40013F5E700BFD88B002010B5094B6C
:1073C0000022D3F8041103F58473914201D1002007
:1073D00010BD13F8014B844201D00132F5E70120C2
:1073E000F6E700BFD88B0020F0B404780A4E049F63
:1073F000650906EB850604F01F04012505FA04F46F
:10740000D6F8745804972C428068F0BC18BF43F03B
:10741000800331F0A7B900BFD88B00201D4B2DE9A8
:10742000F04303EB81038FB0D3F8988306460D46F3
:10743000B8F1000F2BD0184B03EB41031C22B3F81B
:1074400086400023194604F01F07C4F344190DEBCE
:107450000200A413069344F03AF901228DF80B4080
:1074600006AC8DF81420CDE903468DF808508DF850
:1074700009708DF80A9002A8C0479DF814200023D7
:107480002AB100944A46394602A8FFF7ADFF0FB073
:10749000BDE8F08358B90508D88B00202DE9F04FDE
:1074A0001D4D90F801808678DFF870B06FF4D173CD
:1074B00085B004462F1D05EB03094FF4FA6A15F950
:1074C000013B002B1EDB09EB8303D3EDCC7AFDEEF1
:1074D000E77A4FF47A7317EE902AA2F57A720AFBD4
:1074E00002F292FBF3F202ABA2F57A725946184609
:1074F0003DF0BAFD02AB00933246002341462046E0
:10750000FFF772FF0136BD42F6B2D8D100232373D4
:1075100005B0BDE8F08F00BF7B8D0020593506080F
:107520002DE9FF47314B477893F8AC2193F8AD81B3
:10753000436885781E2AA8BF1E22022AB8BF0222ED
:10754000B8F1100FA8BF4FF01008B8F1020F4FF0BC
:107550000B01B8BF4FF0020804461970D6B25FFAAB
:1075600088F90121501E4FF0170C8842636826DC11
:1075700013440B2103F8011C616800238B546268DB
:10758000009239462A4620463E44FFF72DFF013E31
:107590004FF0010AF6B208F1FF33534513DC05EB57
:1075A000090263680093013A0023D2B239462046AB
:1075B000FFF71AFF0023237304B0BDE8F08703F838
:1075C00001C00131D1E705EB0A02D2B216233946D8
:1075D00020460392F6F7AAFE039A16233146204668
:1075E000F6F7A4FE0AF1010AD5E700BFD88B002008
:1075F0002DE9F0433A4B9FED3B7A2DED028B93ED55
:10760000088AF0EEC87AF4EEC77AF1EE10FA85B087
:1076100004465DD5D3ED077AF0EEE76AF4EEC76A6B
:10762000F1EE10FA54D5304B0293304B0393304BAC
:10763000DFED308AB3F90230DFED2F6A002BD8BFBF
:10764000F1EE677A77EEA87ABAEE0C7AA7EEA67A10
:10765000D6BF00250125B1EE488A17EE100A40F08A
:107660006BFF41EC100B42F097FA38EE288A9FED41
:10767000237AFAEE007AE8EE077A59EC108B17EECF
:10768000900A40F059FF41EC100B42F085FA57EC9C
:10769000106BA07840F03EFF32463B4640F0EEFDD6
:1076A00041F03CFAC6B2607840F034FF42464B46A7
:1076B00040F0E4FD41F032FA04AB03EB8505C1B2C2
:1076C00055F8083C0093324600232046FFF78CFE15
:1076D0000023237305B0BDEC028BBDE8F08300BF2F
:1076E000309900206C61D83E93380608AB35060807
:1076F0002C380020DB0F493F539A8E4183F92241F9
:107700002DE9F04F184F91F8018091F80290DFF8C1
:107710005CA0DFF85CB085B006460C4600253B78DF
:10772000AB4204DC0023237305B0BDE8F08F28468C
:10773000B04702AB504502465946A8BF52461846CC
:107740003DF092FC04AB1844002109EB050202ABAA
:1077500000F8081CD2B2009320460B464146FFF7C2
:1077600043FE0135DBE700BFF42C00209F860100BB
:107770002D74060801460148C2E700BF0534010820
:1077800001460148BCE700BF8D330108F8B5364D0E
:10779000364C2A6800239007C4F8043108D503202A
:1077A000FAF7D0FA2A20FAF7CDFA3C20FAF7CAFA0B
:1077B0002F4F002617F8010B0136FAF7C3FA312EC6
:1077C000F8D12B68990617D50E20FAF7BBFA0D20D1
:1077D000FAF7B8FA1820FAF7B5FA1720FAF7B2FA5A
:1077E0001F20FAF7AFFA1E20FAF7ACFA2F20FAF7AB
:1077F000A9FA3A20FAF7A6FA1E4D2B681A011DD4F1
:107800001D4B9B7903BB3B20FAF79CFA94F87C3D17
:1078100043B31A4B1A4F1D680121284630F094FFDC
:10782000284630F0C5FF0026D4F804319E4212D31A
:1078300028460021BDE8F84030F086BF2320FAF743
:1078400081FA2B681B01DBD52420FAF77BFA332061
:10785000FAF778FAD7E717F8011B2846FFF7DEFD9D
:107860000136E1E7F8BD00BF34380020D88B002096
:10787000E8BD0508CC3700204C3300204C520020D6
:10788000E08C0020074B032883F8680103D8064AE0
:10789000012308B9137079E7013803FA00F010707A
:1078A000F9E700BFD88B00200006002070B53F4BE1
:1078B0003F4C1B783F4D03F00103286884F87D3D61
:1078C0000023C4F87438C4F8783803681B6B92B08E
:1078D000002B64D00121984784F87E0D0021286890
:1078E00030F032FF286803685B6C0BB102219847C7
:1078F00028680AAE30F05CFFF4F7E8FC2E4A2F4906
:1079000030463DF0B1FB0096002306221421286882
:1079100030F028FF2A4B0093082200230721286813
:1079200030F020FF274B0093092200230B21286809
:1079300030F018FF244B0093286800230A220B2103
:1079400002AE30F00FFF3046FDF738F930B128684D
:10795000009600230C22052130F004FF29F0E2F804
:1079600094F8683100F5741000F51060032BC4F82A
:10797000800D03D8154901229BB90A7094F87E3D09
:1079800084F87C3D0023C4F80431FFF7FFFE28682B
:1079900030F0C8FE012384F8843D12B070BD184653
